:100000000C9474250C944D9E0C94229E0C94F79D98
:100010000C94CC9D0C94A19D0C94769D0C944B9DBE
:100020000C94209D0C94A5250C94A5250C94A52535
:100030000C94A5250C94EFA40C94A5250C94A5254F
:100040000C94A5250C94B0B70C94A5250C94A5256B
:100050000C94A5250C94A5250C940CE60C94DA9F21
:100060000C94A5250C940F790C94A9790C94A525D2
:100070000C94A5250C94A5250C94A5250C94A525D8
:100080000C94A5250C94A5250C94A5250C94A525C8
:100090000C94A5250C94A5250C94A5250C94A525B8
:1000A0000C94A5250C94A5250C94A5250C94A525A8
:1000B0000C94A5250C94A5250C94A5250C94A52598
:1000C0000C94A5250C94A5250C94A5250C94A52588
:1000D0000C94A5250C94A5250C94A5250C94A52578
:1000E0000C94A52542794879597964796C7981799C
:1000F000707981797479787981797E7987998A990B
:1001000079997D998399C1998E99929998999C9999
:10011000A099A699AA99AE99C199B499B899BC9990
:10012000F69EFB9E009F0A9F149F8D9F1E9F269FF9
:100130002E9F389F429F4C9F5B9F659F8D9F6F9F17
:10014000799F839FD5EDD5EDDCEDDCEDDCEDE3EDC6
:10015000E3EDE3EDF0EDEAEDEAEDEAED084AD73B39
:100160003BCE016E84BCBFFDC12F3D6C74319ABD86
:1001700056833DDA3D00C77F11BED9E4BB4C3E91AA
:100180006BAAAABE000000803F05A84CCDB2D44E99
:10019000B93836A9020C50B9918688083CA6AAAA9B
:1001A0002ABE000000803F004E414E494E4954593E
:1001B000494E46CDCCCC3D0AD7233C17B7D1387732
:1001C000CC2B329595E6241FB14F0A000020410048
:1001D00000C84200401C4620BCBE4CCA1B0E5AAE92
:1001E000C59D74434F4D4D554E49434154494F4E63
:1001F0000044525952554E004552524F52530049F5
:100200004E464F004543484F00556E6B6E6F776EFC
:1002100020636F6D6D616E643A20220041637469E2
:1002200076652045787472756465723A20004E6F69
:100230002063617365206C696768740A00000000C0
:100240000000000000000000004F666673657473D4
:10025000206170706C696564004572723A20546F59
:100260006F206661722100546F6F20666172206694
:10027000726F6D207265666572656E636520706F62
:10028000696E740A00FFFFFF4B64200023646566FB
:10029000696E65202044454641554C545F004B69CA
:1002A000200023646566696E6520204445464155FB
:1002B0004C545F004B70200023646566696E6520B6
:1002C0002044454641554C545F00504944204175F7
:1002D000746F74756E652066696E697368656421F4
:1002E0002050757420746865206C617374204B70A5
:1002F0002C204B6920616E64204B6420636F6E7309
:1003000074616E74732066726F6D2062656C6F77B6
:1003100020696E746F20436F6E66696775726174D1
:10032000696F6E2E680A00504944204175746F74DD
:10033000756E65206661696C6564212074696D6500
:100340006F75740A00544845524D414C2052554E29
:100350004157415900546865726D616C2052756E49
:10036000617761790048656174696E6720666169CB
:100370006C65640048656174696E67206661696CCC
:10038000656400504944204175746F74756E652032
:100390006661696C6564212054656D706572617475
:1003A00075726520746F6F20686967680A00204B5A
:1003B000643A2000204B693A2000204B703A20001C
:1003C0000A20436C617373696320504944200A001A
:1003D0002054753A2000204B753A2000206D61783A
:1003E0003A2000206D696E3A200020643A200020F7
:1003F000626961733A200043290A0061626C656496
:1004000020286D696E2074656D702000436F6C64E8
:1004100020657874727564657320617265200020B0
:10042000643A0020693A0020703A0020643A0020C3
:10043000693A0020703A00205A00205900580020E4
:10044000204D61783A2000205A00205900580020A1
:10045000204D696E3A20004F6E20004F66660053B3
:100460006F667420656E6473746F70733A20007ADF
:100470005F6D696E3A2000795F6D696E3A20007891
:100480005F6D696E3A20005265706F7274696E67B5
:1004900020656E6473746F70207374617475730A71
:1004A000002F2F2000454D455247454E43595F5080
:1004B000415253455200434153455F4C49474854CC
:1004C0005F4252494748544E45535300544F4747A3
:1004D0004C455F4C494748545300534F465457418D
:1004E00052455F504F574552004255494C445F506A
:1004F000455243454E54004C4556454C494E475F86
:1005000044415441005A5F50524F424500415554B6
:100510004F4C4556454C005052494E545F4A4F424D
:100520000050524F4752455353004155544F524586
:10053000504F52545F54454D5000564F4C554D4509
:100540005452494300454550524F4D00534552497E
:10055000414C5F584F4E5F584F4646004649524DFA
:10056000574152455F4E414D453A4D61726C696E3F
:1005700020204649524D574152455F5645525349F6
:100580004F4E3A312E312E382E353920455854529F
:10059000554445525F545950453A4D4F415273743A
:1005A000727564657220534F555243455F434F4403
:1005B000455F55524C3A68747470733A2F2F636FCD
:1005C00064652E616C6570686F626A656374732E12
:1005D000636F6D2F646966667573696F6E2F4D4129
:1005E000524C494E2050524F544F434F4C5F56454A
:1005F0005253494F4E3A312E30204D414348494ED7
:10060000455F545950453A4C756C7A426F7420548A
:10061000415A20352045585452554445525F434F66
:10062000554E543A3120555549443A6333323535A5
:100630006339362D343039372D343838342D386518
:1006400064302D6465643266663962616536310AEC
:10065000004C756C7A426F742054415A2035204FFB
:1006600066662E002F2F616374696F6E3A70617534
:1006700073650A0042656420646F6E652E00205722
:100680003A004265642068656174696E672E0042B5
:10069000656420636F6F6C696E672E006F6B00047A
:1006A00002FF01F801F101E3016F66660044454273
:1006B00055473A0045787472756465722025730059
:1006C000000125301D0CFF24311C0BFF232F1B0ABA
:1006D000FFFF040308060202222B1A4142033809D5
:1006E000FF3628294527444350726F74656374654B
:1006F000642050696E0A002569730025696D202504
:100700006973002569682025696D202569730025B6
:100710006964202569682025696D20256973002595
:10072000697920256964202569682025696D20255F
:100730006973005072696E742074696D653A2000A7
:1007400046696C652064656C657465643A0044654F
:100750006C6574696F6E206661696C65642C2046F7
:10076000696C653A20006F70656E206661696C6522
:10077000642C2046696C653A20004D3132350045C5
:100780006E642066696C65206C6973740A0042654A
:1007900067696E2066696C65206C6973740A005223
:1007A0006573756D696E67207072696E74004C7543
:1007B0006C7A426F742054415A203520726561640E
:1007C000792E00436C69636B20746F2072657375BA
:1007D0006D652E2E2E00536C6565702E2E2E0047F3
:1007E000322F47332062616420706172616D6574DD
:1007F0006572730A0020746F6F206C6F6E672065DE
:100800007874727573696F6E2070726576656E7438
:1008100065640A0020636F6C642065787472757378
:10082000696F6E2070726576656E7465640A004546
:10083000313A200045303A20005A3A2000593A20F7
:1008400000583A20004D53312C4D53322050696EE0
:10085000730A004572726F722077726974696E67ED
:1008600020746F20454550524F4D210A001FFFFF55
:10087000FFFFFFFF600000000001FF4000000000DC
:1008800000FF8000000000007F83CF00000C303F9D
:1008900087FF80000C301F867980000C000F8C30A1
:1008A000C7838C30E78C30CFC7CC31F38C30DCEC95
:1008B000EC33B98C30D86C6C33198C30D06C0C3371
:1008C000198C30D86C0C33198C30DC6C0E3B198CC5
:1008D00030CF7C079F198C30C77C038F19400000F4
:1008E00000000002600000000000061FFFFFFFFF85
:1008F000FFF82020506C616E6E6572427566666509
:100900007242797465733A20002046726565204D05
:10091000656D6F72793A2000436F6D70696C656424
:100920003A204D617920323320323031380A0020AC
:100930007C20417574686F723A2028416C6570683C
:10094000204F626A6563747320496E632E2C204CBD
:10095000756C7A426F7420476974205265706F73AA
:1009600069746F7279290A004D617920323320321F
:1009700030313831303A30323A343400204C6173FF
:100980007420557064617465643A2000312E312EF4
:10099000380A004D61726C696E0020536F6674777F
:1009A0006172652052657365740A00205761746333
:1009B00068646F672052657365740A002042726F25
:1009C000776E206F75742052657365740A00204538
:1009D000787465726E616C2052657365740A00509C
:1009E0006F77657255700A0073746172740A0065DE
:1009F00072726F722077726974696E6720746F20EB
:100A000066696C650A00456E6473746F70732025A7
:100A10006320256320256320256300205A3A0020A7
:100A2000593A0020583A00656E6473746F707320F1
:100A30006869743A2000446F6E6520736176696E50
:100A4000672066696C652E0A004D323900534420D8
:100A500063617264206F6B0A006F70656E526F6F16
:100A600074206661696C65640A00766F6C756D65EB
:100A70002E696E6974206661696C65640A0053446E
:100A800020696E6974206661696C0A006175746F13
:100A900025692E67004D3234004D32332025730016
:100AA00057726974696E6720746F2066696C653A65
:100AB00020006F70656E206661696C65642C20464D
:100AC000696C653A20006F70656E206661696C65BF
:100AD000642C2046696C653A200046696C65207379
:100AE000656C65637465640A002053697A653A2011
:100AF0000046696C65206F70656E65643A20006F12
:100B000070656E206661696C65642C2046696C6551
:100B10003A20002066696C653A2000646F696E6750
:100B2000006672657368004E6F772000454E442062
:100B3000535542524F5554494E450A002220706F7A
:100B400073002220706172656E743A220053554220
:100B5000524F5554494E452043414C4C20746172CC
:100B60006765743A22004B494C4C45442E20007472
:100B70007279696E6720746F2063616C6C20737585
:100B8000622D67636F64652066696C6573207769A1
:100B9000746820746F6F206D616E79206C65766566
:100BA0006C732E204D4158206C6576656C206973FE
:100BB0003A004572726F723A00486F6D652058595D
:100BC0002066697273740A00486F6D652058592059
:100BD0006669727374004E6F206D6F76652E0053D8
:100BE00044207072696E74696E6720627974652042
:100BF000004E6F74205344207072696E74696E6782
:100C00000A00436F6F6C696E6720646F6E652E001B
:100C100048656174696E6720646F6E652E002057A9
:100C20003A004578747275646572202573004D3101
:100C3000343520533C696E6465783E206F757420AE
:100C40006F662072616E67652028302D31290A0099
:100C5000205A3A0020593A0020436F756E7420588C
:100C60003A0020453A00205A3A0020593A00583AB2
:100C7000003A004361703A0025753A25303275001C
:100C8000253032753A2530327500257564202530BF
:100C900032753A253032750000060900FE0000006A
:100CA000000001090008FE000005080806000040D9
:100CB000F0C88888987810050808060000C0F888F1
:100CC00088888888F80505050600012030F830205E
:100CD0000508080600002070F820202020E0050903
:100CE000090600FF2070A8A8B888887020050909A7
:100CF0000600FFE080C0B0A82830282805090906B2
:100D000000FFF8A88888888888A8F8050A0A0600DD
:100D1000FE205050505088A8A88870030303060096
:100D20000340A04000060900FE0701920321207F36
:100D3000FF07FF07FF00000006000001070706028B
:100D40000080808080800080030202060105A0A050
:100D50000507070600005050F850F85050050707E7
:100D60000600002078A07028F02005070706000084
:100D7000C0C810204098180507070600006090A022
:100D800040A89068020303060104C04080030707DF
:100D900006010020408080804020030707060100F4
:100DA0008040202020408005050506000120A87015
:100DB000A8200505050600012020F82020020303D5
:100DC0000602FFC04080050101060003F80202028E
:100DD000060200C0C005050506000108102040807D
:100DE0000507070600007088888888887003070751
:100DF00006010040C040404040E0050707060000F3
:100E0000708808708080F8050707060000F8102039
:100E1000100808F005070706000010305090F81081
:100E200010050707060000F880F00808887005071D
:100E300007060000708080F08888700507070600AC
:100E400000F8081020202020050707060000708801
:100E50008870888870050707060000708888780801
:100E60000870020505060200C0C000C0C0020606E8
:100E70000602FFC0C000C040800407070600001043
:100E8000204080402010050303060002F800F8040B
:100E90000707060100804020102040800507070654
:100EA0000000708808102000200507070600007069
:100EB000880868A8A870050707060000708888F8E9
:100EC000888888050707060000F08888F08888F081
:100ED0000507070600007088808080887005070776
:100EE000060000F08888888888F00507070600005B
:100EF000F88080F08080F8050707060000F8808001
:100F0000F0808080050707060000708880B8888818
:100F100070050707060000888888F8888888010718
:100F20000706020080808080808080050707060019
:100F30000038101010109060050707060000889018
:100F4000A0C0A090880507070600008080808080F0
:100F500080F805070706000088D8A88888888805D3
:100F600007070600008888C8A8988888050707062C
:100F7000000070888888888870050707060000F0E0
:100F80008888F080808005070706000070888888C0
:100F9000A89068050707060000F08888F0A09088F0
:100FA000050707060000788080700808F00507072D
:100FB000060000F82020202020200507070600005A
:100FC00088888888888870050707060000888888D0
:100FD000888850200507070600008888888888A828
:100FE00050050707060000888850205088880507AC
:100FF0000706000088888850202020050707060083
:1010000000F80810204080F8030707060100E08080
:1010100080808080E00505050600018040201008E2
:10102000030707060100E02020202020E00503033D
:10103000060004205088050101060000F8020202A3
:1010400006020580400505050600007008788878CE
:101050000507070600008080B0C88888F0050505F0
:1010600006000070808088700507070600000808E9
:1010700068988888780505050600007088F88070F3
:101080000507070600003048E040404040050606DE
:101090000600FF7088887808700507070600008042
:1010A00080B0C88888880107070602008000808019
:1010B0008080800308080601FF200020202020A057
:1010C00040040707060000808090A0C0A09003079E
:1010D00007060100C04040404040E005050506000D
:1010E00000D0A8A8A8A8050505060000B0C88888F3
:1010F00088050505060000708888887005060606C4
:1011000000FFF08888F080800506060600FF7888DA
:1011100088780808050505060000B0C880808005AD
:10112000050506000070807008F00407070600003F
:101130004040E040404030050505060000888888B2
:101140009868050505060000888888502005050573
:101150000600008888A8A8500505050600008850EC
:101160002050880506060600FF88888878087005E4
:101170000505060000F8102040F8030707060100E7
:101180002040408040402001070706020080808008
:101190008080808003070706010080404020404097
:1011A0008005020206000268900000000600005A56
:1011B0000059005800092000000000000000000055
:1011C000000000007FFFE0000000000000000000C1
:1011D0000000007000E000000000000000000000BF
:1011E000000061F860000000000000000000000046
:1011F0000041F82000000000000000000000000096
:1012000040F020000000000000000000000000404E
:1012100060200000000000000000000000005801F5
:10122000A07F80000000000000004104005C63A07B
:10123000FFC0000000000000002082005EF7A0FF59
:10124000C0000000000000002082005EF7A0FFC088
:10125000000000000000004104005C63A07F8000EB
:101260000000000000008208005801A07F800000FC
:101270000000000001041000406020FFC0000000DA
:101280000000000104100040F020FFC0000000003A
:1012900000000082080041F820FFC00000000000AC
:1012A000000041040061F8603F0000000000000001
:1012B000000000007000E01E0000000000000001BF
:1012C000FFFF807FFFE00C0000000000000001FF36
:1012D000FF8000000000000000000000000000008F
:1012E000007FFFE0000000000000000000000000A0
:1012F0007000E0000000000000000000000000633B
:101300000C60000000000000000000000000470E1C
:10131000200000000000000000000000004F0F202F
:101320000000000000000000000000005F0FA000AF
:1013300000000000000000000000005E07A07F80A9
:1013400000000000000000410400406020FFC000D9
:1013500000000000000020820040F020FFC00000DC
:10136000000000000020820040F020FFC0000000CC
:10137000000000004104004060207F800000000069
:101380000000008208005E07A07F800000000000CF
:1013900000010410005F0FA0FFC00000000000006B
:1013A000010410004F0F20FFC000000000000000EB
:1013B000820800470E20FFC000000000000000412E
:1013C0000400630C603F000000000000000000000B
:1013D000007000E01E0000000000000001FFFF8020
:1013E0007FFFE00C0000000000000001FFFF800014
:1013F000000053657474696E672054726176656C81
:1014000020416363656C65726174696F6E3A200098
:1014100053657474696E67205265747261637420D9
:10142000416363656C65726174696F6E3A20005345
:10143000657474696E67205072696E7420416363CD
:10144000656C65726174696F6E3A200053657474DF
:10145000696E67205072696E7420616E64205472E8
:101460006176656C20416363656C65726174696F58
:101470006E3A2000526573656E643A200020420087
:101480002050006F6B004B494C4C45442E20004BC4
:10149000494C4C2063617573656420627920746FD8
:1014A0006F206D75636820696E616374697665206D
:1014B00074696D65202D2063757272656E7420638A
:1014C0006F6D6D616E643A200020204E6F7A7A6CE9
:1014D000653A2000200068656174206E6F7A7A6C2E
:1014E000652E00507265737320627574746F6E2080
:1014F000746F005052494E5420504155534544009A
:1015000020204E6F7A7A6C653A2000746F20636FEA
:101510006E74696E75652E2E2E00616E6420707279
:1015200065737320627574746F6E00496E736572B3
:10153000742066696C616D656E74005052494E543A
:10154000205041555345440020204E6F7A7A6C65F7
:101550003A2000200066696C616D656E74206C6FC6
:101560006164005761697420666F72005052494E81
:1015700054205041555345440020204E6F7A7A6CD8
:10158000653A2000200066696C616D656E742065A7
:10159000787472756465005761697420666F7200B3
:1015A0005052494E542050415553454400746F20C9
:1015B000726573756D65005761697420666F72207E
:1015C0007072696E74005052494E54205041555308
:1015D000454400436172642072656D6F76656400F6
:1015E0004361726420696E736572746564001000F3
:1015F000C90210012C014001220170011801B00143
:101600000E01F00104015002FA00B002F0003003B4
:10161000E600D003DC009004D2007005C800A006EC
:10162000BE000008B400B009AA00D00BA000600EF4
:10163000960060118C000015820020197800C01DF2
:101640006E00A0226400B0275A00902C5000003198
:101650004600E0343C0010383200903A2800603CEC
:101660001E00A03D1400803E0A00203F00007C3C8C
:101670003E5E2B3D3F2F5B5D3B2C2A225C004B499D
:101680004C4C45442E200020746F6F206C6F6E67A9
:1016900020657874727573696F6E207072657665F7
:1016A0006E7465640A0020636F6C642065787472E0
:1016B0007573696F6E2070726576656E7465640A05
:1016C0000043616E6E6F74206F70656E207375627B
:1016D00064697220006563686F3A00544845524D52
:1016E000414C2052554E41574159204245440054E7
:1016F0006865726D616C2052756E61776179005416
:101700004845524D414C2052554E41574159204574
:101710003100544845524D414C2052554E4157419D
:10172000592045300000002200250028002B002E03
:10173000003100340002010000050108010B010026
:10174000002100240027002A002D00300033000172
:10175000010000040107010A010505050507050848
:10176000080808020202020A0A0808040404040124
:101770000101010101010103030303030303030446
:101780000707070C0C0C0C0C0C0C0C0202020206D6
:10179000060606060606060B0B0B0B0B0B0B0B01C6
:1017A0000210202008081020401020408002010272
:1017B000010804020101020408102040808040203A
:1017C0001008040201800402018040201008040275
:1017D00001080402010102040810204080010204F3
:1017E0000810204080000020002300260029002C43
:1017F000002F003200000100000301060109010270
:1018000001050800FF060121023520FFFF07FF0642
:10181000FF090050221656808080800080153353C7
:10182000A0A0A00257575050F850F85050025757F8
:101830002070A07028702013355580A040A0200291
:10184000475740A0A040A0A050251353808080128D
:10185000265640808080804012265680404040407E
:10186000800245559060F060900255552020F82088
:1018700020113353604080044151F011335340E054
:101880004002465610102040808012365640A0A0DC
:10189000A0A04012365640C0404040E0024656608C
:1018A00090106080F0024656F02060109060024672
:1018B000562060A0F02020024656F080E010906094
:1018C0000246566080E0909060024656F01020205C
:1018D000404002465660906090906002465660908C
:1018E00090701060122555C0C000C0C011365660FF
:1018F00060006040801236562040808040200343C4
:1019000053F000F0123656804020204080123656A8
:1019100040A020400040015858304898A8A8904066
:1019200030024656609090F09090024656E090E06B
:101930009090E0024656609080809060024656E0AB
:1019400090909090E0024656F080E08080F0024651
:1019500056F080E0808080024656609080B09060B3
:101960000246569090F0909090123656E0404040DB
:1019700040E002465670202020A04002465690A02B
:10198000C0A0A0900246568080808080F00246561B
:1019900090F0F090909002465690D0F0B0B0900247
:1019A0004656609090909060024656E09090E0809D
:1019B00080014757609090D0B06010024656E0908A
:1019C00090E090900246566090402090601236560B
:1019D000E040404040400246569090909090600217
:1019E0004656909090906060024656909090F0F02D
:1019F00090024656909060609090025656888850AB
:101A0000202020024656F010204080F0123656E08A
:101A100080808080E0024656808040201010123680
:101A200056E020202020E016325240A0014151F023
:101A300016225280400244547090907002465680A4
:101A400080E09090E012345460808060024656102E
:101A5000107090907002445460B0C06002465620EE
:101A60005040E0404001455560907010600246567D
:101A70008080E09090901236564000C04040E011C7
:101A800037572000202020A040024656808090E05A
:101A90009090123656C040404040E0025454D0A8C6
:101AA000A8A8024454E09090900244546090906042
:101AB000014555E090E08080014555709070101010
:101AC000024454A0D0808012345460C020C002462A
:101AD000564040E0405020024454909090701234A0
:101AE00054A0A0A04002545488A8A8500244549086
:101AF0006060900145559090709060024454F020D1
:101B000040F0024757304020C02040302216568017
:101B10008080808080024757C02040304020C0062F
:101B2000425250A0FFFFFFFFFFFFFFFFFFFFFFFF3D
:101B3000FFFFFFFFFFFFFFFFFFFFFFFFFFFFFFFFB5
:101B4000FFFFFFFFFF0900502216568000808080B3
:101B5000800146562070A0A070200246562050E01A
:101B60004050A002555588705070880256568850D3
:101B7000F820F8202217578080800080808002475C
:101B8000577080E0907010E0173151A002565670E7
:101B9000A8C8C8A87014355560A06000E00343537E
:101BA00050A050123353E02020143151E002565619
:101BB00070E8D8E8D870173151E015335340A04091
:101BC00012355540E04000E014355540A02040E07B
:101BD000143555C020C020C0162252408001455502
:101BE000909090E08002565678E8E8682828241102
:101BF0005180112252408014355540C04040E014BD
:101C0000355540A04000E0034353A050A002475781
:101C1000808080A060F0200247578080A0D01020F4
:101C20007002475780408060A0F020123656400076
:101C30004080A04002475740206090F090900247BB
:101C40005720406090F0909002475760906090F06D
:101C5000909002475750A06090F0909002475790A4
:101C6000006090F0909002475760906090F09090E4
:101C700002465670A0A0F0A0B00147576090808047
:101C80009060400247574020F080E080F0024757C4
:101C90002040F080E080F00247576090F080E080C4
:101CA000F00247579000F080E080F01237578040F4
:101CB000E0404040E01237572040E0404040E01212
:101CC000375740A0E0404040E0123757A000E040C6
:101CD0004040E00256567048E84848700247575066
:101CE000A090D0B0909002475740206090909060B4
:101CF0000247572040609090906002475760906084
:101D00009090906002475750A0609090906002477A
:101D10005790006090909060123353A040A002460C
:101D20005670B0B0D0D0E0024757402090909090CD
:101D30006002475720409090909060024757609013
:101D40009090909060024757900090909090600221
:101D500057571020885020202002465680E090904F
:101D6000E0800246566090A0A090A0024757402015
:101D70000070909070024757204000709090700261
:101D800047572050007090907002475750A0007045
:101D900090907002465650007090907002475760C5
:101DA000906070909070025454F068B0781135557E
:101DB000608080604002475740200060B0C06002F1
:101DC000475720400060B0C06002475760900060F5
:101DD000B0C060024656500060B0C06012375780F5
:101DE0004000C04040E0123757204000C04040E073
:101DF00012375740A000C04040E0123656A000C045
:101E00004040E0024757A040A01070906002475742
:101E100050A000E0909090024757402000609090C2
:101E200060024757204000609090600247576090E2
:101E3000006090906002475750A000609090600250
:101E400046569000609090601235554000E000408A
:101E500002445470B0D0E002475740200090909068
:101E60007002475720400090909070024757609052
:101E700000909090700246569000909090700148AB
:101E80005820400090907090600147578080E0900B
:101E9000E0808001475790009090709060010507A6
:101EA00000FE0500FB01F220FFFE05FE05FE02001C
:101EB000400215258080800080053242A0A0025596
:101EC0006550F850F8500146562070C030E02002AE
:101ED00055659010204048025565608068906805FF
:101EE0001222808002253540808080400225358086
:101EF00040404080043343A040A003334340E040CF
:101F00000122324080043141E002112180025565F6
:101F10000810204080024555609090906002253561
:101F2000C040404040024555E0106080F0024555F9
:101F3000E0106010E00245552060A0F020024555F9
:101F4000F080E010E00245556080E0906002455569
:101F5000F010204040024555609060906002455569
:101F600060907010600313238000800214248000AE
:101F700080800235452040804020033343E000E06C
:101F80000235458040204080024555E01060004009
:101F90000255657088B8A870024555609090F09021
:101FA000024555E090E090E0023545608080806019
:101FB000024555E0909090E0023545E080E080E0F9
:101FC000023545E080E080800245557080B0907019
:101FD0000245559090F09090023545E0404040E039
:101FE000024555301010906002455590A0C0A09059
:101FF00002354580808080E002556588D8A88888B1
:1020000002455590D0B090900245556090909060F8
:10201000024555E09090E0800146566090909060B7
:1020200010024555E09090E0900245557080601098
:10203000E0023545E0404040400245559090909088
:10204000600245559090A0A04002556588A8A8A8B8
:1020500050024555909060909002455590907010B8
:1020600060023545E0204080E0022535C080808058
:10207000C00255658040201008022535C040404010
:10208000C005324240A0024151F005223280400298
:1020900044547090907002455580E09090E0023476
:1020A00044608080600245551070909070024454E6
:1020B00060B0C0600235452040E0404000465670A8
:1020C000909070106002455580E090909002152528
:1020D00080008080800027374000404040408002E0
:1020E00045558090A0E09002152580808080800278
:1020F0005464F0A8A8A8024454E09090900244547C
:1021000060909060004656E09090E08080004656D7
:10211000709090701010023444A0C080800244542B
:1021200070C030E002354540E04040200244549009
:102130009090700244549090A040025464A8A8501B
:1021400050023444A04040A0004656909090701039
:1021500060024454F02040F0023545604080406009
:102160000215258080808080023545C0402040C017
:1021700005425250A0FFFFFFFFFFFFFFFFFFFFFFE1
:10218000FFFFFFFFFFFFFFFFFFFFFFFFFFFFFFFF5F
:10219000FFFFFFFFFFFF020040FFFFFFFFFFFFFF0A
:1021A000FFFFFFFFFFFFFFFFFFFFFFFFFFFFFFFF3F
:1021B000FFFFFFFFFFFFFFFFFFFFFFFFFFFFFFFF2F
:1021C000FFFFFFFFFFFFFFFFFFFFFFFFFFFFFFFF1F
:1021D000FFFFFFFFFFFFFFFFFFFFFFFFFFFFFFFF0F
:1021E000FFFFFFFFFFFFFFFFFFFFFFFFFFFFFFFFFF
:1021F000FFFFFFFFFFFFFFFF01060D00FE09016665
:1022000002D620FFFE0BFE0AFE0D00602219698037
:102210008080808080800080183363A0A0A0035756
:10222000675050F850F850500259692078A0A070BB
:102230002828F02002596948A85010204050A89042
:1022400002586840A0A040A098906828136380803E
:1022500080113B6B20404080808080804040201176
:102260003B6B804040202020202040408006556568
:1022700020A870A8200455652020F8202011336381
:10228000604080065161F811336340E040025969B3
:10229000080810102040408080025969205088882A
:1022A00088888850200259692060A02020202020A2
:1022B000F80259697088880810204080F80259692E
:1022C000F808102070080888700259691010305002
:1022D0005090F81010025969F88080B0C80808883A
:1022E0007002596970888080F08888887002596906
:1022F000F8081010202040404002596970888888F2
:102300007088888870025969708888887808088879
:102310007011386840E040000040E04011386840EB
:10232000E040000060408002596908102040804071
:10233000201008045464F80000F802596980402015
:1023400010081020408002596970888808102020E9
:10235000002002596970888898A8A8B0807802592E
:10236000692050888888F8888888025969F0484828
:102370004870484848F002596970888080808080A1
:102380008870025969F048484848484848F002595E
:1023900069F8808080F0808080F8025969F8808038
:1023A00080F0808080800259697088808080988861
:1023B000887002596988888888F8888888881239DE
:1023C00069E040404040404040E002596938101008
:1023D000101010109060025969888890A0C0A090D9
:1023E00088880259698080808080808080F80259C6
:1023F000698888D8A8A88888888802596988C8C840
:10240000A8A89898888802596970888888888888D8
:102410008870025969F0888888F080808080015A2D
:102420006A70888888888888A87008025969F08846
:102430008888F0A090888802596970888080700828
:10244000088870025969F8202020202020202002CE
:102450005969888888888888888870025969888836
:102460008888505050202002596988888888A8A8F8
:10247000A8A8500259698888505020505088880276
:102480005969888850502020202020025969F80876
:10249000101020404080F8113B6BE08080808080ED
:1024A00080808080E00259698080404020101008C0
:1024B00008113B6BE0202020202020202020E00875
:1024C0005363205088015161F82A226280400256ED
:1024D00066700878889868025969808080F08888DA
:1024E0008888F00256667088808088700259690872
:1024F00008087888888888780256667088F8808806
:102500007002596930484040F040404040005868EF
:102510007088888878088870025969808080B0C87F
:10252000888888881238684000C040404040E000F9
:102530004A6A1000301010101090906002596980A3
:10254000808090A0C0A09088123969C0404040406F
:10255000404040E0025666D0A8A8A8A88802566667
:10256000B0C8888888880256667088888888700015
:102570005868F0888888F08080800058687888885B
:102580008878080808025666B0C8808080800256A5
:10259000667088601088700258684040F040404083
:1025A0004830025666888888889868025666888807
:1025B000885050200256668888A8A8A850025666FF
:1025C0008850202050880058688888889868088833
:1025D00070025666F810204080F8015B6B182020CE
:1025E0002020C0202020201822196980808080802F
:1025F00080808080015B6BC020202020182020205C
:1026000020C008536348A890FFFFFFFFFFFFFFFFB4
:10261000FFFFFFFFFFFFFFFFFFFFFFFFFFFFFFFFCA
:10262000FFFFFFFFFFFFFFFFFF0D00602219698022
:1026300000808080808080800358682070A8A0A0DF
:10264000A8702002596930484040E0404048B0033B
:10265000566688705050708802596988885050F8C2
:1026600020F820202219698080808000808080806E
:10267000124A6A609080609090601090601A326296
:10268000A0A00359697088A8D8C8D8A88870045732
:1026900067700878887800F80356662850A0A05024
:1026A00028045363F80808163161E00359697088FB
:1026B000E8D8D8E8D888700A5161F8174464609067
:1026C00090600357672020F8202000F80735654008
:1026D000A02040E007356540A04020C02A2262408B
:1026E000800058688888888898E8808002596978CE
:1026F000E8E8E8E868282828262161C0202262400E
:102700008007356540C04040E0045767708888887E
:102710007000F8035666A050282850A0025A6A405C
:10272000C04040E00818283808025A6A40C04040BB
:10273000E01028081038025A6A40A04020A048182B
:1027400028380802596920002020408088887002BB
:102750005A6A40200020508888F88888025A6A10F7
:10276000200020508888F88888025A6A3048002063
:10277000508888F88888025A6A2850002050888833
:10278000F88888025A6A50500020508888F8888853
:10279000025A6A20502020508888F8888802596997
:1027A00058A0A0A0B0E0A0A0B8005B6B70888080AB
:1027B00080808088702040025A6A402000F8808023
:1027C000F08080F8025A6A102000F88080F0808043
:1027D000F8025A6A304800F88080F08080F8025A87
:1027E0006A505000F88080F08080F8123A6A804089
:1027F00000E04040404040E0123A6A204000E040A3
:1028000040404040E0124A6A609000E04040404052
:1028100040E0123A6AA0A000E04040404040E002A0
:102820005969F0484848E8484848F0025A6A285030
:10283000008888C8A8988888025A6A402000708852
:102840008888888870025A6A102000708888888872
:102850008870025A6A3048007088888888887002B8
:102860005A6A28500070888888888870025A6A508E
:10287000500070888888888870035565885020507B
:1028800088015B6B08709898A8A8A8C8C8708002D7
:102890005A6A40200088888888888870025A6A109E
:1028A000200088888888888870025A6A30480088A2
:1028B000888888888870025A6A505000888888887A
:1028C000888870025A6A10200088885020202020B2
:1028D00002596980F0888888F08080800259696098
:1028E0009090A0A0908888B002596940200070089C
:1028F000788898680259691020007008788898686C
:102900000259693048007008788898680259692827
:102910005000700878889868025969505000700813
:1029200078889868025A6A30483000700878889829
:1029300068025666702870A0A85000586870888099
:1029400080887020400259694020007088F8808893
:10295000700259691020007088F8808870025969E7
:102960003048007088F880887002596950500070B3
:1029700088F8808870123969804000C0404040402B
:10298000E0123969204000C040404040E0124969EF
:10299000609000C040404040E0123969A0A000C0F3
:1029A00040404040E0025A6A502060107088888899
:1029B0008870025969285000B0C8888888880259F0
:1029C000694020007088888888700259691020004A
:1029D00070888888887002596930480070888888B3
:1029E0008870025969285000708888888870025958
:1029F00069505000708888888870035767202000CD
:102A0000F8002020015868087098A8A8C8708002B3
:102A10005969402000888888889868025969102080
:102A200000888888889868025969304800888888B2
:102A3000889868025969505000888888889868008A
:102A40005B6B1020008888889868088870005A6A34
:102A50008080B0C88888C8B08080005B6B50500010
:102A600088888898680888700000000000000000CE
:102A70000000000000000000000000000000000056
:102A800000000000000000000000000C000000003A
:102A90000000000C00000000000000120000000018
:102AA00000000023000000000000002100000000E2
:102AB0000000004C800000000000005E800000006C
:102AC0000000009240000000000000A14000000053
:102AD00000000121200000000000027F90000000A3
:102AE0000000020010000000000007FFF8000000D6
:102AF00000000400080000000000080004000000BE
:102B000000000800060000000000100002000000A5
:102B10000000301E010000000000207F8100000046
:102B2000000041FFE0800000000043FCF080000056
:102B30000000873B7840000000018EDBFC60000055
:102B400000010FEBCC20000000021FEDB6100000CA
:102B500000021FDEB6100000000439CD7F0800001F
:102B6000000436E0FF08000000087EC0BB840000BF
:102B700000187F005D86000000107FC0ED8200001D
:102B800000203CC07301000000203B337F010000A7
:102B900000701BE77E03800000C81DEEDE04C0004D
:102BA00000880FDEDC04400001240FDF3C09200018
:102BB000012607DBF8192000027203E7F0139000EA
:102BC000025101FFE02290000489007F8024480028
:102BD0000904801E004824000BFE400000DFF400C2
:102BE00010004000008002001FFFFFFFFFFFFE00FB
:102BF00000000000000000000000000000000000D5
:102C000000000000000000001022103C3C0E1F00DD
:102C100010221004221104001022100822110400B6
:102C2000102210083C110400102210102211040080
:102C300010221020221104001E1C1E3C3C0E040019
:102C40000000000000000000000000000000000084
:102C50000000000000000000000000000000000074
:102C60000000000000000000000000000000000064
:102C70000000000000000000000000000000000054
:102C80000000000000000000000000000000000044
:102C90000000000000000000000000000000000034
:102CA0000000000000004573746570732F6D6D00A7
:102CB0004573746570732F6D6D005A73746570730E
:102CC0002F6D6D005A73746570732F6D6D0059739D
:102CD000746570732F6D6D005973746570732F6D0B
:102CE0006D005873746570732F6D6D005873746543
:102CF00070732F6D6D004D6F74696F6E004F666657
:102D0000004F6E2000456E6473746F702061626FB7
:102D100072740053746570732F6D6D004A65726B29
:102D200000416363656C65726174696F6E0056651E
:102D30006C6F6369747900416476616E63656420C9
:102D400053657474696E67730043616E6E6F7420AF
:102D5000656E746572207375626469723A20000250
:102D60002E2E004D61696E0020204E6F7A7A6C65C0
:102D70003A200020004261636B004D696E696D75F9
:102D80006D2054656D70206973203132302E0048FB
:102D9000656174696E67206661696C656400457879
:102DA0007472756465206D6F726500526573756D20
:102DB00065207072696E7400524553554D45204F21
:102DC0005054494F4E533A0020204E6F7A7A6C652A
:102DD0003A20006368616E6765006F6620746865FD
:102DE0002066696C616D656E740057616974206658
:102DF0006F72207374617274005052494E542050A7
:102E000041555345440020204E6F7A7A6C653A2034
:102E100000200066696C616D656E7420756E6C6F64
:102E20006164005761697420666F72005052494EA8
:102E300054205041555345440020204E6F7A7A6CFF
:102E4000653A20002000506C6561736520776169E8
:102E5000742E2E2E0048656174696E67206E6F7A3D
:102E60007A6C65005052494E5420504155534544A8
:102E700000506C6561736520726573657400505213
:102E8000494E5445522048414C54454400507269C3
:102E90006E7465722068616C7465642E206B696C59
:102EA0006C28292063616C6C6564210A00656E7171
:102EB00075657565696E6720220000004842000054
:102EC000484200004040000000005761726E696E89
:102ED000673A20486F6D696E672042756D702044B7
:102EE000697669736F72203C20310A000202040087
:102EF00000A0400000A040000000400000904300FF
:102F0000008A4300007A432F2F616374696F6E3A21
:102F1000726573756D650A004D36303020486F74E8
:102F2000656E6420746F6F20636F6C6420746F2013
:102F30006368616E67652066696C616D656E740AB1
:102F4000004578747275646572004D6F7665205A1D
:102F5000004D6F76652059004D6F76652058004D05
:102F60006F76656D656E7400436F6F6C646F776E1E
:102F70000046616E20737065656420310046616EA5
:102F800020737065656420310042656400426564A9
:102F9000004E6F7A7A6C65004E6F7A7A6C65004DE0
:102FA00061696E005654726176206D696E005654E8
:102FB000726176206D696E005654726176206D697B
:102FC0006E00566D696E00566D696E00566D696EC5
:102FD00000566D6178204500566D61782045005699
:102FE0006D6178204500566D6178205A00566D61FC
:102FF00078205A00566D6178205A00566D6178200D
:103000005900566D6178205900566D61782059003D
:10301000566D6178205800566D6178205800566DC5
:1030200061782058004D6F74696F6E00416D617852
:10303000204500416D6178204500416D6178205A3E
:1030400000416D6178205A00416D6178205900413E
:103050006D6178205900416D6178205800416D61A3
:1030600078205800412D74726176656C00412D7492
:10307000726176656C00412D7265747261637400D3
:10308000412D7265747261637400416363656C0005
:10309000416363656C004D6F74696F6E0056652DFA
:1030A0006A65726B0056652D6A65726B0056652DF8
:1030B0006A65726B00567A2D6A65726B00567A2DBE
:1030C0006A65726B0056792D6A65726B0056792DB0
:1030D0006A65726B0056792D6A65726B0056782DA1
:1030E0006A65726B0056782D6A65726B0056782D92
:1030F0006A65726B004D6F74696F6E0024F4D43092
:1031000050C38E20C2A24017828B7011127A910D8B
:10311000816CD90AA861E108C75866076151430666
:103120001E4B5D05C145A7041A411104093D9803D2
:10313000713931034036DB0265339102D4305402D9
:10314000802E1D02632CEE01752AC501B028A00156
:10315000102781018F2564012B244B01E0223401CB
:10316000AC211F018D200D01801FFC00841EED008D
:10317000971DDF00B81CD200E61BC600201BBC0058
:10318000641AB200B219A8000A19A0006A189900BE
:10319000D117910040178B00B516840031167E00C0
:1031A000B31579003A157300C7146F0058146A00FC
:1031B000EE1366008813630025135E00C7125B00E0
:1031C0006C12570015125400C111510070114F00BC
:1031D00021114B00D61049008D10470046104400C5
:1031E00002104200C00F4000800F3E00420F3C0022
:1031F000060F3B00CB0E3800930E37005C0E3500F7
:10320000270E3400F30D3200C10D3100900D300057
:10321000600D2E00320D2D00050D2C00D90C2B0059
:10322000AE0C2900850C29005C0C2700350C27000A
:103230000E0C2600E80B2400C40B2400A00B230076
:103240007D0B23005A0B2100390B2100180B2000A5
:10325000F80A1F00D90A1E00BB0A1E009D0A1D00A5
:10326000800A1D00630A1C00470A1B002C0A1B0071
:10327000110A1A00F7091A00DD091900C40919001A
:10328000AB091900920917007B09180063091700A0
:103290004C09160036091600200916000A09150007
:1032A000F5081500E0081400CC081400B808140054
:1032B000A4081400900813007D0812006B08130086
:1032C00058081200460812003408110023081100A3
:1032D0001208110001081100F0071000E0071000AB
:1032E000D0071000C0071000B0070F00A1071000A2
:1032F00091070E0083070F0074070F0065070E008B
:1033000057070E0049070E003B070D002E070E0061
:1033100020070D0013070D0006070D00F9060C002D
:10332000ED060D00E0060C00D4060C00C8060C00EB
:10333000BC060C00B0060C00A4060B0099060C009D
:103340008D060B0082060B0077060B006C060B0047
:1033500061060A0057060B004C060A0042060A00E6
:1033600038060A002E060A0024060A001A060A0079
:103370001006090007060A00FD050900F40509000A
:10338000EB050900E2050900D9050900D00509008F
:10339000C7050900BE050900B5050800AD05080010
:1033A000A50509009C050800940508008C05080087
:1033B000840508007C050800740508006C050700FA
:1033C000650508005D050700560508004E05070065
:1033D00047050700400508003805070031050700CC
:1033E0002A050700230507001C050600160507002F
:1033F0000F0507000805060002050700FB0406008C
:10340000F5040700EE040600E8040600E2040700E5
:10341000DB040600D5040600CF040600C90406003C
:10342000C3040600BD040600B7040600B10405008D
:10343000AC040600A6040600A00405009B040600D8
:1034400095040500900406008A0405008504050023
:10345000800406007A040500750405007004050068
:103460006B04050066040500610405005C040500AA
:1034700057040500520405004D04050048040500EA
:10348000430405003E0404003A0405003504050029
:10349000300404002C040500270404002304050064
:1034A0001E0404001A04040016040500110404009C
:1034B0000D040400090405000404040000040400D1
:1034C000FC030400F8030400F4030400F003040008
:1034D000EC030400E8030400E4030400E003040038
:1034E000DC030400D8030400D4030400D003040068
:1034F000CC030400C8030300C503030024F404D96B
:10350000201BC40C5C0E9804C4095F02650771019E
:10351000F405F900FB04B30048048700C103690007
:103520005803550003034500BE023A0084023100EF
:1035300053022A002902250004022000E4011C0095
:10354000C8011900AF01170098011400840113008D
:10355000710110006101100051010E0043010D00C6
:1035600036010B002B010B0020010B001501090097
:103570000C01090003010800FB000800F30008002B
:10358000EB000700E4000600DE000600D80006009D
:10359000D2000600CC000500C7000500C2000500EF
:1035A000BD000400B9000400B5000400B10004002F
:1035B000AD000400A9000400A5000300A200030060
:1035C0009F0004009B000300980003009500020088
:1035D00093000300900003008D0002008B000300A5
:1035E00088000200860002008400030081000200BF
:1035F0007F0002007D0002007B00020079000200D3
:1036000077000100760002007400020072000100E1
:10361000710002006F0002006D0001006C000200EA
:103620006A000100690002006700010066000100F5
:1036300065000100640002006200010061000100F9
:10364000600001005F0002005D0001005C000100FD
:103650005B0001005A000100590001005800010000
:103660005700010056000100550001005400010000
:1036700053000000530001005200010051000100FE
:10368000500001004F0001004E0000004E000100FC
:103690004D0001004C0001004B0000004B000100F8
:1036A0004A000100490001004800000048000100F4
:1036B00047000100460000004600010045000000F0
:1036C00045000100440001004300000043000100E8
:1036D00042000000420001004100000041000100E2
:1036E000400001003F0000003F0001003E000000DC
:1036F0003E0001003D0000003D0001003C000000D4
:103700003C0000003C0001003B0000003B000100C9
:103710003A0000003A0001003900000039000100C1
:1037200038000000380000003800010037000000B9
:1037300037000100360000003600000036000100AE
:1037400035000000350000003500010034000000A5
:10375000340000003400010033000000330000009A
:10376000330001003200000032000000320001008E
:103770003100000031000000310001003000000085
:1037800030000000300001002F0000002F0000007A
:103790002F0000002F0001002E0000002E0000006E
:1037A0002E0001002D0000002D0000002D00000063
:1037B0002D0001002C0000002C0000002C00000057
:1037C0002C0001002B0000002B0000002B0000004B
:1037D0002B0001002A0000002A0000002A0000003F
:1037E0002A00010029000000290000002900000033
:1037F0002900000029000100280000002800000026
:103800002800000028000000280001002700000018
:10381000270000002700000027000000270001000B
:103820002600000026000000260000002600000000
:1038300026000100250000002500000025000000F2
:1038400025000000250000002500010024000000E4
:1038500024000000240000002400000024000100D7
:1038600023000000230000002300000023000000CC
:1038700023000000230000002300010022000000BC
:1038800022000000220000002200000022000000B0
:1038900022000100210000002100000021000000A2
:1038A0002100000021000000210000002100010093
:1038B0002000000020000000200000002000000088
:1038C0002000000020000000200000002000010077
:1038D0001F0000001F0000001F0000001F0000006C
:1038E0001F0000001F0000001F0001001E0000005C
:1038F0001E0000001E0000001E0000004D38342095
:10390000582059205A20450000060900FE0601896A
:1039100002FE20FFFE07FE06FE0000000600070173
:1039200006060602008080808000800303030601F3
:1039300003A0A0A00507070600FF5050F850F8505C
:10394000500509090600FE2070A8A07028A8702064
:103950000608080600FF40A848102048540805073C
:10396000070600FF609090609890680103030602CC
:10397000038080800207070602FF408080808080ED
:10398000400207070602FF80404040404080050596
:10399000050600008850F85088050505060000203F
:1039A00020F820200204040602FEC04040800501E9
:1039B00001060002F8020202060200C0C004060668
:1039C00006010010102040808004060606010060F9
:1039D000909090906003060606010040C040404071
:1039E000E00406060601006090102040F004060680
:1039F000060100F020601010E00506060600001029
:103A0000305090F810040606060100F080E0101017
:103A1000E00406060601006080E09090600406065F
:103A2000060100F010102040400406060601006068
:103A300090609090600406060601006090907010FF
:103A400060020505060200C0C000C0C002070706EC
:103A500002FEC0C000C040408005050506000018F9
:103A600060806018050303060001F800F8050505ED
:103A7000060000C0300830C004070706010060904F
:103A800010604000400506060600007090A8B08057
:103A900070050606060000205088F888880506068E
:103AA000060000F088F08888F00406060601006031
:103AB0009080809060040606060100E0909090904F
:103AC000E0040606060100F080E08080F0040606AF
:103AD000060100F080E08080800406060601006098
:103AE0009080B090600406060601009090F09090DF
:103AF00090030606060100E040404040E00506064F
:103B000006000038101010906004060606010090B0
:103B1000A0C0A090900406060601008080808080EE
:103B2000F005060606000088D8A8A88888040606BE
:103B300006010090D0B09090900506060600007037
:103B40008888888870040606060100E09090E0806E
:103B5000800407070601FF609090D0B06010040653
:103B600006060100E09090E0909004060606010031
:103B7000609040209060050606060000F820202096
:103B800020200406060601009090909090600406A4
:103B900006060100909090F06060050606060000A1
:103BA0008888A8A8D8880506060600008850202026
:103BB000508805060606000088885020202004064C
:103BC00006060100F010204080F003060606010002
:103BD000E080808080E004060606010080804020AE
:103BE0001010030606060100E020202020E0050357
:103BF000030600032050880501010600FEF80202BA
:103C000002060204804004040406010070909070D3
:103C10000406060601008080E09090E0040404069B
:103C2000010070808070040606060100101070907C
:103C3000907004040406010060B0C070040606061B
:103C40000100205040E040400406060601FE60905E
:103C5000907010600406060601008080E09090904D
:103C60000306060601004000C04040E003080806C5
:103C700001FE200060202020A0400406060601006E
:103C80008080A0C0A090030606060100C04040400E
:103C900040E0050404060000D0A8A8880404040637
:103CA0000100E09090900404040601006090906090
:103CB0000406060601FEE09090E0808004060606F9
:103CC00001FE709090701010040404060100A0D052
:103CD000808004040406010070C030E0040606067B
:103CE00001004040E0405020040404060100909090
:103CF00090700404040601009090606005040406BE
:103D0000000088A8A8500404040601009060609098
:103D10000406060601FE909090709060040404066C
:103D20000100F02040F0030707060100204040801A
:103D30004040200107070602FF808080808080804D
:103D40000307070601008040402040408004020233
:103D500006010350A0FFFFFFFFFFFFFFFFFFFFFF74
:103D6000FFFFFFFFFFFFFFFFFFFFFFFFFFFFFFFF63
:103D7000FFFFFFFFFFFF0000000600070106060629
:103D800002008000808080800406060601FF20700B
:103D9000A0A070200507070600FF304840F0404013
:103DA000F8050505060000A8508850A80506060677
:103DB00000008850F820F8200107070602FF8080E5
:103DC00080008080800407070601FF70806090609B
:103DD00010E0030101060105A006070706000078B0
:103DE0008494A494847803050506010160A0600012
:103DF000E00505050600002850A05028040303062E
:103E00000100F01010040101060102F00607070688
:103E100000007884B4A4A48478040101060105F0AC
:103E20000403030601026090600507070600FF20F7
:103E300020F8202000F803050506010140A02040DD
:103E4000E0030505060101C0204020C00202020671
:103E5000020440800405050601FF9090B0D0800563
:103E6000060606000078E8E8682828010101060235
:103E700002800202020602FE4080030505060101DF
:103E800040C04040E003050506010140A04000E0BD
:103E9000050505060000A0502850A00508080600EA
:103EA000FF40C04050703078100508080600FF4001
:103EB000C04050680810380508080600FFC02040C0
:103EC00030F03078100407070601002000206080E1
:103ED0009060050707060000402020507088880584
:103EE0000707060000102020507088880507070685
:103EF0000000205020507088880507070600002821
:103F00005020507088880507070600005000205098
:103F100070888805070706000020502050708888A8
:103F200005060606000078A0F0A0A0B80408080660
:103F300001FE609080809060204004070706010029
:103F40004020F080E080F00407070601002040F0E8
:103F500080E080F00407070601002050F080E08038
:103F6000F00407070601005000F080E080F003072E
:103F7000070601008040E0404040E00307070601DB
:103F8000002040E0404040E003070706010040A059
:103F9000E0404040E0030707060100A000E0404089
:103FA00040E00506060600007048E848487004072F
:103FB0000706010050A090D0B090900407070601BA
:103FC00000402060909090600407070601002040A8
:103FD0006090909060040707060100205060909068
:103FE000906004070706010050A060909090600464
:103FF00007070601005000609090906005050506D7
:10400000000088502050880408080601FF1070B096
:10401000B0D0D0E0800407070601004020909090C7
:104020009060040707060100204090909090600483
:104030000707060100205090909090600407070643
:104040000100500090909090600507070600001056
:1040500020885020202004060606010080E0909071
:10406000E0800406060601006090A0A090A004076E
:1040700007060100402000709090700407070601B9
:104080000020400070909070040707060100205047
:10409000007090907004070706010050A000709017
:1040A000907004060606010050007090907004079E
:1040B000070601002050207090907005040406004F
:1040C0000070A8B0780406060601FE70808070209B
:1040D0004004070706010040200060B0C0700407DC
:1040E0000706010020400060B0C070040707060109
:1040F0000020500060B0C0700406060601005000A9
:1041000060B0C070030707060100804000C0404057
:10411000E0030707060100204000C04040E003071D
:104120000706010040A000C04040E003060606016B
:1041300000A000C04040E004070706010030601006
:104140007090906004070706010050A000E0909076
:10415000900407070601004020006090906004076B
:1041600007060100204000609090600407070601E8
:10417000002050006090906004070706010050A0E6
:104180000060909060040606060100500060909068
:10419000600505050600002000F800200404040660
:1041A000010070B0D0E00407070601004020009035
:1041B00090907004070706010020400090909070D6
:1041C0000407070601002050009090907004060636
:1041D0000601005000909090700409090601FE202D
:1041E00040009090907090600408080601FE808066
:1041F000E09090E080800408080601FE5000909056
:10420000907090604C696E65204E756D626572208D
:104210006973206E6F74204C617374204C696E65F5
:10422000204E756D6265722B312C204C61737420A9
:104230004C696E653A200053544F505045442E202F
:10424000005072696E7465722073746F707065646B
:104250002064756520746F206572726F72732E20F2
:1042600046697820746865206572726F7220616E8D
:104270006420757365204D39393920746F2072655B
:1042800073746172742E202854656D706572617448
:104290007572652069732072657365742E2053658D
:1042A000742069742061667465722072657374612C
:1042B0007274696E67290A004E6F20436865636BEC
:1042C00073756D2077697468206C696E65206E75F2
:1042D0006D6265722C204C617374204C696E653A76
:1042E0002000636865636B73756D206D69736D6124
:1042F0007463682C204C617374204C696E653A209D
:10430000004D313130004D3331005344207265612E
:1043100064206572726F720A00446F6E652070725D
:10432000696E74696E672066696C650A0020496E63
:1043300076616C69642065787472756465722000BA
:10434000000000000000000000000000000090439A
:1043500000008A4300007A4348617264636F6465B9
:10436000642044656661756C742053657474696E6D
:104370006773204C6F616465640A0028230000287D
:104380002300006400000010270000000096430096
:10439000009643000040400000C8410000C94200B0
:1043A00000C9420000C84400804F44204400204916
:1043B0000020204D3330342050002044002049009C
:1043C00020204D3330312050005049442073657413
:1043D00074696E67733A0A00204600204200204844
:1043E0000020204D3134352053004D6174657269D1
:1043F000616C2068656174757020706172616D65B3
:10440000746572733A0A00205A0020590020204D2A
:10441000323036205800486F6D65206F66667365D0
:10442000743A0A00204500205A0020590020580004
:1044300020420020540020204D32303520530041CE
:104440006476616E6365643A20533C6D696E5F66A5
:10445000656564726174653E20543C6D696E5F747D
:10446000726176656C5F66656564726174653E2035
:10447000423C6D696E5F7365676D656E745F7469EC
:104480006D655F75733E20583C6D61785F78795F2C
:104490006A65726B3E205A3C6D61785F7A5F6A652F
:1044A000726B3E20453C6D61785F655F6A65726B3B
:1044B0003E0A0020540020520020204D323034208B
:1044C0005000416363656C65726174696F6E20288A
:1044D000756E6974732F7332293A20503C7072697B
:1044E0006E745F616363656C3E20523C72657472EA
:1044F0006163745F616363656C3E20543C747261F8
:1045000076656C5F616363656C3E0A002045002040
:104510005A0020590020204D3230312058004D6182
:1045200078696D756D20416363656C65726174694E
:104530006F6E2028756E6974732F7332293A0A00E2
:10454000204500205A0020590020204D32303320D1
:1045500058004D6178696D756D206665656472619E
:104560007465732028756E6974732F73293A0A0075
:10457000204500205A0020590020204D3932205873
:104580000053746570732070657220756E69743A9B
:104590000A0020204D3230302044300A0020204DC7
:1045A0003230302044002044697361626C65640AD3
:1045B0000046696C616D656E742073657474696E14
:1045C00067733A0020204D3134392043203B205579
:1045D0006E69747320696E2043656C736975730A24
:1045E000002020473231202020203B20556E697466
:1045F0007320696E206D6D0A00290A0020627974AB
:1046000065733B20637263200053657474696E6741
:10461000732053746F726564202800202863616CD6
:1046200063756C6174656429210A0020213D2000B6
:10463000454550524F4D20435243206D69736D6183
:10464000746368202D202873746F726564292000BC
:10465000290A002062797465733B2063726320002D
:104660002073746F7265642073657474696E677308
:1046700020726574726965766564202800204D613A
:10468000726C696E3D563437290A002845455052F0
:104690004F4D3D00454550524F4D20766572736930
:1046A0006F6E206D69736D6174636820004D6F7665
:1046B0006520617869730044697361626C65207379
:1046C00074657070657273004D3834004175746F95
:1046D00020686F6D6500473238004D61696E004D8E
:1046E0003530320A4D353030004C6F6164207365CF
:1046F0007474696E677300526573746F72652066B7
:1047000061696C736166650053746F7265207365CF
:104710007474696E677300416476616E63656420CA
:1047200053657474696E6773004D61696E00466C01
:104730006F7700466C6F770046616E207370656519
:104740006420310046616E2073706565642031001D
:1047500042656400426564004E6F7A7A6C65004E73
:104760006F7A7A6C65005370656564005370656597
:1047700064004D61696E004D6F76652058004D6F85
:1047800076652059004D6F7665205A004578747221
:1047900075646572004D6F766520302E316D6D0049
:1047A0004D6F766520316D6D004D6F76652031302F
:1047B0006D6D004D6F766520617869730045787482
:1047C0007275646572004D6F7665205A004D6F7684
:1047D000652059004D6F76652058006265640A00B7
:1047E0002C2073797374656D2073746F70706564B9
:1047F00021204865617465725F49443A200048652C
:104800006174696E67206661696C65642042454425
:104810000048656174696E67206661696C65640053
:1048200048656174696E67206661696C65640048FB
:10483000656174696E67206661696C6564204530E6
:10484000001000AD0330016A0150022B0170030A11
:10485000019004F500B005E500D006D800F007CEC1
:10486000001009C500300ABE00500BB700700CB133
:1048700000900DAB00B00EA600D00FA200F0109D6E
:104880000010129900301395005014920070158E8C
:104890000090168B00B0178700D0188400F01981A3
:1048A00000101B7E00301C7B00501D7900701E76AE
:1048B00000901F7300B0207000D0216E00F0226BBA
:1048C00000102469003025660050266300702761BF
:1048D0000090285E00B0295C00D02A5900F02B56C9
:1048E00000102D5400302E5100502F4E0070304BD0
:1048F0000090314800B0324500D0334200F0343EE1
:104900000010363B00303737005038330070392EF6
:1049100000903A2900B03B2300D03C1B00F03D1131
:1049200000103F0100F03F00004572723A204D49EF
:104930004E54454D5020424544004D494E54454D3E
:104940005020747269676765726564004572723AD7
:10495000204D494E54454D50204531004572723A24
:10496000204D494E54454D50204530004572723A15
:10497000204D415854454D5020424544004D41582A
:1049800054454D50207472696767657265640045CF
:1049900072723A204D415854454D502045310045E2
:1049A00072723A204D415854454D502045300020F8
:1049B0002F002042403A0020403A004D363030204F
:1049C0004230005072696E742070617573656400C6
:1049D0004D31323500004D3234005072696E742012
:1049E00061626F72746564004E6F2053442063618E
:1049F0007264005072696E742066726F6D20534449
:104A00000053746F70207072696E740041626F752C
:104A100074204669726D7761726500526573756DB9
:104A200065207072696E74005061757365207072D4
:104A3000696E74004368616E67652066696C616DBC
:104A4000656E7400436F6E66696775726174696F35
:104A50006E0054656D7065726174757265004D6F9E
:104A600076656D656E740054756E6500496E666F8F
:104A70002073637265656E0000000A0B02090C0D5D
:104A80000E08070304010000000000000000000001
:104A90000000000000000000000000000000000016
:104AA00000000000121110000000000000000000D3
:104AB0000000000000000000000000000000486F3F
:104AC0006D652025732573257320666972737400E4
:104AD0002066697273740A005A0059005800486FC2
:104AE0006D652000DD9137AF11241FBECFEFD1E2FD
:104AF000DEBFCDBF00E00CBF13E0A0E0B2E0EEE20D
:104B0000F4EF01E00BBF02C007900D92A23FB10786
:104B1000D9F725E1A2EFB3E001C01D92A132B2079F
:104B2000E1F715E2C3E7D5E200E006C021970109ED
:104B3000802FFE010E9488F9C237D10780E0080764
:104B4000A9F70E94FF4B0C9406FA0C9400002F92D8
:104B50003F924F925F926F927F928F929F92AF920D
:104B6000BF92CF92DF92EF92FF920F931F93CF935A
:104B7000DF93CDB7DEB7C15CD1090FB6F894DEBFC5
:104B80000FBECDBF8091B6048D3409F443C6843581
:104B900011F40C94D53F873411F00C941640809199
:104BA000B4049091B5048A31910509F4F3C57CF4FD
:104BB000843091053CF4823091057CF597FF26C046
:104BC0000C943040049709F49EC50C9430408A350B
:104BD000910509F416C66CF48B31910509F4E1C511
:104BE0004C9711F00C94304080E00E948B5E0C9446
:104BF00030408B35910509F408C68C35910511F0CC
:104C00000C9430400E940A5E0C9430408091200247
:104C100081110C9433400C943040209120022223C7
:104C200011F40C94304011E0029709F010E00E945A
:104C300079C482E50E946DC4882309F45CC10E9496
:104C40000BC46B017C014090F5145090F6146090F9
:104C5000F7147090F8148091F9149091FA14A091BF
:104C6000FB14B091FC142B968CAF9DAFAEAFBFAFD1
:104C70002B9720919F043091A0044091A104509162
:104C8000A2042F962CAF3DAF4EAF5FAF2F97809110
:104C9000A3049091A404A091A504B091A6046396E6
:104CA0008CAF9DAFAEAFBFAF639720E030E0A901FE
:104CB000C701B6010E9464F2882309F40AC5A30162
:104CC00092012F966CAD7DAD8EAD9FAD2F970E945A
:104CD00064F2811111C02B962CAD3DAD4EAD5FAD90
:104CE0002B9763966CAD7DAD8EAD9FAD63970E94A3
:104CF00064F2882309F4EDC420E030E0A901C70183
:104D0000B6010E9464F2881F8827881F18130BC001
:104D100020E030E040E85FE3A3962CAF3DAF4EAF1C
:104D20005FAFA3970AC080E090E0A0E8BFEBA39636
:104D30008CAF9DAFAEAFBFAFA397A30192012F96EB
:104D40006CAD7DAD8EAD9FAD2F970E949CF66B969E
:104D50006CAF7DAF8EAF9FAF6B972B962CAD3DADFB
:104D60004EAD5FAD2B9763966CAD7DAD8EAD9FADB7
:104D700063970E949CF66F966CAF7DAF8EAF9FAF2E
:104D80006F976B962CAD3DAD4EAD5FAD6B97CA0185
:104D9000B9010E94C9F24B015C016F962CAD3DAD8B
:104DA0004EAD5FAD6F97CA01B9010E94C9F29B0178
:104DB000AC01C501B4010E949DF60E9408F96796F6
:104DC0006CAF7DAF8EAF9FAF679720E030E040E0E3
:104DD0005FE30E94C9F24B015C01A7019601C70184
:104DE000B6010E94C9F26B017C01A5019401C501C5
:104DF000B4010E94C9F29B01AC01C701B6010E9437
:104E00009CF60E9408F99B01AC01A3966CAD7DADA8
:104E10008EAD9FADA3970E94C9F24B015C012F9606
:104E20002CAD3DAD4EAD5FAD2F97C301B2010E94D9
:104E30009DF620E030E040E05FE30E94C9F26B01A4
:104E40007C016F966CAD7DAD8EAD9FAD6F97905828
:104E500067962CAD3DAD4EAD5FAD67970E9479F77B
:104E60009B01AC01C501B4010E94C9F29B01AC01D8
:104E7000C701B6010E949DF6A30192010E949CF613
:104E80006B017C0163962CAD3DAD4EAD5FAD63977C
:104E90002B966CAD7DAD8EAD9FAD2B970E949DF690
:104EA00020E030E040E05FE30E94C9F22B013C01CA
:104EB00067962CAD3DAD4EAD5FAD67976B966CAD13
:104EC0007DAD8EAD9FAD6B970E9479F79B01AC01D4
:104ED000C501B4010E94C9F29B01AC01C301B2013A
:104EE0000E949DF62B962CAD3DAD4EAD5FAD2B9740
:104EF0000E949CF614C089E40E946DC4882329F0A6
:104F00000E940BC46B017C0103C0C12CD12C760123
:104F10008AE40E946DC48823F9F00E940BC4639652
:104F20006CAF7DAF8EAF9FAF639720E030E0A901FB
:104F3000C701B6010E9464F281111EC020E030E07A
:104F4000A90163966CAD7DAD8EAD9FAD63970E9458
:104F500064F2811111C0BDC320E030E0A901C70196
:104F6000B6010E9464F2882309F4B3C363961CAEB1
:104F70001DAE1EAE1FAE6397A701960150582B962B
:104F80002CAF3DAF4EAF5FAF2B9763968CAD9DAD11
:104F9000AEADBFAD6397B0582F968CAF9DAFAEAF9F
:104FA000BFAF2F97CA01B9010E94C9F24B015C0142
:104FB0002F962CAD3DAD4EAD5FAD2F97CA01B90117
:104FC0000E94C9F29B01AC01C501B4010E949DF68B
:104FD0000E9408F9E3966CAF7DAF8EAF9FAFE39769
:104FE0002091F5143091F6144091F7145091F81473
:104FF00067962CAF3DAF4EAF5FAF6797A7019601A5
:1050000067966CAD7DAD8EAD9FAD67970E949DF6A6
:10501000A3966CAF7DAF8EAF9FAFA3978091F9142D
:105020009091FA14A091FB14B091FC146F968CAF80
:105030009DAFAEAFBFAF6F9763962CAD3DAD4EAD9C
:105040005FAD6397BC01CD010E949DF6A7966CAF42
:105050007DAF8EAF9FAFA79720919F043091A004A2
:105060004091A1045091A204AB962CAF3DAF4EAF3E
:105070005FAFAB97A3962CAD3DAD4EAD5FADA397A3
:10508000AB966CAD7DAD8EAD9FADAB970E949CF69F
:105090006B017C018091A3049091A404A091A504CC
:1050A000B091A604AF968CAF9DAFAEAFBFAFAF9738
:1050B000A7962CAD3DAD4EAD5FADA797BC01CD0120
:1050C0000E949CF64B015C012091FD143091FE146E
:1050D0004091FF1450910015EB962CAF3DAF4EAFB1
:1050E0005FAFEB976091A7047091A8048091A90429
:1050F0009091AA040E949CF66B966CAF7DAF8EAF28
:105100009FAF6B978091AB049091AC04A091AD04DC
:10511000B091AE04E7968CAF9DAFAEAFBFAFE7974F
:1051200020910115309102154091031550910415FD
:10513000EF962CAF3DAF4EAF5FAFEF97A701960153
:105140002B966CAD7DAD8EAD9FAD2B970E94C9F2B5
:105150002B013C01A50194012F966CAD7DAD8EAD68
:105160009FAD2F970E94C9F29B01AC01C301B20110
:105170000E949DF62B013C01A50194012B966CAD7C
:105180007DAD8EAD9FAD2B970E94C9F24B015C01A6
:10519000A70196012F966CAD7DAD8EAD9FAD2F977B
:1051A0000E94C9F29B01AC01C501B4010E949CF6AA
:1051B000A30192010E9410F76B017C0120E030E016
:1051C000A9010E9464F287FF0AC02BED3FE049EC81
:1051D00050E4C701B6010E949DF66B017C011123CA
:1051E00051F02BED3FE049EC50E4C701B6010E94BD
:1051F0009CF66B017C0120E030E0A901C701B601FB
:105200000E9464F2811128C0AB962CAD3DAD4EAD2D
:105210005FADAB9767966CAD7DAD8EAD9FAD67977B
:105220000E9464F2811118C0AF962CAD3DAD4EAD19
:105230005FADAF976F966CAD7DAD8EAD9FAD6F9747
:105240000E9464F2811108C04BEDC42E4FE0D42EB1
:1052500049ECE42E40E4F42EE3962CAD3DAD4EAD8A
:105260005FADE397C701B6010E94C9F29B01AC0193
:105270000E94C9F24B015C016B962CAD3DAD4EAD69
:105280005FAD6B97CA01B9010E94C9F29B01AC01E5
:10529000C501B4010E949DF60E9408F94B015C0112
:1052A0002FE632E143E85AE30E9464F287FD0DC223
:1052B000C501B4010E9412F80E94E6F71B01672B9A
:1052C00019F422242394312CB10180E090E00E9453
:1052D00068F24B015C019B01AC01C701B6010E9461
:1052E00079F767966CAF7DAF8EAF9FAF6797A501DB
:1052F00094016B966CAD7DAD8EAD9FAD6B970E94AA
:1053000079F7E3966CAF7DAF8EAF9FAFE397EF96E3
:105310002CAD3DAD4EAD5FADEF97E7966CAD7DAD7D
:105320008EAD9FADE7970E949CF6A50194010E9467
:1053300079F7E7966CAF7DAF8EAF9FAFE797679633
:105340002CAD3DAD4EAD5FAD6797CA01B9010E946E
:10535000C9F220E030E040E05FE30E94C9F29B0127
:10536000AC0160E070E080E89FE30E949CF6AB96A1
:105370006CAF7DAF8EAF9FAFAB97EB968CAD9DAD15
:10538000AEADBFADEB9789879A87AB87BC87EF96A9
:105390002CAD3DAD4EAD5FADEF972D873E874F876E
:1053A000588B6091160270911702072E000C880B23
:1053B000990B0E946AF220911802309119024091D3
:1053C0001A0250911B020E94C9F22AE037ED43E213
:1053D0005CE30E94C9F268A379A38AA39BA30E94FD
:1053E000CE9F9B01AC0128533F4F4F4F5F4FAF966D
:1053F0002CAF3DAF4EAF5FAFAF9728964FAC28971D
:1054000029965FAC29972A966FAC2A972B967FAC8A
:105410002B9741E050E06D965FAF4EAF6D9759E12D
:1054200068965FAF68976D96AEADBFAD6D97A215EC
:10543000B30509F439C10E9472E70E94CE9FDC01D6
:10544000CB01AF962CAD3DAD4EAD5FADAF97821B9E
:10545000930BA40BB50BB7FD11C00E94CE9F9B010F
:10546000AC0128533F4F4F4F5F4FAF962CAF3DAF2E
:105470004EAF5FAFAF9780E00E94676768963FAD21
:105480006897315068963FAF6897332309F44BC053
:10549000AB962CAD3DAD4EAD5FADAB972F966CADE1
:1054A0007DAD8EAD9FAD2F970E94C9F26B017C013F
:1054B00067962CAD3DAD4EAD5FAD6797B201C301B0
:1054C0000E94C9F2A70196010E949DF67B018C0102
:1054D000AB962CAD3DAD4EAD5FADAB97B201C30108
:1054E0000E94C9F24B015C0167962CAD3DAD4EADFB
:1054F0005FAD67972F966CAD7DAD8EAD9FAD2F974D
:105500000E94C9F29B01AC01C501B4010E949CF646
:105510002B013C01C701D8012F968CAF9DAFAEAFD8
:10552000BFAF2F9761C06D964EAD5FAD6D97BA015D
:1055300080E090E00E9468F267962CAD3DAD4EADE4
:105540005FAD67970E94C9F24B015C010E9476F73C
:105550006B017C01C501B4010E94FEF84B015C01A6
:10556000A70196012B966CAD7DAD8EAD9FAD2B97AF
:105570000E94C9F22B013C01A501940163966CAD18
:105580007DAD8EAD9FAD63970E94C9F29B01AC01CA
:10559000C301B2010E949DF62B013C01A5019401BB
:1055A0002B966CAD7DAD8EAD9FAD2B970E94C9F251
:1055B0004B015C01A701960163966CAD7DAD8EAD8C
:1055C0009FAD63970E94C9F29B01AC01C501B40174
:1055D0000E949CF62F966CAF7DAF8EAF9FAF2F973A
:1055E00059E168965FAF68979201A301A3966CADED
:1055F0007DAD8EAD9FADA3970E949DF669837A83A2
:105600008B839C832F962CAD3DAD4EAD5FAD2F9718
:10561000A7966CAD7DAD8EAD9FADA7970E949DF610
:105620006D837E838F839887E3962CAD3DAD4EAD21
:105630005FADE39769857A858B859C850E949DF691
:1056400069877A878B879C87E7962CAD3DAD4EADF9
:105650005FADE7976D857E858F8598890E949DF661
:105660006D877E878F87988BCE0101960E944B694C
:10567000E0909D048E01005E1F4F9E01235F3F4F0F
:10568000AE01475F5F4FBE016B5F7F4FCE0101965A
:105690000E9436C06D968EAD9FAD6D9701966D964A
:1056A0009FAF8EAF6D97BFCEE0909D048E01005EE0
:1056B0001F4F2BEA34E047EA54E063EA74E08FE9D5
:1056C00094E00E9436C00E9464C50E947DA30C94A1
:1056D0003040E2EBFBE084918F010F5F1F4F882386
:1056E00021F00E948384F801F6CFEFEDF7E084917A
:1056F0008F010F5F1F4F882311F40C9430400E94DC
:105700008384F801F4CF80E50E946DC4882329F0DA
:105710000E94CBC36B017C0103C0C12CD12C76014C
:1057200083E50E946DC4882361F00E940BC420E0D1
:1057300030E04AE754E40E94C9F20E94E6F76B01A8
:105740007C010E94E44B80912B02811105C060E036
:1057500086ED97E00E941CC60E947DA3809199046B
:1057600090919A04A0919B04B0919C04C80ED91EFC
:10577000EA1EFB1E0E94CE9FDC01CB018C199D0905
:10578000AE09BF09B7FD02C00C94304080E00E9412
:105790006767F0CF81E08093200210924D0A0C944D
:1057A00030400E94E8EC81110C94304080E090E0A1
:1057B000A8ECB2E489839A83AB83BC8380E090E059
:1057C000A6E9B3E48D839E83AF83B88780E090E041
:1057D000A0EAB1E489879A87AB87BC8780E50E94FD
:1057E0006DC4882319F00E94DBC301C060E068A388
:1057F000BE016F5F7F4FCE0180960E94CCCA0C9491
:1058000030401092B3040C94304081E08093B30494
:105810000C9430408091B4049091B5048637910582
:1058200011F40C9438340CF0E4C08B34910509F475
:10583000E9C40CF05FC08831910509F494C26CF59D
:105840008231910509F4ECC684F497FF02C00C94F0
:105850003040823091050CF4B7C1419711F00C949F
:1058600030400E94005E0C9430408531910509F46F
:1058700070C23CF4449711F00C943040EEE8F7E02D
:1058800027C28631910509F468C2479711F00C943C
:1058900030400E94E35C0C9430408E31910509F455
:1058A000A1C2C4F48A31910509F48AC20CF47AC207
:1058B0008B31910509F492C24C9711F00C94304051
:1058C00040E060E080919704909198040E94CD524E
:1058D0000C9430408032910509F492C30CF498C3C3
:1058E0008A32910509F43AC48934910509F47DC4DA
:1058F0000C9430408836910509F490C40CF044C0F3
:105900008235910509F483C634F58D34910509F487
:1059100081C40CF47BC48135910511F00C943040A6
:105920000E949BE40E94E44B0E9442691092920400
:1059300010929104109294041092930468EE73E014
:1059400080E090E00E94D24960E081E596E00E940C
:105950001CC60C9430408435910509F461C60CF4E2
:105960005AC68535910509F48EC68C35910511F01E
:105970000C9430404CE3C42E43E0D42E55E0E52E89
:1059800055E1F52E10E09AC68E36910509F487C4CC
:105990009CF48A36910509F47BC50CF421C58B363D
:1059A000910509F4A1C58D36910511F00C94304094
:1059B0000E94A45A0C9430408237910509F4FEC627
:1059C00034F48F36910509F47DC40C94304083374C
:1059D000910509F4F9C68537910511F00C94304012
:1059E00060E080919704909198040E94BAC80C944A
:1059F00030408C32B1E09B0711F40C94D6360CF099
:105A000069C0883C910509F4E1C75CF58D379105C3
:105A100009F482C58CF48837910509F4CCC70CF4DD
:105A200066C78937910511F00C9430401092930DA0
:105A30001092920D0C9430408139910509F4C2C73F
:105A400034F48C38910509F4ADC40C9430408B3992
:105A5000910509F4DFC48E3B910509F402C50C944D
:105A600030408E3C910511F40C945F35C4F48B3CAE
:105A7000910509F4AFC74CF4893C910511F00C94E1
:105A800030400E94956D0C9430408C3C910509F497
:105A9000A5C78D3C910509F4A5C70C9430408C3DF9
:105AA000910511F40C9436364CF4833D910511F0B8
:105AB0000C943040E5EDF6E10C9463358D3D910595
:105AC00011F40C944536823E910511F40C948F36F6
:105AD0000C943040843FF1E09F0711F40C946B3E2E
:105AE000D4F58E3531E0930711F40C94A43FB4F44F
:105AF0008E3251E0950711F40C941D3814F40C9477
:105B000000378F32B1E09B0711F40C947138803369
:105B1000914011F40C949F370C9430408336F1E09F
:105B20009F0711F40C94A73F4CF48F35914011F06E
:105B30000C9430400E94AA6B0C943040803941E0B4
:105B4000940711F40C94823D8C3A914011F40C941A
:105B5000853D0C9430408835A2E09A0711F40C94EE
:105B60008B3EB4F4863FE1E09E0711F40C94713E45
:105B700014F40C946E3E873F21E0920711F40C94CC
:105B8000743E8C31924011F40C94803E0C94304061
:105B90008C3843E0940711F40C94A13F4CF48B38FB
:105BA000934011F00C9430400E94546C0C9430409F
:105BB000803AB3E09B0709F427C2873E934011F473
:105BC0000C94C03F0C943040A0909704B09098047F
:105BD00080E50E946DC4882359F00E94CBC36B01FD
:105BE0007C0111E0672B682B692B31F410E004C0B5
:105BF00010E0C12CD12C760183E50E946DC488236E
:105C0000F1F00E940BC420E030E04AE754E40E9427
:105C1000C9F20E94E6F76B017C01111112C0672BDB
:105C2000682B692B71F4A114B10459F0D5018C9142
:105C3000882339F061E0C5010E94BAC807C011236A
:105C400091F360E083EC97E00E941CC681E08093B2
:105C500096040E94E44B0E947DA3C114D104E10488
:105C6000F104F1F08091990490919A04A0919B0421
:105C7000B0919C04C80ED91EEA1EFB1E0E94CE9F46
:105C8000DC01CB018C199D09AE09BF09B7FF1CC00F
:105C9000809196048823C1F080E00E946767EECF70
:105CA00080919604882321F080E00E946767F8CFF6
:105CB0008091920A60E0823019F48EEA97E002C087
:105CC0008FE997E00E941CC6109296040C94304015
:105CD00084918F010F5F1F4F882321F00E948384DE
:105CE000F801F6CF10924D0D40E050E0BA0189EF77
:105CF0009AE00E94DC798BE1E9EFFAE0DE0115968B
:105D000001900D928A95E1F78091F70A9091F80A37
:105D10009C838B838BE893E09A83898340E050E0F7
:105D2000BE016F5F7F4F87EE93E00E94D796CE0152
:105D300001960E9454AFEFE7F7E084918F010F5F67
:105D40001F4F882311F40C9430400E948384F80183
:105D5000F4CF0E9412560C9430401092A10A109277
:105D6000A20A0C94304019821A821B821C8218A24B
:105D700019A21AA21BA280919504882341F040E049
:105D8000BE016F5F7F4FCE0180960E942BAE809147
:105D9000A20A882319F081E08093A10A0E947F94CF
:105DA0000C9430401092A10A0E9421948AE797E057
:105DB0009093F6088093F5080E94F3C20C9430404B
:105DC0008091A20A882311F40C94304083E50E944C
:105DD0006DC481110C94E4400C9430400E94A65C88
:105DE0000C9430408091A20A882311F40C94304026
:105DF00083E99CE00E94667C83E99CE00E941A7E15
:105E00001092A00A10929F0AE0909704F0909804D4
:105E10008091A20A882311F40C9430400E94C2524F
:105E20001D8218861C821B828BE893E09A838983EB
:105E300085EF9AE09093150B8093140BF701808106
:105E40008F3209F068C06FE270E0C7010E94CCF9A0
:105E50008C010F5F1F4F9E012F5F3F4F49010115BE
:105E6000110509F45EC06FE270E0C8010E94CCF930
:105E70006C01009709F456C00817190708F052C0C2
:105E80005C01A01AB10AA501B801CE0180960E945A
:105E9000ECF9E0E2F0E0EC0FFD1FEA0DFB1D1082D3
:105EA0008E01005E1F4FD8018D918D01882319F05E
:105EB0000E948384F8CF8AE00E9483846091140B4F
:105EC0007091150B6115710511F06C5F7F4F21E02A
:105ED000AE01405E5F4FCE0105960E940B8081119E
:105EE00012C0BE01605E7F4F86E697E00E941EA44E
:105EF0008EE20E9483848AE00E948384C4010E940F
:105F000054AF0C9430409092150B8092140B860184
:105F10000F5F1F4FA4CF86E19BE09093150B8093FA
:105F2000140B87016091140B7091150B61157105AD
:105F300011F06C5F7F4F18A21BA222E0A801CE01D6
:105F400080960E940B80811102C0F12C14C0CE01FA
:105F500080960E9445968823C1F361E0CE01809629
:105F60000E944A7C009789F325EEFC0120831BA246
:105F70000E94DDC8F82ECE0180960E944BC5FF20FE
:105F800009F1E0E4F7E084917F012FEFE21AF20AD1
:105F9000882321F00E948384F701F5CFD8018D91E9
:105FA0008D01882319F00E948384F8CF8AE00E9433
:105FB00083841092440D1092450D1092460D10925C
:105FC000470D18C0EEE4F7E084917F01BFEFEB1AB4
:105FD000FB0A882321F00E948384F701F5CFF801A2
:105FE00081918F01882319F00E948384F8CF8EE27B
:105FF0000E948384CE0101960E9454AF0C943040DD
:106000000E94655C0C9430400E945A5C0C943040B5
:106010000E944B942CE3C22ED12CE12CF12CA70131
:1060200096010E943FF6762E672ECA01B901A7019C
:1060300096010E943FF66B017C01CA01B90128E17B
:1060400030E040E050E00E943FF64B015C01C901A6
:106050006DE671E00E9461F98E010F5F1F4F6115BF
:10606000710599F06F927F92DF92CF929F928F92FB
:106070009F938F937F936F938FE197E09F938F937D
:106080001F930F930E94FDF112C00097B1F06F9221
:106090007F92DF92CF929F928F929F938F938FE008
:1060A00097E09F938F931F930F930E94FDF10FB67C
:1060B000F894DEBF0FBECDBF36C081149104A10499
:1060C000B10479F06F927F92DF92CF929F928F927C
:1060D00083E097E09F938F931F930F930E94FDF1AE
:1060E000E6CFC114D104E104F10469F06F927F920C
:1060F000DF92CF928BEF96E09F938F931F930F9336
:106100000E94FDF1D4CF6F927F9287EF96E09F932C
:106110008F931F930F930E94FDF10F900F900F909C
:106120000F900F900F9060E0C8010E94BAC8E5ED93
:10613000F6E184917F01BFEFEB1AFB0A882321F07F
:106140000E948384F701F5CFB80183E397E00E94B2
:106150001EA48AE00E9483840C94304083E50E9450
:106160006DC4882311F40C9430400E94EBC3E82ED8
:1061700080E50E946DC4882311F40C94304080E5C2
:106180000E946DC4882341F00E94DBC38B0177FF1E
:1061900002C00C94304002C00DE010E0902FE0EC03
:1061A000F6E088E28E0F2491921729F031968E1333
:1061B000FACF0C94F540E2EBFBE084918F010F5F86
:1061C0001F4F882321F00E948384F801F6CFE8EE68
:1061D000F6E084918F010F5F1F4F882311F40C9418
:1061E00030400E948384F801F4CF8091A10A81118C
:1061F0000C94304080E50E943EC481110C94124101
:106200000C9430400E947F940C9430400E94219462
:106210000C9430400E9436940C94304088E690E014
:106220000E940BC581110C94304080919E0483FF25
:1062300002C00C94304083E50E946DC4882311F4A1
:106240000C9430400E940BC40E94E1F770938B04C1
:1062500060938A0480E00E9450E40E940BC4209165
:106260008C0430918D0440918E0450918F040E94D3
:10627000C3F8181614F00C94304084EE92E09F930B
:106280008F9384EB96E09F938F931F920E94B89414
:106290000F900F900F900F900F900C9430408EE461
:1062A0000E946DC4882311F40C9430400E94DBC31B
:1062B0006093E6067093E7068093E8069093E906FC
:1062C0000C94304083E50E943EC4882359F083E556
:1062D0000E946DC4882319F00E94EBC301C080E0C6
:1062E00080939E04E5EDF6E184918F010F5F1F4FCF
:1062F000882321F00E948384F801F6CFEDEAF6E0CE
:1063000084918F010F5F1F4F882321F00E948384A7
:10631000F801F6CFC0909E04CC2099F10FE9A02E91
:1063200006E0B02EE12CF12C80E0D12C96010E2C51
:1063300002C0359527950A94E2F720FF17C09924EB
:106340009394980E882319F08CE20E948384F501BF
:1063500025913491F901849189010F5F1F4F8823A2
:1063600021F00E9483849801F5CF892DFFEFEF1A69
:10637000FF0A22E0A20EB11C35E0E316F104B1F6EB
:106380000CC0E9EAF6E084918F010F5F1F4F88236C
:1063900021F00E948384F801F6CF8AE00E94838472
:1063A0000C94304080919E0483FF02C00C943040D6
:1063B00083E50E946DC4882311F40C9430400E9440
:1063C0000BC40E94E1F76739710514F066E970E0CB
:1063D00070938904609388040E9405E40C94304013
:1063E00089E690E00E940BC581110C94A344ECE96E
:1063F000F6E084918F010F5F1F4F882321F00E94E8
:106400008384F801F6CF0E9482E38AE00E948384AD
:106410000C94A34483E50E946DC4882311F40C946A
:1064200030400E94EBC3182F8D3308F01CE310930B
:1064300087040E94CE9F6B017C01212F30E0A8EEE3
:10644000B3E00E948DF6C60ED71EE81EF91EC0925C
:106450008304D0928404E0928504F09286040C9424
:10646000304080919E0483FF02C00C94304083E54D
:106470000E946DC460968FAF609781110C941D418E
:1064800082E50E946DC481110C941D410C94304032
:1064900080E50E946DC4882341F00E94EBC3182F51
:1064A000823010F00C94304001C010E083E50E946F
:1064B0006DC4882329F00E94DBC3362F272F02C02A
:1064C0003FEF20E0E12FF0E0EE0FFF1FEF56FB4F14
:1064D000832F922F8F3F910519F010F08FEF90E0EE
:1064E000918380830C94304080E50E946DC48823A2
:1064F00041F00E94DBC36230710510F00C94304013
:1065000002C060E070E0660F771FFB01EF56FB4FA3
:10651000118210820C9430408CE40E943EC4882387
:1065200019F00E940BC404C060E070E080E090ECC1
:106530006BAF7CAF8DAF9EAF80E090E0A8ECB2E493
:1065400089839A83AB83BC8380E090E0A6E9B3E4BF
:106550008D839E83AF83B88780E090E0A0EAB1E4AA
:1065600089879A87AB87BC8788E50E946DC488239A
:1065700079F088E50E946DC4882319F00E940BC44D
:1065800003C060E070E0CB0169837A838B839C83D6
:1065900089E50E946DC4882379F089E50E946DC465
:1065A000882319F00E940BC403C060E070E0CB01A7
:1065B0006D837E838F8398878AE50E946DC48823CC
:1065C00079F08AE50E946DC4882319F00E940BC4FB
:1065D00003C060E070E0CB0169877A878B879C8776
:1065E00018A219A21AA21BA28091950481110C94E1
:1065F000304000E020E0AE01405E5F4FBE016F5FC3
:106600007F4FCE01CB960E9436AD0C943040109255
:10661000B2040C94304081E08093B2040C9430407A
:1066200083E50E946DC48823A1F00E940BC420E082
:1066300030E04AE754E40E94C9F20E94E6F7609312
:1066400011027093120280931302909314020C941F
:10665000304088E50E943EC481110C94994289E53E
:106660000E943EC481110C9499428AE50E943EC466
:1066700081110C94994285E40E943EC481110C94CE
:1066800099420C94BC4283E50E943EC4882311F4D5
:106690000C9430400E940BC420E030E04AE754E400
:1066A0000E94C9F20E94E6F760937A0470937B041B
:1066B00080937C0490937D040C943040D6018D919E
:1066C0006D010E943EC4882309F46DC0133009F0A7
:1066D00063C00E940BC44B015C0120E030E040EA43
:1066E00051E40E9464F287FF4EC0A50194016091BD
:1066F00011157091121580911315909114150E9427
:1067000079F72B013C019B01AC01609176047091FB
:10671000770480917804909179040E94C9F2609383
:106720007604709377048093780490937904A3019E
:106730009201609166047091670480916804909161
:1067400069040E94C9F260936604709367048093A1
:106750006804909369046091560470915704809185
:106760005804909159040E9468F2A30192010E947A
:10677000C9F20E94E6F76093560470935704809321
:106780005804909359048092111590921215A0927A
:106790001315B092141507C00E940BC4F701608353
:1067A0007183828393831F5FF4E0EF0EF11C14303A
:1067B00009F084CF0E940CC00C9430400E94E44B3E
:1067C0000E9450590C943040ECE5F5E084918F0123
:1067D0000F5F1F4F882321F00E948384F801F6CFBA
:1067E00060E08CE495E00E940C5961E085E495E05E
:1067F0000E940C5961E08AE395E00E940C5961E027
:106800008AE295E00E940C5960E081E295E00E94E6
:106810000C5961E087E195E00E940C5960E08DE041
:1068200095E00E940C5960E085E095E00E940C59CB
:1068300060E087EF94E00E940C5961E089EE94E0FB
:106840000E940C5960E08AED94E00E940C5960E0CF
:106850008CEC94E00E940C5960E086EB94E00E947E
:106860000C5961E085EA94E00E940C590C94304088
:1068700085E40E946DC4882319F00E94FCC303C004
:1068800085E40E943EC4882361F0E5EDF6E1849141
:106890008F010F5F1F4F882321F00E948384F8012E
:1068A000F6CF81E40E946DC4882319F00E94FCC3D6
:1068B00003C081E40E943EC4882361F0E1EAF4E071
:1068C00084918F010F5F1F4F882321F00E948384E2
:1068D000F801F6CF0091970410919804D8018D919A
:1068E0008D01882309F459CD0E948384F7CFE7E80E
:1068F000F4E084918F010F5F1F4F882321F00E94E5
:106900008384F801F6CFEFE7F4E084918F010F5F05
:106910001F4F882321F00E948384F801F6CF1E9B2D
:1069200003C00DEC12E002C002ED12E0F80181910B
:106930008F01882319F00E948384F8CF8AE00E9497
:106940008384E7E7F4E084918F010F5F1F4F882372
:1069500021F00E948384F801F6CF1D9B03C00DEC4B
:1069600012E002C002ED12E0D8018D918D01882362
:1069700019F00E948384F8CF8AE00E948384EFE6B6
:10698000F4E084918F010F5F1F4F882321F00E9454
:106990008384F801F6CF1C9B03C00DEC12E002C00B
:1069A00002ED12E0F80181918F01882309F4F5CC02
:1069B0000E948384F7CF81E08093930D8093920DA2
:1069C0000C9430400E942D5A0C9430400E94BA6DB5
:1069D0000C9430400E94736D0C9430400E940A6DFC
:1069E0000C94304083E50E943EC4882351F00E94FD
:1069F0000BC46093460470934704809348049093BB
:106A0000490484E50E943EC4882351F00E940BC4CF
:106A1000609342047093430480934404909345042C
:106A200082E40E943EC4882351F00E94CBC360934D
:106A30003E0470933F04809340049093410488E5A2
:106A40000E943EC4882351F00E940BC460936A04E4
:106A500070936B0480936C0490936D0489E50E949D
:106A60003EC4882351F00E940BC460936E0470935F
:106A70006F0480937004909371048AE50E943EC471
:106A8000882351F00E940BC46093720470937304C6
:106A9000809374049093750485E40E943EC4882317
:106AA00011F40C9430400E940BC4609376047093F0
:106AB000770480937804909379040C9430400E947A
:106AC000E16C0C94304084918F010F5F1F4F88233D
:106AD00021F00E948384F801F6CF83E50E943EC432
:106AE000882321F00E94FCC380931002EFE5F4E0BC
:106AF00084918F010F5F1F4F882321F00E948384B0
:106B0000F801F6CF80911002811103C0EBE5F4E0AB
:106B100002C0E7E5F4E084918F010F5F1F4F8823E7
:106B200021F00E948384F801F6CFEFE4F4E0849131
:106B30008F010F5F1F4F882321F00E948384F8018B
:106B4000F6CF40902604509027046090280470905F
:106B5000290420913204309133044091340450913F
:106B60003504C301B2010E949DF6AB01BC018DE466
:106B700094E00E94C1A380902A0490902B04A090DE
:106B80002C04B0902D0420913604309137044091AC
:106B9000380450913904C501B4010E949DF6AB013F
:106BA000BC018AE494E00E94C1A3C0902E04D0905E
:106BB0002F04E0903004F090310420913A04309199
:106BC0003B0440913C0450913D04C701B6010E9432
:106BD0009DF6AB01BC0187E494E00E94C1A3EFE302
:106BE000F4E084918F010F5F1F4F882321F00E94F2
:106BF0008384F801F6CF2091040230910502409180
:106C0000060250910702C301B2010E949DF6AB013A
:106C1000BC018DE394E00E94C1A320910802309151
:106C2000090240910A0250910B02C501B4010E9471
:106C30009DF6AB01BC018AE394E00E94C1A32091C0
:106C40000C0230910D0240910E0250910F02C701CB
:106C5000B6010E949DF6AB01BC0187E394E00E945F
:106C6000C1A38AE00E9483840C94304083E50E9493
:106C70006DC4882311F40C9430400E94DBC37093E0
:106C80001702609316020C9430408DED90E00E9444
:106C90000BC581110C94304083E50E946DC488239C
:106CA00011F40C9430400091820410E00E94DBC388
:106CB000000F111FF801EE5FFD4F7183608380911B
:106CC000820490E08C01000F111F000F111F98012A
:106CD000245E3D4F7901880F991FFC01EE5FFD4F47
:106CE00060817181072E000C880B990B0E946AF25B
:106CF0002AE037ED43E25CE30E94C9F2F801EE5D61
:106D0000FB4F20813181428153810E94C9F2D7011A
:106D10006D937D938D939C9313970C94304080E5F5
:106D20000E943EC4882311F40C9430400E94DBC3BF
:106D30006B017C0183E50E946DC4882321F00E94D1
:106D4000DBC38B0102C00FEF1FEF98012F5F3F4F96
:106D50002330310510F00C943040D7FE02C00C9463
:106D600030400E94E44B0F3FBFEF1B0731F0013072
:106D7000110571F401E010E00DC08C2D0E94789E89
:106D800031E020E0892B09F030E0032F122F02C000
:106D900000E010E08C2D0E94789E8017910711F47E
:106DA0000C94304080E00E946767F4CF83E50E9436
:106DB0006DC4882319F00E94DBC302C064E071E057
:106DC00079A368A380E50E946DC4882339F00E94EE
:106DD000DBC36938E3E17E0730F402C068EE73E09C
:106DE0007A83698304C088E893E19A838983BE012A
:106DF000605E7F4FCE0101960E9498570C94304000
:106E000085E40E946DC4811110C080E50E943EC4DB
:106E1000882391F00E940BC460931E0470931F049A
:106E2000809320049093210407C00E94EBC3882321
:106E300061F3E2EBFBE072C089E40E943EC4882368
:106E400081F00E940BC42CEA35EC47E25EE30E941D
:106E5000C9F260931A0470931B0480931C049093EE
:106E60001D0484E40E943EC4882381F00E940BC468
:106E70002CEA35EC47E25EE30E9479F76093160452
:106E8000709317048093180490931904E5EDF6E1CC
:106E900084918F010F5F1F4F882321F00E9483840C
:106EA000F801F6CF40911E0450911F046091200418
:106EB0007091210483E394E00E94C1A32CEA35EC95
:106EC00047E25EE360911A0470911B0480911C04F8
:106ED00090911D040E9479F7AB01BC018FE294E010
:106EE0000E94A4A32CEA35EC47E25EE3609116040D
:106EF0007091170480911804909119040E94C9F2AE
:106F0000AB01BC018BE294E00E94A4A38AE00E9442
:106F100083840C9430400E948384F80184918F0113
:106F20000F5F1F4F8111F7CF0FEE12E0D8018D9147
:106F30008D01882309F431CA0E948384F7CF80E54C
:106F40000E943EC4882351F00E940BC46093120437
:106F500070931304809314049093150489E40E94A1
:106F60003EC4882381F00E940BC42CEA35EC47E232
:106F70005EE30E94C9F260930E0470930F04809345
:106F800010049093110484E40E943EC4882381F08D
:106F90000E940BC42CEA35EC47E25EE30E9479F7CD
:106FA00060930A0470930B0480930C0490930D0477
:106FB000E5EDF6E184918F010F5F1F4F882321F0EB
:106FC0000E948384F801F6CF40911204509113047B
:106FD000609114047091150487E294E00E94C1A3AB
:106FE0002CEA35EC47E25EE360910E0470910F04E9
:106FF00080911004909111040E9479F7AB01BC01BB
:1070000083E294E00E94A4A32CEA35EC47E25EE31D
:1070100060910A0470910B0480910C0490910D040E
:107020000E94C9F2AB01BC018FE194E00E94A4A3CD
:107030008AE00E9483840C94304083E50E943EC421
:10704000182F882371F00E940BC40E94E1F77093FF
:1070500001026093000221E0672B09F020E02093F9
:10706000090480E50E943EC4882359F02091000263
:1070700030910102232B11F00E94FCC3809309047C
:10708000EFC71111EDC7E5EDF6E184918F010F5FB8
:107090001F4F882321F00E948384F801F6CF80914E
:1070A0000904811103C06CED72E002C06FEC72E064
:1070B0008CE094E00E941EA4609100027091010295
:1070C0008BEF93E00E9405A4E7EFF3E084918F013A
:1070D0000F5F1F4F882309F4C3C70E948384F80100
:1070E000F5CF85E40E946DC4882321F00E94DBC3A4
:1070F0007B0102C0E12CF12C83E40E946DC4882343
:1071000041F00E94DBC3C757DF4F6883C958D040A6
:1071100006C045E0C757DF4F4883C958D04085E5D2
:107120000E946DC4882319F00E94FCC303C085E54A
:107130000E943EC4CB56DF4F8883C559D040F7FC30
:1071400007C0812C912C16E1A12E13E4B12E06C0AC
:10715000812C912CBCE8AB2EB2E4BB2E83E50E94BF
:107160006DC4882321F00E940BC44B015C01E11423
:10717000F10411F4109282042896EFAE28970E9431
:10718000CE9FA7966CAF7DAF8EAF9FAFA797289687
:107190005FAD289757FF0FC080E090E0A0E0B1E41A
:1071A000CA55DF4F88839983AA83BB83C65AD040D0
:1071B0001CE342E00EC080E090E0A8EAB1E4CA55CA
:1071C000DF4F88839983AA83BB83C65AD04018E2D5
:1071D0004AE0CB57DF4F4883C558D04061E06E0D81
:1071E000623028F4A0E0EA2EA3E0FA2E0BC003E1FF
:1071F00013E0D8018D918D01882309F4CEC80E9437
:107200008384F7CFF70181917F01882319F00E94D1
:107210008384F8CF8AE00E9483840E949BE42896AE
:10722000FFAD2897F7FF09C087E680930804F7E6CB
:107230004F2E512C612C712C0FC028962FAD289702
:10724000E22F220FFF0BE95FFB4F8FE78083EFE711
:107250004E2E512C612C712CC501B4010E94E1F716
:10726000072E000C880B990B0E946AF264966FAF90
:10727000649768967FAF68976C968FAF6C97A0966F
:107280009FAFA097212F30E0A8EEB3E00E948DF6CB
:10729000CA56DF4F688379838A839B83C659D0405F
:1072A000DC01CB01A7962CAD3DAD4EAD5FADA797F0
:1072B000820F931FA41FB51FCE55DF4F888399837C
:1072C000AA83BB83C25AD04081E0809315022896DE
:1072D0003FAD289737FF05C08EEC90E0A0E0B0E00E
:1072E00004C08FEF90E0A0E0B0E09C01AD0123511D
:1072F000310941095109C455DF4F288339834A8335
:107300005B83CC5AD0409C01AD0124513109410925
:107310005109C055DF4F288339834A835B83C05BA3
:10732000D0409C01AD015595479537952795CC5494
:10733000DF4F288339834A835B83C45BD0409C0141
:10734000AD012150310941095109C854DF4F28834B
:1073500039834A835B83C85BD04063964CAE5DAE95
:107360006EAE7FAE6397A7968CAD9DADAEADBFAD53
:10737000A797C357DF4F88839983AA83BB83CD58D0
:10738000D040C656DF4F88839983AA83BB83CA59EE
:10739000D040C457DF4F1882CC58D040C256DF4F80
:1073A000188219821A821B82CE59D040E8961FAEED
:1073B000E89790E4EC969FAFEC97ACE1E096AFAF26
:1073C000E097B6E4E496BFAFE497C158DF4F188268
:1073D000CF57D040C058DF4F1882C058D040CF5749
:1073E000DF4F1882C158D040CE57DF4F1882C258A5
:1073F000D040812C912C5401AF968CAE9DAEAEAE98
:10740000BFAEAF9775016401CF56DF4F1882198266
:107410001A821B82C159D040E1E0C557DF4FE88393
:10742000CB58D040A9961FAE1EAEA99710E000E041
:10743000212C312C2896FFAD28978F2FFF0F990B09
:107440009C01295F3B4FC655DF4F39832883CA5AB9
:10745000D040880F991F880F991FAC0144575B4F8C
:10746000CD57DF4F59834883C358D040CB57DF4FA8
:107470008881C558D040082E000C990BAA0BBB0B75
:10748000CB57DF4F88839983AA83BB83C558D040ED
:10749000C757DF4FA881C958D0400A2E000CBB0B3C
:1074A000C757DF4FB983A883C958D04080911502D0
:1074B000882309F455C10E94CE9F2F966CAF7DAFF3
:1074C0008EAF9FAF2F9780910604882309F425C1C2
:1074D0000E945FE52896BFAD2897B7FF09C01091BD
:1074E0007E0400917F0420908004309081040AC0C3
:1074F000CD57DF4FE881F981C358D0401081018119
:1075000022803380212F302FA101C158DF4F6881A5
:10751000CF57D040C058DF4F7881C058D040CF57A8
:10752000DF4F8881C158D040CE57DF4F9881C25875
:10753000D0400E9464F287FF14C0C158DF4F188307
:10754000CF57D040C058DF4F0883C058D040CF57E6
:10755000DF4F2882C158D040CE57DF4F3882C25803
:10756000D040212F302FA101E8966FADE897EC961F
:107570007FADEC97E0968FADE097E4969FADE497F2
:107580000E94C3F8181664F4E8961FAFE897EC96CB
:107590000FAFEC97E0962FAEE097E4963FAEE497FE
:1075A000C557DF4FF881CB58D04064962FAD649714
:1075B00068963FAD68976C964FAD6C97A0965FAD9F
:1075C000A097612F702FC101FF2309F488C00E948A
:1075D000C3F818160CF0A1C02F962CAD3DAD4EADE2
:1075E0005FAD2F97A7968CAD9DADAEADBFADA79704
:1075F000281B390B4A0B5B0BC254DF4F288339839E
:107600004A835B83CE5BD040DA01C901885893413D
:10761000A109B109B7FD81C0D301C20163962CADA8
:107620003DAD4EAD5FAD6397821B930BA40BB50BC5
:1076300028963FAD2897B595A7959795879537FFDD
:1076400003C08093080407C0C655DF4FE881F98165
:10765000CA5AD0408083C254DF4F288139814A8181
:107660005B81CE5BD040CF56DF4F288339834A837E
:107670005B83C159D04064963FAD6497C158DF4FDA
:107680003883CF57D04068964FAD6897C058DF4FCA
:107690004883C058D0406C965FAD6C97CF57DF4F92
:1076A0005883C158D040A0968FADA097CE57DF4FDA
:1076B0008883C258D0402F962CAD3DAD4EAD5FAD06
:1076C0002F97C357DF4F288339834A835B83CD5875
:1076D000D040C557DF4F1882CB58D0401EC00E9403
:1076E00064F287FF1AC02F968CAD9DADAEADBFADD5
:1076F0002F97C357DF4F288139814A815B81CD584D
:10770000D040821B930BA40BB50BAC01BD014858B4
:1077100053416109710977FF34C720E030E040EA46
:1077200051E464966FAD649768967FAD68976C96E8
:107730008FAD6C97A0969FADA0970E949DF69B0180
:10774000AC01612F702FC1010E94C3F818167CF4A0
:10775000E3E8F3E084918F010F5F1F4F811103C0B5
:107760000E949BE47DC40E948384F801F3CF2F968E
:107770008CAD9DADAEADBFAD2F97C656DF4F288106
:1077800039814A815B81CA59D040821B930BA40B7B
:10779000B50BB7FDC9C00E9482E38AE00E948384D2
:1077A0002F968CAD9DADAEADBFAD2F978053984F4A
:1077B000AF4FBF4FC656DF4F88839983AA83BB83E1
:1077C000CA59D040C457DF4F9881CC58D04091114E
:1077D00087C0C256DF4F288139814A815B81CE59EB
:1077E000D040612F702FC1010E94C3F818160CF011
:1077F0005EC0CA55DF4F288139814A815B81C65AF4
:10780000D04064966FAD649768967FAD68976C962C
:107810008FAD6C97A0969FADA0970E949CF69B01A0
:10782000AC01A1E0C457DF4FA883CC58D040612FF2
:10783000702FC1010E94C3F818162CF0C457DF4FF7
:107840001882CC58D040CB57DF4F688179818A812C
:107850009B81C558D0400E946AF29B01AC01612F08
:10786000702FC1010E949DF6C256DF4F6883798355
:107870008A839B83CE59D0402F962CAD3DAD4EAD23
:107880005FAD2F97CA56DF4F88819981AA81BB814E
:10789000C659D040280F391F4A1F5B1FCE55DF4FF6
:1078A000288339834A835B83C25AD0403DC02F96D8
:1078B0008CAD9DADAEADBFAD2F97CE55DF4F2881BE
:1078C00039814A815B81C25AD040821B930BA40B41
:1078D000B50BB7FD29C045E653E064E773E01FC070
:1078E00020E030E040EA51E464966FAD649768961A
:1078F0007FAD68976C968FAD6C97A0969FADA09763
:107900000E949CF69B01AC01612F702FC1010E9467
:1079100064F287FF09C045E453E065E573E028960B
:107920008FAD28970E9482E52F968CAD9DADAEADB0
:10793000BFAD2F97880F991FAA1FBB1FC357DF4FDB
:10794000288139814A815B81CD58D040821B930BBD
:10795000A40BB50BA7962CAD3DAD4EAD5FADA79773
:10796000821B930BA40BB50B81389F44A241B10538
:1079700068F0E7E2F3E084918F010F5F1F4F8823E7
:1079800009F4EECE0E948384F801F5CFA9964EAD9E
:107990005FADA997C757DF4F88819981C958D040FB
:1079A000841795070CF0ABC0EAECF2E084918F01EC
:1079B0000F5F1F4F882321F00E948384F801F6CFC8
:1079C00028969FAD289797FD03C007EE13E002C0ED
:1079D00000EE12E0B80188EB92E00E941EA4B7010D
:1079E000A60184EB92E00E94C1A38AE00E948384F6
:1079F000B80182EA92E00E941EA4AF964CAD5DAD44
:107A00006EAD7FADAF978EE992E00E94C1A38AE090
:107A10000E948384B8018CE892E00E941EA4B50104
:107A2000A40188E892E00E94C1A38AE00E948384B6
:107A3000CB56DF4FA881C559D040AA2309F410C303
:107A40002896BFAD2897B7FF2DC0C0921204D092E0
:107A50001304E0921404F09215042CEA35EC47E28A
:107A60005EE3AF966CAD7DAD8EAD9FADAF970E94DE
:107A7000C9F260930E0470930F04809310049093E6
:107A800011042CEA35EC47E25EE3C501B4010E9423
:107A900079F760930A0470930B0480930C0490931D
:107AA0000D04DEC2C0921E04D0921F04E092200496
:107AB000F09221042CEA35EC47E25EE3AF966CAD20
:107AC0007DAD8EAD9FADAF970E94C9F260931A0451
:107AD00070931B0480931C0490931D042CEA35ECD6
:107AE00047E25EE3C501B4010E9479F76093160492
:107AF000709317048093180490931904B1C20E94E4
:107B0000E073D4CC0E94E44BABC20E94E8EC81113C
:107B1000A7C22DE3822E22E0922EE5EFF4E1299612
:107B2000FFAFEEAF29979E012F5F3F4F590105E848
:107B300012E0190133E0300F2C963FAF2C97F4017F
:107B400065917591859194912996AEADBFAD2997B8
:107B5000CD90DD90ED90FD902996BFAFAEAF299707
:107B6000A70196010E949CF62B013C0120E030E029
:107B700040EA51EC0E94C3F887FD10C020E030E0DD
:107B800040EA51E4C301B2010E9464F2181634F0D5
:107B9000F10140825182628273820DC0F8018491AA
:107BA0001816B4F7F7FAF094F7F8F094F101C082E0
:107BB000D182E282F382D101CD90DD90ED90FD90F3
:107BC0001D0120E030E040EA51ECC701B6010E94FF
:107BD000C3F887FF03C0E2EBFBE00BC020E030E01E
:107BE00040EA51E4C701B6010E9464F2181674F528
:107BF000F2CF84918F010F5F1F4F882321F00E94E5
:107C00008384F801F6CFE7E6F2E084918F010F5FFD
:107C10001F4F882321F00E948384F801F6CF61E092
:107C200089E592E00E941CC60E94FE6588E290E011
:107C300099A388A388EC90E09CAF8BAFBE01605EF7
:107C40007F4FCE01CB960E9498570AC2B4E08B0EAC
:107C5000911C0F5F1F4F2C96EFAD2C97E0136FCF49
:107C60009AEFE92E93E0F92E10E0F50181919191C0
:107C7000A191B1915F01F70181939193A193B19388
:107C80007F01812F0E9497C21F5F133071F70E94FE
:107C9000505960E089E492E00E941CC683E992E0BA
:107CA0009CAF8BAF04E610E019A308A3BE01655C8E
:107CB0007F4FCE0180960E9498578AEB92E09CAF4E
:107CC0008BAF19A308A3BE01655C7F4FCE018096E0
:107CD0000E949857C5C10E9481D5C2C10E9473D02D
:107CE000BFC10E943DCFBCC183E50E943EC4882332
:107CF00021F00E94FCC391E089270E9464CBB0C1AF
:107D000083E50E943EC4882309F4AAC10E94FCC3F3
:107D10008093F903A5C180E090E0A8ECB2E48983E8
:107D20009A83AB83BC8380E090E0A6E9B3E48D83C3
:107D30009E83AF83B88780E090E0A0EAB1E48987B2
:107D40009A87AB87BC870E94E8EC882319F081E012
:107D50000E948B5E85E40E943EC4882319F00E9435
:107D60000BC404C060E070E080E090EC27966CAF3C
:107D70007DAF8EAF9FAF27978AE50E946DC48823A1
:107D800079F08AE50E946DC4882319F00E940BC423
:107D900003C060E070E0CB0169877A878B879C879E
:107DA00088E50E946DC4882379F088E50E946DC43F
:107DB000882319F00E940BC403C060E070E0CB017F
:107DC00069837A838B839C8389E50E946DC48823B1
:107DD00079F089E50E946DC4882319F00E940BC4D4
:107DE00003C060E070E0CB016D837E838F83988752
:107DF00085E50E943EC4882319F00E940BC404C08C
:107E000060E070E088EC92EC23966CAF7DAF8EAFB3
:107E10009FAF23978CE40E943EC4882319F00E94F0
:107E20000BC403C060E070E0CB016BAF7CAF8DAFE3
:107E30009EAF82E40E946DC4882321F00E94DBC3C0
:107E4000162F01C015E0F090920A809195048111DF
:107E500072C001E0212FAE01415C5F4FBE016F5F38
:107E60007F4FCE018D5B9F4F0E9436AD882309F472
:107E700062C081E08093960480919604882309F47F
:107E800046C060E0812F0E948B5D8091440A882368
:107E9000D1F10093480A8BE693E70E9414958091F4
:107EA0009604882321F081E00E946767F8CF109242
:107EB000F5031092F6031092F7031092F803109254
:107EC000440A0E9450E40E942E5D0093480A84E117
:107ED00093E70E9414950E94CE9FDC01CB0188534A
:107EE0009045AF4FBF4F8093F5039093F603A09357
:107EF000F703B093F8031092440A0093960461E0EC
:107F0000812F0E948B5D81E00E946767B5CF80E082
:107F100090E0A0EAB1E488A399A3AAA3BBA38091AF
:107F20009504882341F0412FBE01605E7F4FCE0152
:107F3000CB960E942BAEF1E0FF1292C00E947F947C
:107F40008FC00E94376C8CC00E94FF6B89C0E2EB2F
:107F5000FBE084918F010F5F1F4F882321F00E9467
:107F60008384F801F6CFEEE2F2E084918F010F5F97
:107F70001F4F882309F474C00E948384F801F5CF51
:107F800081E08093200210924D0A83E50E946DC427
:107F9000882319F00E94FCC303C083E50E943EC4FD
:107FA00081115EC00E940E6A5BC0F090B404FF2095
:107FB00029F1E5EDF6E184918F010F5F1F4F8823D2
:107FC00021F00E948384F801F6CF84E50E94838427
:107FD0006F2D70E080E090E04AE00E94BD9080E26A
:107FE0000E9483840FEE12E0D8018D918D018823C9
:107FF00011F40C94CD310E948384F6CF10929D042D
:10800000E5EDF6E184918F010F5F1F4F882321F08A
:108010000E948384F801F6CF60E070E08CE192E08A
:108020000E9405A48AE00E9483841AC0E5EDF6E16F
:1080300084918F010F5F1F4F882321F00E9483845A
:10804000F801F6CF6091F2037091F30389E092E0BA
:108050000E941EA482E20E9483848AE00E9483849C
:108060000E94A06970C40E9479C48FE994E00E94C4
:108070004B690E947DA380919E0483FD86C0C090C1
:10808000AB04D090AC04E090AD04F090AE0420912D
:108090000115309102154091031550910415C70147
:1080A000B6010E9464F2882309F46FC00E9416ADE5
:1080B000882301F1C0920115D0920215E0920315B8
:1080C000F0920415E5EDF6E184918F010F5F1F4FEB
:1080D000882321F00E948384F801F6CFE4E1F8E0E0
:1080E00084918F010F5F1F4F882321F00E948384AA
:1080F000F801F6CFC090AB04D090AC04E090AD0492
:10810000F090AE04209101153091021540910315B5
:1081100050910415C701B6010E949CF69F77E0912B
:108120009D0424E0E29FF0011124E45EFD4F2081D4
:108130003181428153810E94C9F220E030E048E45D
:1081400053E40E94C3F8181604F5C0920115D092AA
:108150000215E0920315F0920415E5EDF6E1849125
:108160008F010F5F1F4F882321F00E948384F80145
:10817000F6CFE5EFF7E084918F010F5F1F4F882363
:1081800021F00E948384F801F6CF6091160270916D
:108190001702072E000C880B990B0E946AF220919F
:1081A00018023091190240911A0250911B020E944C
:1081B000C9F22AE037ED43E25CE30E94C9F20E9473
:1081C00072C20E9464C54CCF0E94DBC3AB01BC01EC
:1081D0004093440D5093450D6093460D7093470DA9
:1081E00083E99CE00E94DC793BCF802F0E94C19202
:1081F0006E2D802F0E94A09EF12CB701802F0E942F
:10820000CF9E0630110529F4F0929404E092930475
:1082100027CF0830110509F023CFF0929204E092A5
:1082200091041ECF0E94EBC3853620F084E6809334
:10823000900416CF8093900413CF0E940BC40E9429
:10824000E1F76739710514F066E970E0709389040D
:10825000609388040E9405E4609188047091890409
:10826000072E000C880B990B0E946AF220917E0465
:1082700030917F0440918004509181040E9464F207
:1082800087FF04C060E08FE896E003C060E082E80A
:1082900096E00E941CC681E08093150280919D04A7
:1082A000809382042F961CAE1DAE1EAE1FAE2F977C
:1082B00067961CAE1DAE1EAE1FAE679728961FAE0A
:1082C000289768961FAE68974CE36C964FAF6C97F3
:1082D0005CE1A0965FAFA09786E4A4968FAFA497C9
:1082E000C12CD12CB0E8EB2E1FEBF12E812C912C60
:1082F00054016091880470918904072E000C880B4A
:10830000990B0E946AF2162F072F782E692E262FBE
:10831000372F482F592FB601C7010E9464F28823D6
:1083200031F120917E0430917F044091800450917E
:108330008104612F702F872D962D0E9464F2881F73
:108340008827881F28968FAF289760969FAD6097E3
:10835000992389F0882379F080911502882309F404
:108360007FCE60E084E796E00E941CC679CE1C2D8B
:108370000D2D7E2C6F2C0E94CE9F6B017C01DC01A9
:10838000CB0167962CAD3DAD4EAD5FAD6797821BBF
:10839000930BA40BB50BB7FD3DC0D701C6018851A7
:1083A0009C4FAF4FBF4F67968CAF9DAFAEAFBFAF87
:1083B00067970E9482E3EEE7F6E084912F019FEF3A
:1083C000491A590A882321F00E948384F201F5CFCB
:1083D00081149104A104B104B9F0D501C4018851FC
:1083E0009C4FAF4FBF4FBC01CD016C197D098E0969
:1083F0009F0928EE33E040E050E00E943FF6CA01BA
:10840000B9010E94259103C08FE30E9483848AE012
:108410000E94838480E00E9467670E947DA3209071
:108420007E0430907F04409080045090810491013C
:10843000A201612F702F872D962D0E949CF69F77A9
:1084400020E030E040EA50E481149104A104B1043A
:1084500029F40E9464F287FF07C004C00E94C3F899
:10846000181614F4460157012896AFAD2897AA2391
:1084700009F443C02F962CAD3DAD4EAD5FAD2F97A7
:10848000211531054105510541F0D701C601821B77
:10849000930BA40BB50BB7FD30C09101A2016896F8
:1084A0006FAD68976C967FAD6C97A0968FADA097D7
:1084B000A4969FADA4970E949CF620E030E040EC8B
:1084C0005FE30E9464F287FD47CFD701C601805A5F
:1084D0009541AF4FBF4F2F968CAF9DAFAEAFBFAFA3
:1084E0002F9768962FAE68976C963FAE6C97A096C4
:1084F0004FAEA097A4965FAEA497809115028823F3
:1085000009F42ACF81149104A104B10429F4C12EE5
:10851000D02EE72CF62CEDCE98EEC91A93E0D90AAE
:10852000E108F108C818D908EA08FB08F7FE14CFDB
:10853000EECF0E94E44B88E50E943EC4882319F0E8
:10854000179A1092151589E50E943EC4882319F0E8
:10855000169A109216158AE50E943EC4882319F0D7
:10856000159A1092171585E40E943EC4882309F4D9
:1085700077CD0E94656774CD0E94E44B0E944269EA
:108580006FCDA9964EAD5FADA997452B09F46FC18C
:10859000CF56DF4F288139814A815B81C159D04054
:1085A000280F391F4A1F5B1FA7962CAF3DAF4EAF58
:1085B0005FAFA797CF56DF4F288139814A815B8112
:1085C000C159D040281B390B4A0B5B0BCA01B901BA
:1085D00063962CAD3DAD4EAD5FAD63970E9430F616
:1085E000A7962CAD3DAD4EAD5FADA7970E9461F64D
:1085F000420E531E641E751E34E14316510461047D
:1086000071040CF487C1C455DF4F88819981AA8118
:10861000BB81CC5AD040481659066A067B060CF03E
:1086200089C1CC54DF4F288139814A815B81C45B89
:10863000D04024153505460557059CF4C854DF4F36
:1086400088819981AA81BB81C85BD0408419950932
:10865000A609B70963968CAF9DAFAEAFBFAF639766
:1086600006C063964CAE5DAE6EAE7FAE6397B3014F
:10867000A2018FEE93E00E94DEA363964CAD5DAD48
:108680006EAD7FAD63978AEE93E00E94DEA3E8961D
:108690004FADE897EC965FADEC97E0966FADE09745
:1086A000E4967FADE49783EE93E00E94C1A3C158A6
:1086B000DF4F4881CF57D040C058DF4F5881C05856
:1086C000D040CF57DF4F6881C158D040CE57DF4FE1
:1086D0007881C258D0408CED93E00E94C1A3A99646
:1086E000AEADBFADA99713970CF4C1C063966CAD46
:1086F0007DAD8EAD9FAD63970E946AF220E030E0C1
:1087000040E850E40E94C9F26B017C01E8962FAD6D
:10871000E897EC963FADEC97E0964FADE097E49686
:108720005FADE497C158DF4F6881CF57D040C05844
:10873000DF4F7881C058D040CF57DF4F8881C15874
:10874000D040CE57DF4F9881C258D0400E949CF64F
:108750002BED3FE049E450E40E94C9F220E030E014
:1087600040E05FE30E94C9F29B01AC01C701B60182
:108770000E9479F76B017C01A7966CAD7DAD8EAD43
:108780009FADA7970E946AF22FE632E143E85AE3D1
:108790000E94C9F24B015C01B701A60186ED93E08E
:1087A0000E94C1A3B501A40180ED93E00E94C1A382
:1087B0002AE939E949E15FE3C701B6010E94C9F23C
:1087C0006B017C019B01AC010E949DF6A501940107
:1087D0000E9479F7AF966CAF7DAF8EAF9FAFAF972A
:1087E000A5019401C701B6010E94C9F220E030E062
:1087F00040E05EE30E94C9F24B015C01E0ECF3E073
:1088000084919F012F5F3F4F8823C1F0C454DF4FF5
:108810002883CC5BD040C354DF4F3883CD5BD0403E
:108820000E948384C454DF4F2881CC5BD040C35462
:10883000DF4F3881CD5BD040F901E2CFB701A6010F
:108840008AEB93E00E94C1A3AF964CAD5DAD6EADD7
:108850007FADAF9784EB93E00E94C1A3B501A40163
:108860008EEA93E00E94C1A38AE00E94838463960B
:108870008CAD9DADAEADBFAD6397840D951DA61DAE
:10888000B71D2896EFAD2897B595A795979587952D
:10889000E7FF03C08093080407C0C655DF4FE88197
:1088A000F981CA5AD0408083A9962EAD3FADA997D1
:1088B0002F5F3F4FA9963FAF2EAFA99764963FAD6C
:1088C0006497E8963FAFE89768964FAD6897EC9647
:1088D0004FAFEC976C965FAD6C97E0965FAFE0970B
:1088E000A0968FADA097E4968FAFE4972F962CAD0E
:1088F0003DAD4EAD5FAD2F97A7962CAF3DAF4EAFC0
:108900005FAFA79731E0C557DF4F3883CB58D040D2
:108910000C948D3B84E1482E512C612C712C24E168
:1089200030E040E050E063962CAF3DAF4EAF5FAF1C
:1089300063979DCEC055DF4F488059806A807B8009
:10894000C05BD0407BCECF53DF4F0FB6F894DEBF75
:108950000FBECDBFDF91CF911F910F91FF90EF9090
:10896000DF90CF90BF90AF909F908F907F906F904F
:108970005F904F903F902F900895AF92BF92CF920B
:10898000DF92EF92FF920F931F93CF93DF931F928B
:10899000CDB7DEB77C016B018A0159018091821449
:1089A000811119C0F701808191810E941AF6898393
:1089B000F60181936F01BE016F5F7F4FC5010E9479
:1089C000D0ECF701408151814F5F5F4F518340836D
:1089D0000150110939F70F90DF91CF911F910F913D
:1089E000FF90EF90DF90CF90BF90AF9008958F925F
:1089F0009F92AF92BF92CF92DF92EF92FF920F932E
:108A00001F93CF93DF931F921F92CDB7DEB7E091F4
:108A10008214E1114AC059016C018B017B01E40E03
:108A2000F51E0E151F0509F440C0F60180809180E7
:108A3000F80161918F016983C4016A830E941AF66B
:108A40006A81681729F1C4010E9422F6C4010E94BC
:108A50001AF699818917E1F0E5EDF6E184918F012D
:108A60000F5F1F4F882321F00E948384F801F6CF07
:108A7000E3E5F8E084918F010F5F1F4F882321F019
:108A80000E948384F801F6CF81E0809382140DC0A8
:108A9000BE016F5F7F4FC5010E94D0ECF60180815F
:108AA0009181019691838083BCCF0F900F90DF91CD
:108AB000CF911F910F91FF90EF90DF90CF90BF90DB
:108AC000AF909F908F900895CF93DF93CDB7DEB78F
:108AD0002C970FB6F894DEBF0FBECDBF8091F51472
:108AE0009091F614A091F714B091F81489839A83A9
:108AF000AB83BC838091F9149091FA14A091FB147C
:108B0000B091FC148D839E83AF83B8878091FD1450
:108B10009091FE14A091FF14B091001589879A8757
:108B2000AB87BC870E94DFBE0E941E8480E00E944B
:108B300097C281E00E9497C282E00E9497C20E9481
:108B40000CC04CE050E065EF74E1CE0101960E944C
:108B500098F9892B51F02C960FB6F894DEBF0FBE12
:108B6000CDBFDF91CF910C9450592C960FB6F8944D
:108B7000DEBF0FBECDBFDF91CF91089561E0FC0154
:108B800080810C94A09E8EBD0DB407FEFDCF08958C
:108B90008FEF8EBD0DB407FEFDCF8EB508950F93F8
:108BA0001F93CF93DF938B010E94CE9FEB01F0DFE9
:108BB0008F3F49F00E94CE9F6C1B7D0B60177107A1
:108BC000B0F380E001C081E0DF91CF911F910F9160
:108BD0000895CF92DF92EF92FF921F93CF93DF938E
:108BE00000D01F92CDB7DEB76C01162FFC01928129
:108BF000892F806A86958CBD90FD03C081E09630F8
:108C000009F480E08DBD60E0F601808129833A831C
:108C10004B835C830E94A09E6CE271E0C601BFDFC3
:108C2000812F8064B0DF88E1E82EF12C5C814B81DC
:108C30003A812981DA01C9010E2C04C0B695A795A5
:108C4000979587950A94D2F729833A834B835C835F
:108C50009ADFF8E0EF1AF10829813A814B815C81B3
:108C600088EFE8168FEFF80629F7112321F0183066
:108C700021F08FEF03C085E901C087E884DF1C3055
:108C800009F486DF10E084DFF601838387FF04C0E8
:108C90001F3F11F01F5FF7CF0F900F900F900F90B5
:108CA000DF91CF911F91FF90EF90DF90CF900895CB
:108CB0000F931F93CF93DF93EC0189018C81833055
:108CC00039F089E0440F551F661F771F8A95D1F749
:108CD0009A01AB0168E1CE017CDF882311F086E0C8
:108CE0002FC08EEF8EBD80E090E00DB407FEFDCF6B
:108CF000F801E80FF91F20812EBD0DB407FEFDCF4E
:108D000021812EBD0296811522E0920771F70DB4E4
:108D100007FEFDCF8FEF37DF8FEF35DF39DF8B8336
:108D20008F71853029F083E18983CE0127DF09C067
:108D300068E572E0CE0133DF182F811106C087E1AC
:108D40008983CE011BDF10E00FC020E030E0A901D5
:108D50006DE0CE013EDF811103C01ADF882311F0E0
:108D600086E1EECFCE010ADF812FDF91CF911F91F7
:108D70000F910895EF92FF920F931F93CF93DF937C
:108D8000EC0179018C81833039F089E0440F551F63
:108D9000661F771F8A95D1F79A01AB0161E1CE0179
:108DA00018DF882329F084E08983CE01E7DE35C00F
:108DB0000E94CE9F8B01ECDE8B838F3F49F40E9493
:108DC000CE9F601B710B6D327140A8F381E103C02F
:108DD0008E3F39F08FE08983CE01D0DE8FEFD3DE76
:108DE0001CC08FEF8EBDF701D701A150BE4F0DB44F
:108DF00007FEFDCF9EB591938EBDEA17FB07B9F72D
:108E00000DB407FEFDCF8EB58C93C2DEC1DECE0160
:108E1000B5DE8FEFB8DE81E001C080E0DF91CF9159
:108E20001F910F91FF90EF9008958F929F92AF92B4
:108E3000BF92CF92DF92EF92FF92CF93FC01C0805E
:108E4000D180E280F38020E030E0A901C701B601C3
:108E50000E9464F287FF08C0C701B601905820E065
:108E600030E048EC52E406C020E030E048EC52E448
:108E7000C701B6010E94C9F20E94E1F76B017C01B3
:108E8000603AF6E87F07F1E08F07910584F020EA69
:108E900036E841E050E00E9461F6CA01B9012AE0DB
:108EA00030E040E050E00E9461F6605D01C060E2A9
:108EB0006093BF0480E1C81687E2D806E104F1049C
:108EC00094F0C701B60120E137E240E050E00E9493
:108ED00061F6CA01B9012AE030E040E050E00E94AA
:108EE00061F6605D01C060E26093C004E8EECE16FA
:108EF000E3E0DE06E104F10494F0C701B60128EED8
:108F000033E040E050E00E9461F6CA01B9012AE076
:108F100030E040E050E00E9461F6605D01C060E238
:108F20006093C104C701B60124E630E040E050E0A0
:108F30000E9461F68AE0882E912CA12CB12CCA01E6
:108F4000B901A50194010E9461F6605D6093C204BD
:108F50008EE28093C304C701B601A50194010E946B
:108F600061F6C62FCA01B901A50194010E9461F6FC
:108F7000605D6093C404C05DC093C5048FEB94E052
:108F8000CF91FF90EF90DF90CF90BF90AF909F90E8
:108F90008F9008958F929F92AF92BF92CF92DF925F
:108FA000EF92FF92CF9320E030E048EC52E4FC01D6
:108FB00060817181828193810E94C9F20E94E1F7F0
:108FC0006B017C0197FF0AC0F094E094D094C094A8
:108FD000C11CD11CE11CF11C8DE201C08BE280930D
:108FE000BF04C701B60120E137E240E050E00E9433
:108FF00061F68AE0882E912CA12CB12CCA01B9010E
:10900000A50194010E9461F6605D6093C004C701F0
:10901000B60128EE33E040E050E00E9461F6CA015C
:10902000B901A50194010E9461F6605D6093C104DD
:10903000C701B60124E630E040E050E00E9461F64E
:10904000CA01B901A50194010E9461F6605D6093B7
:10905000C2048EE28093C304C701B601A501940146
:109060000E9461F6C62FCA01B901A50194010E94B0
:1090700061F6605D6093C404C05DC093C5048FEB6E
:1090800094E0CF91FF90EF90DF90CF90BF90AF90A2
:109090009F908F9008958F929F92AF92BF92CF92A0
:1090A000DF92EF92FF92FC01C080D180E280F380DA
:1090B00020E030E0A901C701B6010E9464F287FFF9
:1090C00004C0C701B601905802C0C701B6010E9492
:1090D000E1F76B017C016031F7E27F0781059105C3
:1090E00084F020E137E240E050E00E9461F6CA01DE
:1090F000B9012AE030E040E050E00E9461F6605D96
:1091000001C060E26093C10488EEC81683E0D8060F
:10911000E104F10494F0C701B60128EE33E040E029
:1091200050E00E9461F6CA01B9012AE030E040E057
:1091300050E00E9461F6605D01C060E26093C2048D
:10914000E4E6CE16D104E104F10494F0C701B601BF
:1091500024E630E040E050E00E9461F6CA01B90127
:109160002AE030E040E050E00E9461F6605D01C01E
:1091700060E26093C304FAE0CF16D104E104F10485
:109180009CF08AE0882E912CA12CB12CC701B6014D
:10919000A50194010E9461F6CA01B901A5019401DB
:1091A0000E9461F6605D01C060E26093C404C70183
:1091B000B6012AE030E040E050E00E9461F6605DD8
:1091C0006093C50481EC94E0FF90EF90DF90CF9026
:1091D000BF90AF909F908F90089520E030E040E2E4
:1091E00051E4FC0160817181828193810E94C9F206
:1091F0000E94E1F79B0177FF06C022273327261B39
:10920000370B8DE201C08BE28093C004C90168EE88
:1092100073E00E9475F9CB01EAE0F0E0BF010E9423
:1092200075F9805D8093C104C90164E670E00E9415
:1092300075F9CB01BF010E9475F9805D8093C2046E
:10924000C901BF010E9475F9282FCB01BF010E94FF
:1092500075F9805D8093C3048EE28093C404205D21
:109260002093C50480EC94E00895AC01952F991FDC
:109270009927991F29F022273327241B350B01C07A
:109280009A01483E5340ACF0C90168EE73E00E9479
:1092900075F9CB01EAE0F0E0BF010E9475F9805D4D
:1092A0008093C204C90164E670E00E9475F9CB01A5
:1092B00012C024363105B4F0911102C080E201C021
:1092C0008DE28093C204C90164E670E00E9475F9E2
:1092D000CB01EAE0F0E0BF010E9475F9805D809368
:1092E000C3040EC080E28093C2048093C3042A307A
:1092F000310584F091118DE28093C304EAE0F0E03F
:10930000C901BF010E9475F9CB01BF010E9475F927
:10931000805D05C0911102C080E201C08DE28093A2
:10932000C404C9016AE070E00E9475F9805D809311
:10933000C50482EC94E008959C0197FD0EC084362C
:10934000910584F064E670E00E9475F9CB016AE053
:1093500070E00E9475F9805D06C031952195310954
:109360008DE201C080E28093C3042A30310564F0AD
:10937000EAE0F0E0C901BF010E9475F9CB01BF012D
:109380000E9475F9805D01C080E28093C404C90128
:109390006AE070E00E9475F9805D8093C50483ECFB
:1093A00094E00895CF92DF92EF92FF926B017C01DF
:1093B00083E3C816D104E104F10470F082E3C81A13
:1093C000D108E108F10862E370E080E090E00E94DB
:1093D000969F0E9472E7ECCFC701B6010E94969F4C
:1093E000FF90EF90DF90CF900C9472E7CF93DF93D4
:1093F000E5E4F8E08491EF012196882321F00E94B2
:109400008384FE01F7CFE1E4F8E08491EF01219637
:10941000882321F00E948384FE01F7CF62B3669512
:10942000617070E080E090E00E94259162B361700D
:1094300070E080E090E00E9425918AE00E948384A1
:10944000EDE3F8E08491EF012196882321F00E945A
:109450008384FE01F7CF60910601862F660F990B7A
:10946000AA0BBB0BBC01CD01662797FD639577273F
:10947000882799270E94259162B362FB662760F9CD
:1094800070E080E090E00E9425918AE00E94838451
:10949000E9E3F8E08491EF012196882321F00E940E
:1094A0008384FE01F7CF6091060166FB662760F9B1
:1094B00070E080E090E00E9425916091060165FBDC
:1094C000662760F970E080E090E00E9425918AE0D4
:1094D0000E948384E4E3F8E08491EF0121968823DD
:1094E00021F00E948384FE01F7CF6091060163FBA7
:1094F000662760F970E080E090E00E94259160911D
:1095000006016295617070E080E090E00E94259114
:109510008AE00E948384EFE2F8E08491EF012196D3
:10952000882321F00E948384FE01F7CF6091060119
:109530006695617070E080E090E00E9425916091F6
:10954000060162FB662760F970E080E090E00E940F
:1095500025918AE0DF91CF910C94838467FD5CC0F4
:10956000823021F128F4882349F0813069F054C019
:10957000833071F1843009F43DC04EC0662311F090
:10958000A19A8FC0A1988DC09FB7662329F0F89447
:1095900080910801806804C0F894809108018F7759
:1095A000809308019FBF47FF4CC07FC09FB76623D1
:1095B00029F0F89480910801806404C0F8948091A7
:1095C00008018F7B809308019FBF47FF40C06FC099
:1095D0009FB7662329F0F89480910801886004C041
:1095E000F89480910801877F809308019FBF47FF0F
:1095F0003EC05AC09FB7662329F0F89480910801B5
:10960000826004C0F894809108018D7F80930801E6
:109610009FBF47FF39C04AC047FD49C08230B9F0FB
:1096200028F4882341F0813061F008958330F9F007
:10963000843051F10895442311F0A09A0895A09820
:109640000895442311F0A29A0895A29808959FB70F
:10965000442329F0F89480910801806204C0F894B2
:10966000809108018F7D809308019FBF08959FB767
:10967000442329F0F894809108018061F4CFF89494
:10968000809108018F7EEFCF9FB7442329F0F89493
:10969000809108018460E7CFF894809108018B7F66
:1096A000E2CF47FFC8CF089508950895089508951B
:1096B000643079F028F4613041F0623041F008956F
:1096C000683051F0603141F0089540E003C040E05F
:1096D00004C041E060E002C041E061E03FCF5F983C
:1096E0008EBD00000DB407FEFDCF8EB56EBD00002F
:1096F0000DB407FEFDCF8EB55F9A0895CF93DF932B
:1097000000D01F921F92CDB7DEB795E0E8E9F2E0F6
:10971000DE01119601900D929A95E1F7E1E0F0E0FB
:10972000EC0FFD1FE80FF11D808190E00F900F906E
:109730000F900F900F90DF91CF91D1CF24E0820254
:10974000C0011124FC01EB51FB4E4081518162812B
:109750007381FC01EC51FB4F40835183628373831F
:10976000E091BB04F091BC0482899389A489B589F6
:109770008093B7049093B804A093B904B093BA044B
:109780008FEF9FEF9093BE048093BD040895CF9315
:10979000DF932FB7F89494E08902E0011124FE01D1
:1097A000EB51FB4E60817181828193812FBF0E94BA
:1097B0006AF2CC52DB4F288139814A815B810E9459
:1097C000C9F2DF91CF9108950E9451C5882321F0FD
:1097D00080E00E946767F8CF8091BD049091BE043D
:1097E000892BB1F70895BC0180E090E04AE00E9427
:1097F000BD908DE00E9483848AE00C948384CF9393
:10980000DF931F92CDB7DEB7789484B5826084BDB4
:1098100084B5816084BD85B5826085BD85B5816074
:1098200085BD80916E00816080936E0010928100F2
:1098300080918100826080938100809181008160AD
:10984000809381008091800081608093800080916E
:10985000B10084608093B1008091B00081608093FA
:10986000B00080919100826080939100809191007E
:10987000816080939100809190008160809390003E
:109880008091A10082608093A1008091A1008160FD
:109890008093A1008091A00081608093A0008091BE
:1098A0002101826080932101809121018160809358
:1098B00021018091200181608093200180917A00B4
:1098C000846080937A0080917A00826080937A002D
:1098D00080917A00816080937A0080917A0080681C
:1098E00080937A001092C10082E08093C0001092B1
:1098F000C50087E08093C4008091C100806180939F
:10990000C1008091C10088608093C1008091C10036
:1099100080688093C1008091C1008F7D8093C100D9
:109920001092C704E8EEF9E084918F010F5F1F4F9A
:10993000882321F00E948384F801F6CFE5EDF6E15B
:1099400084918F010F5F1F4F882321F00E94838431
:10995000F801F6CF14B710FF0DC0EFEDF9E08491D8
:109960007F019FEFE91AF90A882321F00E9483847E
:10997000F701F5CF11FF0DC0EEECF9E084917F0106
:109980009FEFE91AF90A882321F00E948384F701E6
:10999000F5CF12FF0DC0ECEBF9E084917F019FEF52
:1099A000E91AF90A882321F00E948384F701F5CF90
:1099B00013FF0DC0EBEAF9E084917F019FEFE91AF4
:1099C000F90A882321F00E948384F701F5CF15FF5F
:1099D0000CC0EAE9F9E084918F010F5F1F4F8823E3
:1099E00021F00E948384F801F6CF14BEE3E9F9E088
:1099F00084918F010F5F1F4F882321F00E94838481
:109A0000F801F6CF80E20E948384ECE8F9E08491CB
:109A10008F010F5F1F4F882321F00E948384F8017C
:109A2000F6CF8AE00E948384E5EDF6E184918F0110
:109A30000F5F1F4F882321F00E948384F801F6CF27
:109A4000ECE7F9E084918F010F5F1F4F882321F02D
:109A50000E948384F801F6CFE8E6F9E084918F0153
:109A60000F5F1F4F882321F00E948384F801F6CFF7
:109A7000EFE2F9E084918F010F5F1F4F882321F0FF
:109A80000E948384F801F6CFE5EDF6E184918F0121
:109A90000F5F1F4F882321F00E948384F801F6CFC7
:109AA000E8E1F9E084918F010F5F1F4F882321F0D7
:109AB0000E948384F801F6CFE5EDF6E184918F01F1
:109AC0000F5F1F4F882321F00E948384F801F6CF97
:109AD00080911B1590911C15BE016F5F7F4F009701
:109AE00019F0681B790B02C06152754189E099E059
:109AF0000E9405A460EF74E082EF98E00E9405A444
:109B00008AE00E94838481E08093CF048093D00414
:109B10008093D1048093D2048093D3040E9473D0A5
:109B20008CE0EAEFF3E0A5EFB4E101900D928A95A5
:109B3000E1F70E9452C3809101018064809301018A
:109B40008091010180618093010180910101886011
:109B5000809301016D9A80910101806280930101DF
:109B600088E00E94C3ED809101018860809301012B
:109B700086E00E94C3ED6C9A82E00E94C3ED87EDFF
:109B800080937A0010927E0010927D0080917E007A
:109B9000816080937E0080917E00846080937E004F
:109BA00080E888BD80916E00846080936E006AEFCB
:109BB00070E080E090E00E94969F85E090E09093B6
:109BC000CD048093CC0460E0809123029091240224
:109BD0000E942C8120E030E040EA50E40E9464F2D0
:109BE00087FF0AC0809123029091240240979093AE
:109BF000240280932302E7CF81E391E09093260231
:109C00008093250260E08091CA049091CB040E9469
:109C10002C8120E030E848E953E40E94C3F818168C
:109C200054F48091CA049091CB0440969093CB0455
:109C30008093CA04E7CF80912102909122020E9472
:109C4000C0E420E030E040EA50E40E9464F287FF84
:109C50000AC08091210290912202409790932202A3
:109C600080932102E8CF8091C8049091C9040E949A
:109C7000C0E420E030E046E153E40E94C3F8181647
:109C800054F48091C8049091C90440969093C904FB
:109C90008093C804E8CF98E288E10FB6F894A895BD
:109CA000809360000FBE909360001FB7F89480917E
:109CB000CE04811124C0EEE8F7E18491E4EDF7E1F0
:109CC0009491E82FF0E0EE0FFF1FE15CF84EA591B4
:109CD000B491EC91E92321F461E085E30E94A09E18
:109CE00085E30E94C1928CB580618CBD8CB5806487
:109CF0008CBD84E30E94C19283E30E94C192809153
:109D0000CE048F5F8093CE041FBF579A1AE5E12ED1
:109D100013E0F12E10E0F70161917F0170E0812FD7
:109D2000EDDC1F5F1530B9F7999A989A8091070179
:109D30008068809307019A9A8091070180648093DC
:109D400007018091070180628093070180910701DC
:109D500088608093070180910701806180930701EB
:109D600080910701826080930701809107018460E0
:109D700080930701BFE5EB2EB3E0FB2E10E0F70167
:109D800061917F01812F94DC1F5F1530C1F78091B5
:109D90000A01826080930A0180910A0181608093A8
:109DA0000A0180910A01846080930A0180910A016E
:109DB000806480930A0180910A01806880930A017F
:109DC0000F9A179A0E9A169A0D9A159A0C9A149A37
:109DD0000B9A139A26982E9A25982D9A24982C9AA5
:109DE000389A4098179A10921515399A4198169AF0
:109DF000109216153A9A4298159A109217153B9A96
:109E00004398149A3C9A4498809180008C7F809368
:109E1000800080918100877E88608093810080919E
:109E200080008F738093800080918100887F8260A2
:109E30008093810080E090E4909389008093880073
:109E4000109285001092840080916F008260809350
:109E50006F0081E08093930D78940E944FB76C9AC5
:109E60000E9407770E947BA22091580D30E0790173
:109E7000F8E3EF1AF108F7FE04C0790187E3E81A66
:109E8000F108F594E7942E51310936952795F22E75
:109E90000E94E2940DE618E023E147E06CE08E2D8D
:109EA0000E94189384E00E94C1A20091580D10E016
:109EB00002571109169507956091590D625140E4BA
:109EC00053E08F2D0E9495936091590D665046E4A2
:109ED00053E0802F0E9495930E94E0928111DACF87
:109EE00064EC79E080E090E05DDA40E6542E5DE0DD
:109EF000452E66E0C62E6AE0D62E70E0A72E70E0F2
:109F0000B72E2AE0722E30E2632E8091D206853081
:109F100010F40E943BC680914C0D8823E9F00E940A
:109F2000CE9F0091480D1091490D20914A0D30911E
:109F30004B0DDC01CB01801B910BA20BB30BB7FDCA
:109F40000BC010924C0D8091A20A811112C16AD6E9
:109F50008091A20A81110DC18091D206882309F453
:109F600098C080919F0A882309F480C00091D1068F
:109F7000509E800111240F501B4F69E47AE0C80104
:109F80000E94E3F1892BF9F083E99CE00E94667C52
:109F900083E99CE00E941A7E1092A00A10929F0A08
:109FA000E6E3FAE084918F010F5F1F4F882341F0B1
:109FB0000E948384F801F6CF8091A00A811156C0D7
:109FC0000E94A06955C0F80101900020E9F731977F
:109FD0007F01E01AF10A1092930C6EE470E0C80160
:109FE0000E94CCF94C01009729F4F7013197E00F5A
:109FF000F11F0EC060E270E00E94CCF98C010F5F8F
:10A000001F4F6AE270E0C4010E94CCF9FC01319755
:10A01000418272821382F80101900020E9F73197A2
:10A02000AF01401B510BB80183E99CE00E94987C72
:10A030008091930C882309F4BFCFE2EBFBE084917D
:10A040008F010F5F1F4F882321F00E948384F80146
:10A05000F6CFEFEEF9E084918F010F5F1F4F882359
:10A0600009F4AACF0E948384F801F5CF0E94386AD0
:10A070008091D206882369F081508093D206809126
:10A08000D1068F5F853018F48093D10602C01092FC
:10A09000D1068091F004882309F461C0E5EDF6E172
:10A0A00084918F010F5F1F4F882321F00E948384CA
:10A0B000F801F6CFE7E2FAE084918F010F5F1F4FBE
:10A0C000882321F00E948384F801F6CF8091F00468
:10A0D00080FD51C08091F00484FD4DC090E2F92EC6
:10A0E0008091F00481FD64C08091F00485FD60C022
:10A0F00000E28091F00482FD77C08091F00486FD3B
:10A1000073C010E28AE00E9483841F926F921F92B4
:10A110001F931F920F931F92FF92DF92CF921F9275
:10A120000E94B8941092F0040FB6F894DEBF0FBEF0
:10A13000CDBF8091F903882391F01092A10A83E9A1
:10A140009CE00E94667C83E99CE00E941A7E10924B
:10A15000A00A10929F0A0E94856C0E949BE480E0F6
:10A160000E946767A114B10409F4CFCE0E940000D9
:10A17000C8CEA7D4F1CE6091E4047091E50480913B
:10A18000E6049091E7040E946AF22091D404309191
:10A19000D5044091D6045091D7040E94C9F2AB0176
:10A1A000BC0183E29AE00E94C1A388E5F82E98CF13
:10A1B0006091E8047091E9048091EA049091EB04C5
:10A1C0000E946AF22091D8043091D9044091DA04B7
:10A1D0005091DB040E94C9F2AB01BC018FE19AE00F
:10A1E0000E94C1A309E585CF6091EC047091ED0454
:10A1F0008091EE049091EF040E946AF22091DC04B9
:10A200003091DD044091DE045091DF040E94C9F2D8
:10A21000AB01BC018BE19AE00E94C1A31AE572CFA9
:10A220004F925F926F927F928F929F92AF92BF9266
:10A23000FF920F931F93CF93DF93182F8CE69CE030
:10A240009093F4088093F3081092880C82E090E0D9
:10A25000A0E0B0E08093710C9093720CA093730C0B
:10A26000B093740C1092F2081092EE081092EF085E
:10A270001092F0081092F1088FEF9FEFDC018093AD
:10A28000EA089093EB08A093EC08B093ED08112333
:10A2900079F1153008F0F9C040E060E070E0CB01E2
:10A2A0000E941DC9882309F4F0C020E1129FC0015B
:10A2B00011248652994FFC01E254FE4F20812F77E2
:10A2C00009F0E3C03C96408151816281738144363C
:10A2D00051056105710508F4D8C0349780809180DC
:10A2E000A280B38081149104A104B10421F4CDC0F3
:10A2F000812C912C540140E0C501B4010E941DC97C
:10A30000F82E882309F4C1C08091F5069091F606D5
:10A310008115924009F0B9C0A091FA06AA2309F468
:10A32000B4C06091F8067091F9066115710509F4E1
:10A33000ACC02091F706222309F4A7C0A093830C98
:10A340002093750C80E030E0E1E0F0E0C82FAF0131
:10A35000082E02C0440F551F0A94E2F72417350750
:10A3600041F0982F8F5F983089F789E080937E0CB9
:10A370008CC080937E0C209100073091010721153D
:10A38000310519F040E050E008C020910E073091EF
:10A390000F0740911007509111072093760C3093CE
:10A3A000770C4093780C5093790C24013501460EBC
:10A3B000571E611C711C4092840C5092850C609257
:10A3C000860C7092870CE091FB06F091FC06F093EE
:10A3D0008A0CE093890CB0E00E947DF6460E571E71
:10A3E000681E791E40928B0C50928C0C60928D0CE2
:10A3F00070928E0C85E0EE0FFF1F8A95E1F7E15019
:10A40000FE4FEF2FFF27E6954E0E5F1E611C711C5D
:10A4100040927F0C5092800C6092810C7092820C62
:10A420002091FD063091FE062115310521F08901AC
:10A4300020E030E008C000910A0710910B0720913E
:10A440000C0730910D07B501A4014419550966099F
:10A450007709400F511F621F731F04C076956795DF
:10A4600057954795CA95D2F740937A0C50937B0C39
:10A4700060937C0C70937D0C453F2FE05207610583
:10A48000710528F48CE08093880CF12C1AC0453FAC
:10A490005F4F6105710510F480E111C080911607CE
:10A4A00090911707A0911807B091190780938B0C12
:10A4B00090938C0CA0938D0CB0938E0C80E28093C3
:10A4C000880C8F2DDF91CF911F910F91FF90BF903E
:10A4D000AF909F908F907F906F905F904F90089576
:10A4E000EF92FF920F931F93CF93DF93CDB7DEB719
:10A4F0006F970FB6F894DEBF0FBECDBF7B0104E1AE
:10A500001BE026E13BE0F8013183208322E0209329
:10A510004D0D90933A0A8093390A40E050E0BA0119
:10A520008AE19BE00E94DC79F801808191812BE136
:10A53000FC013496DE01159601900D922A95E1F703
:10A54000FC01828193819C838B838BE893E09A83C7
:10A550008983A701BE016F5F7F4F87EE93E00E9462
:10A56000D796CE0101960E9454AF6F960FB6F8941D
:10A57000DEBF0FBECDBFDF91CF911F910F91FF9036
:10A58000EF9008951092A10A8091960C882321F0F3
:10A5900083E99CE00C941A7E08956F927F928F92CB
:10A5A0009F92AF92BF92DF92EF92FF920F931F9311
:10A5B000CF93DF93CDB7DEB7AE970FB6F894DEBF7B
:10A5C0000FBECDBF2091A20A222309F406C2D62EC7
:10A5D0007C018091960C882309F4A5C0442309F4DA
:10A5E000CFC18091AE0C882329F1E2EBFBE084918E
:10A5F0008F010F5F1F4F882321F00E948384F80191
:10A60000F6CFEFE6FBE084918F010F5F1F4F8823A9
:10A6100021F00E948384F801F6CF61E070E080E0D1
:10A6200090E00E9425918AE00E94838486E69BE068
:10A630000E945CAF84EB9CE09EA78DA78FE2809385
:10A64000B30C81E0898310E00FE180916B0C181747
:10A6500078F4019FC0011124AE014F5F5F4FBE012E
:10A66000635D7F4F8B5C944F0E9499BE1F5FEDCF5F
:10A67000898187FD0FC0AE014F5F5F4FBE01635DF3
:10A680007F4F8FE89CE00E9499BE8DA59EA5019703
:10A690009EA78DA7EDA5FEA51082E091AE0C84E0EB
:10A6A000E89FF0011124E155F34F8091440D909102
:10A6B000450DA091460DB091470D80839183A283F3
:10A6C000B383E5EDF6E184918F010F5F1F4F88237F
:10A6D00021F00E948384F801F6CFB7018DE49BE05E
:10A6E0000E941EA46091AE0C9DE8699FB0011124E8
:10A6F0006D54734F82E49BE00E941EA44091440D70
:10A700005091450D6091460D7091470D8CE39BE093
:10A710000E9487A38AE00E9483848091AE0C8F5FA1
:10A720008093AE0C27C04423C1F0E5EDF6E184919F
:10A730008F010F5F1F4F882321F00E948384F8014F
:10A74000F6CFECE2FBE084918F010F5F1F4F88236F
:10A7500089F00E948384F801F6CF1092AE0C82E05B
:10A76000B82E10C1B70183E19BE00E941EA48AE0CD
:10A770000E94838407DF1D8218861C821B828BE85F
:10A7800093E09A83898385EF9AE09093150B8093E9
:10A79000140BF70180818F3209F05CC087010F5FD5
:10A7A0001F4FCE0101964C010115110509F458C047
:10A7B0006FE270E0C8010E94CCF95C01009709F4D7
:10A7C00050C00817190708F04CC03C01601A710A04
:10A7D000A301B801CE0180960E94ECF9E0E2F0E01E
:10A7E000EC0FFD1FE60DF71D10826091140B7091A8
:10A7F000150B6115710511F06C5F7F4F21E0AE0103
:10A80000405E5F4FCE0105960E940B8081111AC0F9
:10A81000EFEFFAE084918F010F5F1F4F811104C0A9
:10A820008E01005E1F4F04C00E948384F801F2CFA6
:10A83000F80181918F01882319F00E948384F8CF59
:10A840008EE287C09092150B8092140B85010F5FEA
:10A850001F4FAACF86E19BE09093150B8093140BBA
:10A8600087019091140B8091150B692F782FDD20B3
:10A8700009F459C06115710511F06C5F7F4F21E03B
:10A88000A80183E99CE00E940B80882309F447C05B
:10A890008091A40C9091A50CA091A60CB091A70C4E
:10A8A0008093400D9093410DA093420DB093430DC2
:10A8B0001092440D1092450D1092460D1092470DC6
:10A8C000B80181EF9AE00E941EA44091400D509182
:10A8D000410D6091420D7091430D89EE9AE00E9406
:10A8E00087A38AE00E948384EAEDFAE084917F01E5
:10A8F0009FEFE91AF90A882321F00E948384F70167
:10A90000F5CFB80180E090E0EBDD8091B10A8823BB
:10A9100019F081EB9AE001C0C80160E02AC0B801DB
:10A9200086EC9AE010C06115710511F06C5F7F4FE5
:10A9300026E5A80183E99CE00E940B8081110CC0F0
:10A94000B80182EB9AE00E941EA48EE20E948384EA
:10A950008AE00E9483840FC081E080939F0AB70140
:10A9600080EA9AE00E941EA48AE00E94838460E04C
:10A97000C8010E94BAC8CE0101960E9454AF2DC0F2
:10A98000BB24B394E5EDF6E184918F010F5F1F4F77
:10A99000882321F00E948384F801F6CFE7E2FBE0F0
:10A9A00084918F010F5F1F4F882321F00E948384C1
:10A9B000F801F6CFE1E0BE1619F0E1E2FBE002C0DB
:10A9C000EBE1FBE084918F010F5F1F4F882309F4B7
:10A9D000C9CE0E948384F801F5CFAE960FB6F894E5
:10A9E000DEBF0FBECDBFDF91CF911F910F91FF90C2
:10A9F000EF90DF90BF90AF909F908F907F906F907F
:10AA00000895CF92DF92EF92FF920F931F93CF930F
:10AA1000DF93CDB7DEB7EDB6FEB6DC010D900020BA
:10AA2000E9F79D01281B390B2C5F3F4F4DB75EB7EF
:10AA3000421B530B0FB6F8945EBF0FBE4DBF0DB750
:10AA40001EB70F5F1F4F9F938F9389E99AE09F93E3
:10AA50008F931F930F930E94FDF1680154E0C50E80
:10AA6000D11C0F900F900F900F900F900F90F60148
:10AA70008081882339F090E00E9490F9F60181935B
:10AA80006F01F5CF60E0C8010E94D7C2882319F09A
:10AA9000C8010E94F5AC85E99AE09093F60880938E
:10AAA000F5080E94F3C20FB6F894FEBE0FBEEDBECD
:10AAB000DF91CF911F910F91FF90EF90DF90CF909A
:10AAC0000895AF92BF92CF92DF92EF92FF920F93D1
:10AAD0001F93CF93DF93CDB7DEB7AA970FB6F89445
:10AAE000DEBF0FBECDBF8091F40A8F938091F30A31
:10AAF0008F938CE89AE09F938F937E0181E2E80E1A
:10AB0000F11CFF92EF920E94FDF10F900F900F90B9
:10AB10000F900F900F9010E0F70101900020E9F7DF
:10AB20003197EE19FF091E1774F46701C10ED11C8D
:10AB300017FDDA94F601808190E00E9490F9F60109
:10AB400080831F5FE9CF40E050E0BA0189EF9AE0CF
:10AB50000E94DC7900E0CE0101966C018091FC0A34
:10AB6000823028F4011114C08FEF9FEF16C080913E
:10AB7000010B9091020BA091030BB091040B8F710C
:10AB80009927AA27BB27892B8A2B8B2B59F71AC009
:10AB90008091F30A9091F40A01969093F40A8093BD
:10ABA000F30AAA960FB6F894DEBF0FBECDBFDF91B1
:10ABB000CF911F910F91FF90EF90DF90CF90BF90BA
:10ABC000AF90089540E050E0B60189EF9AE00E940E
:10ABD000967B18163CF6F60101900020E9F73197B4
:10ABE0001E2F1C19115068F05601A10EB11C17FD43
:10ABF000BA94F501808190E00E9490F9F50180837C
:10AC0000F1CF8A858E3709F4A9CF45E050E0B7012E
:10AC1000C6010E94DEF9892B09F0A0CFC701F1DE41
:10AC200001E09CCFCF92DF92EF92FF921F93CF93E0
:10AC3000DF931092A20A8091FC0A882321F089EF09
:10AC40009AE00E941A7E1092700C10926D0C85E3AF
:10AC500080936C0C0E94CE9FEB01A89580916C0CA8
:10AC60000E94C1928CE69CE00E94BE452398229AE5
:10AC7000219A209A289A85E080936E0C82E58CBDFB
:10AC80001DBC1AE08FEF0E94C3451150D9F720E098
:10AC900030E0A90160E08CE69CE00E94E945182FB5
:10ACA00080936F0C813049F00E94CE9F6C1B7D0B0E
:10ACB000613D774060F381E054C02AEA31E040E032
:10ACC00050E068E08CE69CE00E94E94582FF03C00A
:10ACD0001093700C0EC014E00E94C84580936F0C56
:10ACE0001150D1F78A3A11F082E03BC082E08093A4
:10ACF000700C8091700C823021F0C12CD12C760127
:10AD000005C0C12CD12CE12C80E4F82E20E030E0ED
:10AD1000A90167E38CE69CE00E94E945A701960142
:10AD200069E28CE69CE00E94E94580936F0C8823E1
:10AD300049F00E94CE9F6C1B7D0B613D774030F344
:10AD40008AE00FC08091700C823011F520E030E075
:10AD5000A9016AE38CE69CE00E94E945882351F052
:10AD600088E080936D0C8CE69CE00E94BE45E5ED8A
:10AD7000F6E119C00E94C845807C803C19F483E04C
:10AD80008093700C0E94C8450E94C8450E94C84527
:10AD90008CE69CE00E94BE4510926E0C81E040DA89
:10ADA000811131C015C08491EF012196882321F0D3
:10ADB0000E948384FE01F7CFEEE7FAE08491EF0171
:10ADC0002196882309F456C00E948384FE01F6CFA1
:10ADD00080E026DA811117C0E2EBFBE08491EF01FD
:10ADE0002196882321F00E948384FE01F7CFEAE6B2
:10ADF000FAE08491EF012196882309F43BC00E9478
:10AE00008384FE01F6CF61E77CE089EF9AE00E943F
:10AE1000F77B811116C0E2EBFBE08491EF012196F4
:10AE2000882321F00E948384FE01F7CFE9E5FAE050
:10AE30008491EF0121968823E9F00E948384FE012A
:10AE4000F7CF81E08093A20AE5EDF6E18491EF016E
:10AE50002196882321F00E948384FE01F7CFEDE440
:10AE6000FAE08491EF012196882321F00E948384E7
:10AE7000FE01F7CF8BE1E9EFFAE0AAE1BBE0019038
:10AE80000D928A95E1F78091F70A9091F80A9093D4
:10AE9000190B8093180B86E19BE09093150B809320
:10AEA000140BDF91CF911F91FF90EF90DF90CF9027
:10AEB0000895EF92FF921F93CF93DF931F92CDB728
:10AEC000DEB7182FE2EBFBE084917F012FEFE21A4F
:10AED000F20A882331F099830E948384F7019981D3
:10AEE000F3CFE12FF92F84917F019FEFE91AF90A3F
:10AEF000882321F00E948384F701F5CF6091E60654
:10AF00007091E7068091E8069091E9060E942591EC
:10AF10008AE00E9483840E940E6A1092E5061092D5
:10AF2000E4060F90DF91CF911F91FF90EF9008956D
:10AF30000F931F93CF93DF938C01EB019091800AC5
:10AF40002091810A921307C084E79AE00E9410A220
:10AF50000E9472E7F3CFF801A081B1814881598145
:10AF600080917F0A34E0839FF0011124E858F54F67
:10AF7000B387A287558744879F5F9093800A8F5F2E
:10AF8000821719F080937F0A02C010927F0ADF9126
:10AF9000CF911F910F910895EF92FF920F931F93FE
:10AFA000CF93DF931F92CDB7DEB78B01622F49831A
:10AFB0000E94A36690918C0D8091E30649818917C8
:10AFC00008F43FC090918E0D8091E206981708F426
:10AFD00038C0442399F120E030E0F801E20FF31F7C
:10AFE000E491EE2319F02F5F3F4FF7CF86E190E019
:10AFF000821B930B97FD01969595879536E1F32E6D
:10B0000049EEE42EE80E8E2D8F0D87FD0EC080E2F6
:10B010000E941694FA94F7CFF8018491882339F0AE
:10B020000E94DBA2F81A0F5F1F4F1F14ACF31F140E
:10B0300044F480E20E941694FA94F9CF86E1F82E47
:10B04000F4CF0F90DF91CF911F910F91FF90EF9070
:10B050000895CF92DF92EF92FF920F931F93CF93B9
:10B06000DF9300D01F92CDB7DEB77C018B0129831F
:10B070003A834B835C830E94DE6583E080932A02DF
:10B08000F092DE06E092DD061093DC060093DB060C
:10B0900029813A814B815C81CA01B9010E9468F221
:10B0A0002AE037ED43E25CE30E94C9F20E94E1F737
:10B0B0006093D7067093D8068093D9069093DA06EA
:10B0C0000E946AF26B017C019B01AC0160E070E8B8
:10B0D00087E794E40E949CF60E94E1F76093D30610
:10B0E0007093D4068093D5069093D606F8016081BC
:10B0F0007181828193810E9468F22AE037ED43E2F8
:10B100005CE30E94C9F2A70196010E949CF60E948E
:10B11000E6F76093490A70934A0A80934B0A90932A
:10B120004C0A83E490E790932902809328028AE8EE
:10B1300093EB9093E1068093E0061092DF060F9068
:10B140000F900F900F90DF91CF911F910F91FF9073
:10B15000EF90DF90CF900895AF92BF92CF92DF92A1
:10B16000EF92FF920F931F93CF93DF937C01EB013C
:10B170005A0169010E94DE6523E020932A02F092C1
:10B18000DE06E092DD06D093DC06C093DB06A50167
:10B19000BB0C660B770B4093D7065093D806609391
:10B1A000D9067093DA06C601DD0CAA0BBB0B841B13
:10B1B000950BA60BB70B8093D3069093D406A09360
:10B1C000D506B093D60688819981092E000CAA0B6A
:10B1D000BB0B841B950BA60BB70B8093490A90936E
:10B1E0004A0AA0934B0AB0934C0A87E292E79093E5
:10B1F0002902809328021093E1060093E006109242
:10B20000DF06DF91CF911F910F91FF90EF90DF90BC
:10B21000CF90BF90AF900895EF92FF920F931F933E
:10B22000CF93DF931F92CDB7DEB7082F162FE3E73A
:10B23000FCE084917F012FEFE21AF20A882331F0BB
:10B2400099830E948384F7019981F3CFE02FF92F2E
:10B2500084917F019FEFE91AF90A882321F00E9467
:10B260008384F701F5CFE1E7FCE084917F012FEFC4
:10B27000E21AF20A882321F00E948384F701F5CFB5
:10B28000612F70E080E090E00E9425918AE00F90AD
:10B29000DF91CF911F910F91FF90EF900C948384D9
:10B2A0004F925F926F927F928F929F92AF92BF92D6
:10B2B000CF92DF92EF92FF92CF93DF93EEE6FCE026
:10B2C0008491EF012196882321F00E948384FE015E
:10B2D000F7CF209126043091270440912804509103
:10B2E00029046091F5147091F6148091F7149091EF
:10B2F000F8140E949DF642E00E944091EAE6FCE0CC
:10B300008491EF012196882321F00E948384FE011D
:10B31000F7CF20912A0430912B0440912C045091B6
:10B320002D046091F9147091FA148091FB1490919E
:10B33000FC140E949DF642E00E944091E6E6FCE08B
:10B340008491EF012196882321F00E948384FE01DD
:10B35000F7CF20912E0430912F044091300450916A
:10B3600031046091FD147091FE148091FF1490914E
:10B3700000150E949DF642E00E944091E2E6FCE04A
:10B380008491EF012196882321F00E948384FE019D
:10B39000F7CF60910115709102158091031590917E
:10B3A000041542E00E9440918FB7F8944090E51454
:10B3B0005090E6146090E7147090E8148090E914BF
:10B3C0009090EA14A090EB14B090EC14C090ED149F
:10B3D000D090EE14E090EF14F090F0148FBFE8E5F9
:10B3E000FCE08491EF012196882321F00E94838460
:10B3F000FE01F7CFC301B2010E942591E4E5FCE014
:10B400008491EF012196882321F00E948384FE011C
:10B41000F7CFC501B4010E942591E0E5FCE08491DD
:10B42000EF012196882321F00E948384FE01F7CF4B
:10B43000C701B6010E9425918AE0DF91CF91FF906C
:10B44000EF90DF90CF90BF90AF909F908F907F90C4
:10B450006F905F904F900C948384CF93DF9383E53C
:10B460000E946DC4882321F00E94DBC3EB0102C05F
:10B47000C0E0D0E0DD27C230D105BCF0E2EBFBE05C
:10B480008491EF012196882321F00E948384FE019C
:10B49000F7CFEEE2FCE08491EF012196882309F4D6
:10B4A00050C00E948384FE01F6CF88E40E946DC4E0
:10B4B0008823A9F00E94DBC3683771053CF0633232
:10B4C00081E078072CF062E271E002C068E770E08A
:10B4D000FE01EE0FFF1FE35AFB4E7183608386E48B
:10B4E0000E946DC48823A9F00E94DBC3FE01EE0F09
:10B4F000FF1FEB5AFB4E718360836F3F710519F09C
:10B5000014F06FEF70E077FF02C060E070E07183CD
:10B51000608382E40E946DC4882399F00E94DBC39B
:10B520006530710534F0683871052CF067E870E01B
:10B5300002C065E070E0CC0FDD1FC75ADB4E798397
:10B540006883DF91CF9108952F923F924F925F923F
:10B550006F927F928F929F92AF92BF92CF92DF9223
:10B56000EF92FF920F931F93CF93DF93CDB7DEB788
:10B570002E970FB6F894DEBF0FBECDBF8DE690E0DC
:10B580000E940BC581117DC180919E0483FD79C10C
:10B5900083E50E946DC4482E811106C082E50E9499
:10B5A0006DC4882309F46DC10E940BC40E94E1F7A9
:10B5B00070938B0460938A0480E00E9450E4609151
:10B5C0008A0470918B04072E000C880B990B0E9443
:10B5D0006AF220918C0430918D0440918E04509138
:10B5E0008F040E94C3F818160CF046C184EE92E056
:10B5F0009F938F9382E29CE09F938F931F920E9470
:10B60000B8940F900F900F900F900F9081E080935F
:10B61000150219821A821B821C821D821E821F82C1
:10B6200018861D8619862CE32A873CE13B8746E471
:10B630004C87E12CF12C00E81FEB812C912C54015C
:10B6400060918A0470918B04072E000C880B990B73
:10B650000E946AF26E87772E682E592E262F372F7A
:10B66000482F592FB701C8010E9464F28823C9F0FE
:10B6700020918C0430918D0440918E0450918F0460
:10B680006E85772D862D952D0E9464F2881F882760
:10B69000881F8D87442049F0882339F051E05D8769
:10B6A000C4C0EE867F2C602E512E0E94CE9F6B016F
:10B6B0007C01DC01CB012D813E814F815885821BAD
:10B6C000930BA40BB50BB7FD3AC0D701C601885147
:10B6D0009C4FAF4FBF4F8D839E83AF83B8870E942F
:10B6E00082E3EEE1FCE084918F010F5F1F4F88231E
:10B6F00021F00E948384F801F6CF81149104A10403
:10B70000B104B9F0D501C40188519C4FAF4FBF4F70
:10B71000BC01CD016C197D098E099F0928EE33E02B
:10B7200040E050E00E943FF6CA01B9010E94259115
:10B7300003C08FE30E9483848AE00E94838480E0B8
:10B740000E9467670E947DA320908C0430908D0436
:10B7500000918E0410918F049101A8016E85772DC0
:10B76000862D952D0E949CF69F7720E030E040E2E8
:10B7700051E481149104A104B10429F40E9464F2FB
:10B7800087FF07C004C00E94C3F8181614F44601CE
:10B7900057019D85992379F129813A814B815C81FB
:10B7A000211531054105510541F0D701C601821B24
:10B7B000930BA40BB50BB7FD1EC09101A8016985C1
:10B7C0007A858B859C850E949CF620E030E040ECD9
:10B7D0005FE30E9464F287FD61CFD701C601805A02
:10B7E0009541AF4FBF4F89839A83AB83BC83298632
:10B7F0003A860B871C87809115028823B1F081144B
:10B800009104A104B10429F4EE84F72C062D152D22
:10B8100017CF98EEC91A93E0D90AE108F108C818C1
:10B82000D908EA08FB08F7FCEFCF809115028823BE
:10B8300041F1AD8560E0AA2319F082E09CE002C0EE
:10B8400080E19CE02E960FB6F894DEBF0FBECDBF10
:10B85000DF91CF911F910F91FF90EF90DF90CF90EC
:10B86000BF90AF909F908F907F906F905F904F9020
:10B870003F902F900C941CC64110C8CE84E693E0F4
:10B88000B7CE2E960FB6F894DEBF0FBECDBFDF91B8
:10B89000CF911F910F91FF90EF90DF90CF90BF90CD
:10B8A000AF909F908F907F906F905F904F903F9060
:10B8B0002F900895809197049091980421E020930F
:10B8C000A00A40E060E00C94CD52CF938091A10A91
:10B8D00081110E94E44B8091A20A8823A9F180E59E
:10B8E0000E946DC4882319F00E94FCC303C080E548
:10B8F0000E943EC4C82F482F61E080919704909128
:10B9000098040E94CD5283E50E946DC4882381F083
:10B910000E94DBC3AB01BC014093440D5093450D25
:10B920006093460D7093470D83E99CE00E94DC799B
:10B930008091A20A882319F081E08093A10AC111A5
:10B9400003C0CF910C947F94CF910895CF93DF9350
:10B950008091A20A882349F1EFEDFBE08491EF0189
:10B960002196882321F00E948384FE01F7CF609105
:10B97000440D7091450D8091460D9091470D4AE020
:10B980000E94BD908FE20E9483846091400D70916F
:10B99000410D8091420D9091430D4AE00E94BD906F
:10B9A0008AE0DF91CF910C948384E1EFFBE08491F6
:10B9B000EF012196882321F00E948384FE01F7CFB6
:10B9C000DF91CF910895E0919704F09198048081E0
:10B9D000882329F0803209F410823196F8CF40E0B4
:10B9E00061E080919704909198040C94CD52CF928D
:10B9F000DF92EF92FF92CF93DF936A017B01C5EF55
:10BA0000D4E1E0919D0424E0E29FF0011124E45E82
:10BA1000FD4F2081318142815381FC016081718120
:10BA2000828193810E9479F79B01AC016C857D85B1
:10BA30008E859F850E949DF66C877D878E879F8768
:10BA40000E945AC5C701B6010E9472C2DF91CF9110
:10BA5000FF90EF90DF90CF900C94E44BCF92DF9269
:10BA6000EF92FF92CF93DF9381E080931502D1E0B4
:10BA7000C1E080911502882309F446C0CC2309F463
:10BA800043C080E00E94676760918A0470918B04D4
:10BA9000C0E06115710569F3072E000C880B990B46
:10BAA0000E946AF29B01AC0160918C0470918D043C
:10BAB00080918E0490918F040E949CF66B017C0112
:10BAC00020E030E0A9010E94C3F818165CF020E0E5
:10BAD00030E040E251ECC701B6010E9464F287FFFA
:10BAE000C8CF0BC020E030E040E251E4C701B6010E
:10BAF0000E94C3F818160CF0BCCFD093480A8DE80A
:10BB000095EA0E941495B4CFDF91CF91FF90EF900A
:10BB1000DF90CF900895CF92DF92EF92FF920F9334
:10BB20001F93CF93DF9300D01F92CDB7DEB7182FAE
:10BB3000662351F0109201091092FD081092FE0840
:10BB40001092FF08109200090E94CE9FC090FD083D
:10BB5000D090FE08E090FF08F09000099B01AC0136
:10BB60002C193D094E095F0957FD3DC017FD16C050
:10BB700040910109212F012E000C330B2C5F3F4F08
:10BB8000E42F042E000CFF0B2E173F0764F1411722
:10BB90002CF000E911E020E030E004C004EC19E0F2
:10BBA00020E030E0DC01CB01800F911FA21FB31F0A
:10BBB0008093FD089093FE08A093FF08B0930009BE
:10BBC00080ED97E09C838B838CE291E09A8389835C
:10BBD000BE016D5F7F4FCE010196AAD98091010908
:10BBE0008F5F809301090F900F900F900F90DF915E
:10BBF000CF911F910F91FF90EF90DF90CF9008951C
:10BC000060E086ED9BE00E941CC617981698159878
:10BC1000149808953F924F925F926F927F928F9205
:10BC20009F92AF92BF92CF92DF92EF92FF920F93CB
:10BC30001F93CF93DF930E94E44B8CE3C82E83E0E5
:10BC4000D82E05EF14E196E2E92E94E0F92EC0E03B
:10BC5000312CD0E0F60181916F010E946DC48823E0
:10BC6000B9F10E940BC44B015C01C33049F0F701EC
:10BC700020813181428153810E949CF64B015C01FD
:10BC8000F8012081318142815381C501B4010E94B4
:10BC90009CF62B013C012DEB37E346E855EB0E9467
:10BCA000C3F887FD0AC02DEB37E346E855E3C3012F
:10BCB000B2010E9464F218165CF4C33019F0332408
:10BCC000339401C0D1E0F80180829182A282B382D4
:10BCD000CF5F0C5F1F4FF4E0EF0EF11CC43009F092
:10BCE000B9CF332019F00E9452C303C0D1110E9472
:10BCF00086EDDF91CF911F910F91FF90EF90DF9034
:10BD0000CF90BF90AF909F908F907F906F905F90FB
:10BD10004F903F90C5CA2F923F924F925F926F9281
:10BD20007F928F929F92AF92BF92CF92DF92EF92CB
:10BD3000FF920F931F93CF93DF93CDB7DEB7629738
:10BD40000FB6F894DEBF0FBECDBF8A8B0E94E44BC6
:10BD5000409118025091190260911A0270911B02D1
:10BD60004093F9085093FA086093FB087093FC081D
:10BD700020911602309117023093F8082093F708AB
:10BD800024E630E030931702209316020E947DA330
:10BD900091E09093930D8A89811119C088E50E94E2
:10BDA0003EC4082F89E50E943EC4182F8AE50E94F0
:10BDB0003EC4282E011106C0111113C0882361F062
:10BDC000012F0FC0112369F0012F382E0BC011E095
:10BDD00001E02224239402C0182F082F3324339427
:10BDE00001C0312C0E945AC5311005C0011103C099
:10BDF000112309F408C180E090E0A0EAB0E4809348
:10BE0000A7049093A804A093A904B093AA049C014A
:10BE1000AD016091FD147091FE148091FF1490911A
:10BE200000150E9464F287FF0BC019821A821B82E0
:10BE30001C82BE016F5F7F4F87EA94E00E946BC255
:10BE400031100DC0011103C01111D8C0DCC0111197
:10BE500006C080E00E9416AC3320B1F3CFC0109230
:10BE6000F9141092FA141092FB141092FC14109210
:10BE7000F5141092F6141092F7141092F8140E9410
:10BE800052C3E5E8F2E02491298BEBEFFEE2C59086
:10BE9000D590E590F490EFEFFEE285909590A59017
:10BEA000B490A5019401C701B6010E94C3F8181609
:10BEB0002CF4A7019601C501B40104C0A5019401A9
:10BEC000C701B6010E9479F76D877E878F87988BAF
:10BED0008AEB682E8EE2782EF3016591759185913B
:10BEE00094912EEB422E2EE2522EF20125913591A5
:10BEF000459154910E9464F287FF02C0F30101C092
:10BF0000F20145905590659074902D853E854F8542
:10BF10005889CA01B9010E94C9F220E030E040E826
:10BF20005FE30E949DF60E9408F99B01AC01C301EA
:10BF3000B2010E94C9F269877A878B879C87E6E8FD
:10BF4000F2E084918D8720E030E040EC5FE3C501B2
:10BF5000B4010E94C9F22B013C012D85622F220FF2
:10BF6000770B880B990B0E946AF29B01AC01C3010D
:10BF7000B2010E94C9F269837A838B839C8320E09B
:10BF800030E040EC5FE3C701B6010E94C9F26B01EB
:10BF90007C012989622F220F770B880B990B0E9455
:10BFA0006AF29B01AC01C701B6010E94C9F26D8320
:10BFB0007E838F8398879E01275F3F4F4DEF54E12B
:10BFC000BE016F5F7F4FCE0105960E9488C110921F
:10BFD000F0041092F9141092FA141092FB141092BB
:10BFE000FC141092F5141092F6141092F71410929B
:10BFF000F81431102ECF01112CCF26CF81E00E94F2
:10C0000016AC311003C0222009F45DC080911515D3
:10C01000882321F08091161581111DC060E088EC05
:10C020009BE00E941CC6E5EDF6E184918F010F5F55
:10C030001F4F882321F00E948384F801F6CFE9EB9B
:10C04000FBE084918F010F5F1F4F8823E1F10E9475
:10C050008384F801F6CF0E9452C380E090E0A0E212
:10C06000B1E480939F049093A004A093A104B093A3
:10C07000A2048093A3049093A404A093A504B09376
:10C08000A6048091FD149091FE14A091FF14B0912C
:10C0900000158093A7049093A804A093A904B093DB
:10C0A000AA0419821A821B821C829E012F5F3F4FB5
:10C0B0004DEF54E163EA74E08FE994E00E9488C197
:10C0C00082E00E9416AC0E9452C38091920D809330
:10C0D000930D8091F9089091FA08A091FB08B09116
:10C0E000FC088093180290931902A0931A02B0934F
:10C0F0001B028091F7089091F808909317028093A3
:10C1000016020E947DA383E080932A02C9D862961A
:10C110000FB6F894DEBF0FBECDBFDF91CF911F9158
:10C120000F91FF90EF90DF90CF90BF90AF909F90D6
:10C130008F907F906F905F904F903F902F900895D9
:10C140004F925F926F927F928F929F92AF92BF9227
:10C15000FF920F931F93CF93DF93CDB7DEB72A974C
:10C160000FB6F894DEBF0FBECDBF10928709809145
:10C170008D09882339F00E945CA280E099EE0E942C
:10C180001495A9C420911602309117024091490AD2
:10C1900050914A0A60914B0A70914C0AC901840F70
:10C1A000951F2436310524F4853691053CF416C0DC
:10C1B0002436310531F08436910584F484E690E02C
:10C1C0000DC0473051056105710514F0069706C092
:10C1D0004A3F5F4F6F4F7F4F6CF406969093170264
:10C1E000809316021092490A10924A0A10924B0A42
:10C1F00010924C0A80911602909117028A30910594
:10C200003CF0883E43E094072CF087EE93E002C0B8
:10C210008AE090E090931702809316020E94CF76F6
:10C22000F82E0E94BDC580918C0D853198F4FF20B9
:10C2300049F08091910490919204892B19F005EDB9
:10C2400012E102C008EB11E123E14FE061E089E077
:10C250000E94189380918C0D8D3108F084C1883034
:10C2600008F03FC08091440AF11002C0811139C02A
:10C2700060918A0470918B04072E000C880B990B37
:10C280000E946AF220E030E040E05FE30E949DF609
:10C290000E94E1F7643671052CF46A30710524F4CC
:10C2A00046E003C042E101C04CE022E130E0241B43
:10C2B000310937FF02C02F5F3F4F359527953195E4
:10C2C000219531092B5F20938F0D27E02093900D4E
:10C2D000CB010E949C490E9413A385EB91E10E942F
:10C2E00006A380918C0D8D31D0F580918E0D853116
:10C2F000B0F120E030E040E05FE360918C047091A9
:10C300008D0480918E0490918F040E949DF60E946E
:10C31000E1F79B01643671050CF0D6C22A30310575
:10C320000CF0D0C246E022E130E0241B310937FF97
:10C3300002C02F5F3F4F35952795319521953109E3
:10C340002B5F20938F0D2CE12093900DCB010E9449
:10C350009C490E9413A385EB91E10E9406A3809162
:10C360008C0D853140F580918E0D813120F16091E9
:10C370008A0470918B04072E000C880B990B0E9485
:10C380006AF220918C0430918D0440918E0450917A
:10C390008F040E94C3F818160CF098C21092780D02
:10C3A00002E022E041E16DE088E59DE00E94A09C72
:10C3B00081E08093780D80918C0D883008F03FC02B
:10C3C00080913B0AF11002C0811139C0609188044C
:10C3D00070918904072E000C880B990B0E946AF259
:10C3E00020E030E040E05FE30E949DF60E94E1F72C
:10C3F000643671052CF46A30710524F446E003C0FC
:10C4000042E101C04CE022E130E0241B310937FF5A
:10C4100002C02F5F3F4F3595279531952195310902
:10C420002F5A20938F0D27E02093900DCB010E946F
:10C430009C490E9413A385EB91E10E9406A3809181
:10C440008C0D8D31D0F580918E0D8531B0F120E0CD
:10C4500030E040E05FE360917E0470917F04809162
:10C460008004909181040E949DF60E94E1F79B0157
:10C47000643671050CF035C22A3031050CF02FC23C
:10C4800046E022E130E0241B310937FF02C02F5F74
:10C490003F4F359527953195219531092F5A209396
:10C4A0008F0D2CE12093900DCB010E949C490E949E
:10C4B00013A385EB91E10E9406A380918C0D853139
:10C4C00040F580918E0D813120F16091880470914A
:10C4D0008904072E000C880B990B0E946AF22091A8
:10C4E0007E0430917F0440918004509181040E9429
:10C4F000C3F818160CF0F7C11092780D02E022E094
:10C5000042E168E588E59DE00E94A09C81E080937F
:10C51000780D80918C0D8C3130F580918E0D8431A9
:10C5200010F18091910490919204019644E6489F05
:10C530009001499F300D112437FF02C021503F4F19
:10C54000832F932F990F990B009769F028E620937A
:10C550008F0D2BE12093900D0E949C490E9413A304
:10C5600085E20E9416948091960C882349F0809170
:10C570008C0D843328F480918E0D8A3208F0BCC172
:10C5800080918C0D853328F480918E0D813308F0D5
:10C59000D9C160919004623048F080918C0D843351
:10C5A00028F480918E0D823308F0D1C180918C0DDA
:10C5B000813308F060C080918E0D893208F45BC031
:10C5C0000E944B942B013C018CE3882E912CA12CD2
:10C5D000B12CC301B201A50194010E943FF6CA012A
:10C5E000B901A50194010E943FF6CA01B62EA72EFB
:10C5F00049018E010F5F1F4F41E8441641E5540683
:10C6000041E06406710408F4BDC1B90128E130E0DD
:10C6100040E050E00E943FF629013A01AF92BF92FC
:10C62000C40168E170E00E9461F99F938F935F926B
:10C630004F928AE89CE09F938F931F930F930E94E1
:10C64000FDF10FB6F894DEBF0FBECDBF9AE04916DC
:10C6500051046104710408F0BFC197E0892F880F6D
:10C66000980F9195955A90938F0D80E38093900D3C
:10C67000C8010E9413A3E091520DF091530D8481E3
:10C680008111ECC0209126043091270440912804A8
:10C69000509129046091F5147091F6148091F7146B
:10C6A0009091F8140E949DF60E94E1F7CB010E9440
:10C6B0003549BC0182E399E00E94D7F920912A0410
:10C6C00030912B0440912C0450912D046091F91469
:10C6D0007091FA148091FB149091FC140E949DF6C5
:10C6E0000E94E1F7CB010E943549BC018DE299E03F
:10C6F0000E94D7F920912E0430912F0440913004EC
:10C70000509131046091FD147091FE148091FF14DA
:10C71000909100150E949DF62CEA35EC47E257E314
:10C720000E949DF620E030E048EC52E40E94C9F2FD
:10C730000E94E1F74B015C0197FD19C090E1891659
:10C7400097E29906A104B104E4F0C501B40120E127
:10C7500037E240E050E00E9461F6CA01B9012AE0E8
:10C7600030E040E050E00E9461F6605D0BC0B094A4
:10C77000A09490948094811C911CA11CB11C6DE22A
:10C7800001C060E26093C00428EE821623E09206A6
:10C79000A104B10494F0C501B40128EE33E040E0F7
:10C7A00050E00E9461F6CA01B9012AE030E040E0A1
:10C7B00050E00E9461F6605D01C060E26093C104D8
:10C7C000C501B40124E630E040E050E00E9461F68B
:10C7D0009AE0492E512C612C712CCA01B901A30198
:10C7E00092010E9461F6605D6093C204C501B401CC
:10C7F000A30192010E9461F64B015C01672B682B3B
:10C80000692B79F08EE28093C304CA01B901A301B8
:10C8100092010E9461F6605D6093C40480E3880D1C
:10C8200015C0CA01B901A30192010E9461F66623F5
:10C8300039F08EE28093C304605D6093C40405C048
:10C8400080E28093C4048093C30480E28093C50493
:10C8500060EC74E086E299E00E94D7F980918C0D3B
:10C860008632A8F480918E0D8E3188F008E020E8A1
:10C870004EE160E088E59DE00E94A09C80918C0DD7
:10C88000863228F480918E0D8F3108F0A7C08091F8
:10C890008C0D823328F480918E0D8C3208F0FCC010
:10C8A00080918C0D8F3308F016C180918E0D8833E6
:10C8B00008F411C110928F0D8EE38093900D0E94A9
:10C8C000D39409C14CE02FCD42E12DCD02E022E00E
:10C8D00041E16DE088E59DE00E94A09C6CCD4CE0BC
:10C8E000D0CD42E1CECD02E022E042E168E588E52C
:10C8F0009DE00E94A09C0DCE07E028E04AE26AE29B
:10C9000088E59DE00E94A09C05E022E04CE262E305
:10C9100088E59DE00E94A09C6AE08AE20E946C93F8
:10C9200060915A0D70915B0D82E38093740D8BE2E0
:10C930008093750D24E73DE042E388E59DE00E9489
:10C94000DE9A1ECE6AE486E30E946C9322CE48E40F
:10C95000649FB0011124072E000C880B990B0E94D4
:10C960006AF22AE037ED43E25CE30E94C9F20E94DA
:10C97000E6F7262F02E042E367E388E59DE00E94A8
:10C98000A09C14CE44E68416910498F4AF92BF9212
:10C990003F932F9380E89CE09F938F931F930F9377
:10C9A0000E94FDF10FB6F894DEBF0FBECDBF95E03B
:10C9B00055CEAF92BF923F932F9388E79CE09F9311
:10C9C0008F931F930F930E94FDF10FB6F894DEBF73
:10C9D0000FBECDBF96E042CE98E040CE1092780DCB
:10C9E00083E080938F0D85E28093900DFF2029F0E6
:10C9F00083EB91E10E9406A307C08091B30E8111E1
:10CA0000F7CF8FE30E9416948BE080938F0D15E291
:10CA10001093900D82E399E00E9413A38BE2809320
:10CA20008F0D1093900DFF2029F081EB91E10E9472
:10CA300006A307C08091B40E8111F7CF8FE30E9447
:10CA4000169483E380938F0D15E21093900D8DE281
:10CA500099E00E9413A383E580938F0D1093900DAE
:10CA6000FF2029F08FEA91E10E9406A307C0809180
:10CA7000B50E8111F7CF8FE30E9416948BE580935A
:10CA80008F0D85E28093900D86E299E00E9413A3BA
:10CA900081E08093780DFBCE84E00E94C1A283E008
:10CAA00080938F0D12E31093900D86E00E94F2A206
:10CAB0000E94BDC58CE080938F0D1093900D8091E6
:10CAC0001602909117020E949C490E9413A385E2CE
:10CAD0000E941694E5CE2A960FB6F894DEBF0FBEDC
:10CAE000CDBFDF91CF911F910F91FF90BF90AF907D
:10CAF0009F908F907F906F905F904F900895282F18
:10CB00008091490A90914A0AA0914B0AB0914C0A2F
:10CB100081309048A105B10540F01092490A109269
:10CB20004A0A10924B0A10924C0A80917C09882381
:10CB300031F08091490A8093A60E1092460A8091A6
:10CB400071091816FCF4082E000C990B821B910930
:10CB50002091A60E022E000C330B2817390794F0F3
:10CB600097FF02C080E090E08093A60E092E000C93
:10CB7000AA0BBB0B8093490A90934A0AA0934B0AD5
:10CB8000B0934C0A8091A60E6623A9F09091720989
:10CB9000891714F48093720920917209022E000CF7
:10CBA000330B2C5F3F4F482F082E000C550B2417DA
:10CBB00035071CF484508093720908958091470AC8
:10CBC0008630D8F496E0899FF0011124EE5FF64F8D
:10CBD0002091280230912902318320834091490A13
:10CBE00050914A0A60914B0A70914C0A42835383D8
:10CBF000648375838F5F8093470A089580EA90E687
:10CC00000C941495E091470AEE2369F0E150E0930B
:10CC1000470A86E0E89FF0011124EE5FF64F80811D
:10CC200091810C941495EACF1092480AEBCFAF9201
:10CC3000BF92CF92DF92EF92FF920F931F93CF9309
:10CC4000DF935C017B0120E030E0F501E20FF31F90
:10CC5000E491EE2319F02F5F3F4FF7CFF701CF019B
:10CC60008E199F0941914111FACF04E110E0081B90
:10CC700011093327021713071CF0DD24D39402C0D7
:10CC800082E0D82E8091590D90E06D2D70E06F5F9D
:10CC90007F4F0E9475F9C62EC6E0C60F80918C0D9D
:10CCA000C81750F080918E0D90E02C2F30E02B5063
:10CCB0003109821793079CF5D0E0E114F104C1F12A
:10CCC0008AE30E94169482E0D8120FC0CC0D8091A6
:10CCD0008C0DC81768F120918E0D30E08C2F90E0FC
:10CCE0000B97281739071CF423C0DD2309F1802F87
:10CCF000880F080F000F00938F0DC093900D80E2F6
:10CD00000E941694C701DF91CF911F910F91FF9060
:10CD1000EF90DF90CF90BF90AF900C9413A3109240
:10CD20008F0DC093900DC5010E9406A3D1E0C5CF21
:10CD3000DF91CF911F910F91FF90EF90DF90CF90F7
:10CD4000BF90AF9008950F934CE0849F402D112425
:10CD500021E0240F2093E2068CE0840F8093E30609
:10CD6000E0918C0DF0E090E002968E179F070CF199
:10CD7000822F90E020918E0D30E082179307CCF443
:10CD8000662371F081E08093780D4D5F0BE020E821
:10CD900060E088E59DE00E94A09C1092780D03C0A1
:10CDA00081E08093780D8091E30610928F0D80933F
:10CDB000900D0F910895CF92DF92EF92FF920F9313
:10CDC000CF93DF93982F862F6A017901692FBBDFFC
:10CDD00090918C0D8091E306891708F453C09091CF
:10CDE0008E0D8091E206981708F44CC0002359F08C
:10CDF00060E070E0F701E60FF71FE491EE2351F0D9
:10CE00006F5F7F4FF7CFD701BD016E197F098D91FD
:10CE10008111FACFC62FD4E1D61BF6018491882365
:10CE200039F00E94DBA2D81BFFEFCF1ADF0AF5CF43
:10CE30008AE30E941694DD2329F080E20E94169472
:10CE4000D150F9CF8091E3066AEFC69F602D11247F
:10CE5000605860938F0D8093900DC701002349F0B7
:10CE6000DF91CF910F91FF90EF90DF90CF900C94D6
:10CE700006A3DF91CF910F91FF90EF90DF90CF90BD
:10CE80000C9413A3DF91CF910F91FF90EF90DF905F
:10CE9000CF9008950F93CF93DF93CDB7DEB7ED8595
:10CEA000FE8560817181828193810E94E1F7CB01CF
:10CEB0000E949C4900E09C0149855A8568858F81C4
:10CEC0007ADFDF91CF910F910895149A0895CF9250
:10CED000DF92EF92FF920F931F93CF93DF93C82FB0
:10CEE0000E94E07380918704882391F00E94CE9F76
:10CEF000009183041091840420918504309186046C
:10CF0000DC01CB01801B910BA20BB30BB7FF35C12A
:10CF10008091D206853010F40E943BC60E94CE9FBD
:10CF2000C0907A04D0907B04E0907C04F0907D0463
:10CF3000C114D104E104F10471F10091990410913C
:10CF40009A0420919B0430919C040C0D1D1D2E1DF4
:10CF50003F1D6B017C01C01AD10AE20AF30AF7FCFB
:10CF60001AC0E2EBFBE08491EF012196882321F0C7
:10CF70000E948384FE01F7CF6091F2037091F30366
:10CF80008FE894E10E941EA48AE00E94838486E8D0
:10CF900094E10E945CAF20919504211128C0C090BB
:10CFA0001102D0901202E0901302F0901402C1140A
:10CFB000D104E104F104D9F00091990410919A048C
:10CFC00020919B0430919C040C0D1D1D2E1D3F1DB6
:10CFD000DC01CB01801B910BA20BB30BB7FD07C08B
:10CFE000C11105C00E9451C5882309F4E5C00E9403
:10CFF000CE9F0091650910916609209167093091D3
:10D0000068096B017C01C01AD10AE20AF30AF7FC35
:10D010003AC08B019C010C53164F2F4F3F4F00938A
:10D020006509109366092093670930936809079B87
:10D03000CEC0069BCCC0059BCAC02091080421111C
:10D04000C6C0049BC4C0009161091091620920917F
:10D05000630930916409011511052105310509F4B1
:10D06000BFC0DC01CB01801B910BA20BB30B805620
:10D070009A4EA109B109B7FFB3C0749A6FEF70E07F
:10D0800082E00E94CF9E0E9451C5811105C0D091BF
:10D090009104C09193041AC0E091730A8FE48E9FAB
:10D0A000F0011124EB5CF04FD081E091730A8E9F68
:10D0B000F0011124E95CF04FC0818091730A9091D6
:10D0C000720A891719F08F5F8F70F9CFDD2329F16C
:10D0D0000E94CE9F0091690910916A0920916B0905
:10D0E00030916C09DC01CB010115110521053105D9
:10D0F00069F48C599F4FAF4FBF4F8093690990934C
:10D100006A09A0936B09B0936C09B0C0801B910BA6
:10D11000A20BB30BB7FFABC0A9C010926909109264
:10D120006A0910926B0910926C09CC2309F478C03B
:10D130000E94CE9F00916D0910916E0920916F0998
:10D1400030917009DC01CB01011511052105310574
:10D1500069F48C599F4FAF4FBF4F80936D099093E7
:10D160006E09A0936F09B09370093DC0801B910BAD
:10D17000A20BB30BB7FF38C036C00E94CE9F6B0125
:10D180007C012091870430E0A8EEB3E00E948DF688
:10D19000DC01CB018C0D9D1DAE1DBF1D8093830452
:10D1A00090938404A0938504B09386040E9482E344
:10D1B0008AE00E948384ACCE179A10921515169AB5
:10D1C00010921615159A109217157FDE10CF6093E6
:10D1D000610970936209809363099093640933CF66
:10D1E000749860E04CCFCFEFDD23D1F129EBD29FD3
:10D1F000C00111246FEF70E00E9475F96A5B7F4FE8
:10D2000088E00E94CF9ECC23C1F029EBC29FC001D1
:10D2100011246FEF70E00E9475F96A5B7F4F0FC0B9
:10D2200010926D0910926E0910926F091092700998
:10D2300060E070E088E00E94CF9E60E070E086E0F1
:10D240000E94CF9E0E9472E784E79AE0DF91CF911F
:10D250001F910F91FF90EF90DF90CF900C9410A250
:10D2600060E070E088E00E94CF9ECFCFDFEFC11179
:10D270005FCF10926D0910926E0910926F09109293
:10D280007009B4CF179AE5E1F5E11082169A118280
:10D29000159A12821ACECF92DF92EF92FF92CF931D
:10D2A000DF9320911002222309F443C0EC01C090C7
:10D2B0000402D0900502E0900602F0900702A70158
:10D2C0009601688179818A819B810E94C3F8181632
:10D2D00024F4C882D982EA82FB82C0900802D090EE
:10D2E0000902E0900A02F0900B02A70196016C81FE
:10D2F0007D818E819F810E94C3F8181624F4CC8210
:10D30000DD82EE82FF82C0900C02D0900D02E09090
:10D310000E02F0900F02A7019601688579858A8533
:10D320009B850E94C3F8181624F4C886D986EA861D
:10D33000FB86DF91CF91FF90EF90DF90CF90089523
:10D34000CF93DF930E947DA3E091D106F0E0E153FB
:10D35000FB4F8081882309F45EC0E3E8F4E1849107
:10D36000EF012196882321F00E948384FE01F7CFEC
:10D37000C091D10680E6C89FE0011124CF50DB4F59
:10D3800088818E3419F0E0E8F4E110C080E20E9458
:10D39000838489910E948384899190ED980F9A30BB
:10D3A000C8F38D32B9F38B32A9F3EDCF8491EF013D
:10D3B0002196882321F00E948384FE01F7CF80917B
:10D3C000720A9091730A891B8F706FE070E0681B7E
:10D3D0007109072E000C880B990B0E942591EDE72F
:10D3E000F4E18491EF012196882321F00E94838447
:10D3F000FE01F7CF8091D20665E070E0681B7109ED
:10D40000072E000C880B990B0E9425918AE0DF9172
:10D41000CF910C948384DF91CF910895CF93DF93C4
:10D420008FB7F8949091110A9093100A8FBFE4E798
:10D43000F4E18491EF012196882321F00E948384F6
:10D44000FE01F7CF8091E6069091E706A091E806ED
:10D45000B091E906BC01CD016F5F7F4F8F4F9F4FA9
:10D460000E9425918AE00E948384DF91CF9168CF4A
:10D47000EF92FF920F931F93CF93DF93C091D1064A
:10D4800080E6C89FE0011124CF50DB4F80919E04BD
:10D4900080FF19C0E5EDF6E184918F010F5F1F4F0A
:10D4A000811102C08E0104C00E948384F801F4CF70
:10D4B000D8018D918D01882319F00E948384F8CFC3
:10D4C0008AE00E94838410929804109297048FE35C
:10D4D0008093B6041092B5041092B40410925D09C2
:10D4E00010925E0910925F0910926009FE01888116
:10D4F00021968032D9F38E34B1F4818190ED980F6A
:10D500009A3020F08D3211F08B3269F43296DF01BF
:10D5100031962C9120532A30D0F3CD01FC01019695
:10D5200020812032D9F3F093F303E093F2038F01CB
:10D530000F5F1F4FC0816AE270E0C8010E94CCF902
:10D54000009731F0FC01319780818032E1F3118244
:10D55000CD3429F0C43519F0C73409F0E5C0F8011D
:10D5600080810F5F1F4F8032D1F380538A3008F0E3
:10D57000DBC0C093B6041092B5041092B4046AE004
:10D580008091B4049091B504689FA001699F500DEB
:10D5900011245093B5044093B4043196DF011197E0
:10D5A0008C91282F30E020533109240F351F309300
:10D5B000B5042093B404808180538A3008F3DF01DE
:10D5C00031968C918032D9F3CD34B9F42E313105B6
:10D5D00079F03CF42731310559F02C31310569F4EB
:10D5E00007C02537310521F0203AE3E03E0729F452
:10D5F000B0939804A093970497C010929804109247
:10D600009704D091F20361E070E0CD0101964C9156
:10D61000442309F489C0413299F4CD3489F420328D
:10D62000310571F4909398048093970463E270E05D
:10D630000E94CCF9009709F477C0DC011C9274C0F9
:10D6400041544A3108F043C0DC01FD015D91503284
:10D65000E1F3CF01A0EDA50FAA30C8F05E3229F4A6
:10D66000518150535A3098F067C05D3219F05B32E7
:10D6700009F062C05181A0EDA50FAA3048F05E32DA
:10D6800009F05AC0528150535A3010F055C0FC0175
:10D69000042F10E0D80153E0B595A7955A95E1F70E
:10D6A000A35AB64F47707B0102C0EE0CFF1C4A958F
:10D6B000E2F7A7015C91452B4C93309711F0ED1BDD
:10D6C00001C0E0E0D801AD5BB64FEC930AC04091D9
:10D6D000970450919804452B21F4B0939804A0939B
:10D6E0009704DC014C9141544A3110F4DC018DCF98
:10D6F000FC018E2FAF2F9191911103C0482F5A2F0B
:10D700000BC040ED490F4A30A0F343ED490F4230C2
:10D7100080F39B3271F3F2CFCA014F5F5F4FDC01A0
:10D72000EC91E032C9F3E2CFDF91CF911F910F91DD
:10D73000FF90EF900C94A725A0919704B0919804C6
:10D74000AB2B29F43197F0939804E0939704E0E031
:10D75000F0E09ECF0F931F93CF9383E50E946DC49B
:10D76000882309F447C00E94EBC3813039F082302E
:10D7700009F040C00CE313E0C0E021C00CE313E06B
:10D78000C0E0F80181918F010E946DC4882339F0B7
:10D790000E94EBC34FEF682F8C2F0E94AE4ACF5FE1
:10D7A000C43079F782E40E946DC4882319F10E9485
:10D7B000EBC34FEF682F1BC0CF5FC43079F0F80187
:10D7C00081918F010E946DC48823B1F30E94EBC345
:10D7D000482F6FEF8C2F0E94AE4AEECF82E40E945A
:10D7E0006DC4882339F00E94EBC3482F6FEF84E0AB
:10D7F0000E94AE4ACF911F910F910C94F6490F935E
:10D800001F93CF9383E50E943EC4811104C00CE3B3
:10D8100013E0C0E00EC0C0E00E94EBC3682F8C2F65
:10D820000E94584BCF5FC530B9F7F1CFCF5FC430FE
:10D8300071F0F80181918F010E943EC48823B1F3F9
:10D840000E94EBC3682F8C2F0E94584BEFCF82E4CD
:10D850000E943EC4882331F00E94EBC3682F84E00D
:10D860000E94584BCF911F910F910C94F649CF9382
:10D87000DF9383E50E946DC4882321F00E94DBC3FF
:10D88000EB0102C0C0E0D0E080E50E946DC48823B7
:10D8900021F00E94DBC3CB0102C080E090E0BE011A
:10D8A000DF91CF910C946F4B0F931F93CF930CE3A9
:10D8B00013E0C0E0F80181918F010E943EC48823EB
:10D8C00029F00E94DBC38C2F0E947E4BCF5FC430B7
:10D8D00089F782E40E943EC4882329F00E94DBC3BA
:10D8E00084E00E947E4B83E50E943EC4882349F079
:10D8F000C0E00E94DBC38C2F0E947E4BCF5FC530FF
:10D90000C1F7CF911F910F91089588E893E190930B
:10D91000BE048093BD0480916F008D7F80936F0063
:10D920000E9451C5882359F00E9451C58823C1F334
:10D930008091730A8F5F8F708093730AF1CF10927A
:10D94000BC041092BB0480916F00826080936F00D2
:10D950008FB7F8941092CB0E1092CC0E1092CD0E81
:10D960001092CE0E8FBF0E94E44B80E00E94C74B06
:10D9700060933709709338098093390990933A0975
:10D9800081E00E94C74B60933B0970933C098093F0
:10D990003D0990933E0982E00E94C74B60933F0986
:10D9A0007093400980934109909342098CE0E7E32A
:10D9B000F9E0A5EFB4E101900D928A95E1F70C949E
:10D9C00052C3EF92FF920F931F93CF938CE3E82EF5
:10D9D00083E0F82E0AEF13E0C0E0F70181917F01A8
:10D9E0000E943EC4882351F00E940BC4F80160835A
:10D9F0007183828393838C2F0E9497C2CF5F0C5FC9
:10DA00001F4FC33051F7CF911F910F91FF90EF90AF
:10DA10000C94505983E50E943EC48823D9F00E949B
:10DA20000BC4AB01BC014093691450936A1460931A
:10DA30006B1470936C144093611450936214609350
:10DA40006314709364148CE494E10E94C1A38AE08F
:10DA50000E94838480E50E943EC4882399F00E943E
:10DA60000BC4AB01BC014093691450936A146093DA
:10DA70006B1470936C148FE294E10E94C1A38AE04E
:10DA80000E94838482E50E943EC4882399F00E940C
:10DA90000BC4AB01BC0140936514509366146093B2
:10DAA00067147093681480E194E10E94C1A38AE036
:10DAB0000E94838484E50E943EC4882399F00E94DA
:10DAC0000BC4AB01BC01409361145093621460938A
:10DAD00063147093641482EF93E10E94C1A38AE0FF
:10DAE0000C9483840895FF920F931F93CF93DF9339
:10DAF0000AE514E0CCE3D3E0FC2E84E0F80E899133
:10DB00000E943EC4882339F00E940BC4F801608350
:10DB10007183828393830C5F1F4FFC12F0CFDF91E0
:10DB2000CF911F910F91FF900895FF920F931F9334
:10DB3000CF93DF930DE614E1CCE3D3E0FC2E84E039
:10DB4000F80E89910E943EC4882349F00E940BC4BC
:10DB50000E94E6F7F80160837183828393830C5FF0
:10DB60001F4FFC12EECFDF91CF911F910F91FF90CD
:10DB70000C94DFBECF9388EC90E00E940BC581111E
:10DB800040C084E40E943EC48823C1F10E940BC4BB
:10DB9000C1E020E030E0A9010E9464F2811101C0DF
:10DBA000C0E0C0938114CC2349F10E940BC4E091E2
:10DBB000820424E0E29FF0011124E358FB4E6083CD
:10DBC00071838283938320E030E0A90160917D140A
:10DBD00070917E1480917F14909180140E9464F261
:10DBE00081110CC080E090E0A0E4B0E480937D144B
:10DBF00090937E14A0937F14B0938014CF910C94D3
:10DC00001E84CF910895CF92DF92EF92FF920F93EF
:10DC10001F93CF93DF9300D01F92CDB7DEB78091D3
:10DC2000490A90914A0AA0914B0AB0914C0AB7FF59
:10DC300008C01092490A10924A0A10924B0A109298
:10DC40004C0A8091D3069091D406A091D506B0914C
:10DC5000D6064091490A50914A0A60914B0A709148
:10DC60004C0A84179507A607B70744F48093490A1E
:10DC700090934A0AA0934B0AB0934C0A80912A02CF
:10DC8000882379F14091490A50914A0A60914B0AE0
:10DC900070914C0A8091D7069091D806A091D90630
:10DCA000B091DA066A017B01C80ED91EEA1EFB1E7E
:10DCB000C701B6010E946AF22AE037ED43E25CE355
:10DCC0000E94C9F269837A838B839C83CE0101967B
:10DCD0000E941547BC018091DD069091DE060E94EE
:10DCE000176680918D091091DF06811106C01123FE
:10DCF000D1F180912A028823B1F14091490A5091D3
:10DD00004A0A60914B0A70914C0A8091D706909113
:10DD1000D806A091D906B091DA066A017B01C80E37
:10DD2000D91EEA1EFB1EC701B6010E946AF22AE054
:10DD300037ED43E25CE30E94C9F2E091DB06F0912B
:10DD4000DC06309721F060837183828393831123F3
:10DD500029F0E091E006F091E106199580918D0996
:10DD600081110E94026680918D09882329F0E0913B
:10DD7000E006F091E10619950F900F900F900F902B
:10DD8000DF91CF911F910F91FF90EF90DF90CF9097
:10DD90000895CF92DF92EF92FF920F931F93CF934C
:10DDA000DF9300D01F92CDB7DEB78091490A9091E2
:10DDB0004A0AA0914B0AB0914C0AB7FF08C01092D2
:10DDC000490A10924A0A10924B0A10924C0A80910A
:10DDD000D3069091D406A091D506B091D606409175
:10DDE000490A50914A0A60914B0A70914C0A841773
:10DDF0009507A607B70744F48093490A90934A0A07
:10DE0000A0934B0AB0934C0A80912A02882379F19F
:10DE10004091490A50914A0A60914B0A70914C0A0C
:10DE20008091D7069091D806A091D906B091DA06D4
:10DE30006A017B01C80ED91EEA1EFB1EC701B6018E
:10DE40000E946AF22AE037ED43E25CE30E94C9F2E5
:10DE500069837A838B839C83CE0101960E94CA4793
:10DE6000BC018091DD069091DE060E9417668091CC
:10DE70008D091091DF06811106C01123D1F1809127
:10DE80002A028823B1F14091490A50914A0A6091CF
:10DE90004B0A70914C0A8091D7069091D806A091B8
:10DEA000D906B091DA066A017B01C80ED91EEA1EB6
:10DEB000FB1EC701B6010E946AF22AE037ED43E279
:10DEC0005CE30E94C9F2E091DB06F091DC0630973A
:10DED00021F06083718382839383112329F0E09181
:10DEE000E006F091E106199580918D0981110E945B
:10DEF00002660F900F900F900F90DF91CF911F91BE
:10DF00000F91FF90EF90DF90CF900895CF92DF9226
:10DF1000EF92FF920F931F93CF93DF9300D01F9246
:10DF2000CDB7DEB78091490A90914A0AA0914B0A79
:10DF3000B0914C0AB7FF08C01092490A10924A0AE1
:10DF400010924B0A10924C0A8091D3069091D406FD
:10DF5000A091D506B091D6064091490A50914A0A3F
:10DF600060914B0A70914C0A84179507A607B70772
:10DF700044F48093490A90934A0AA0934B0AB093C1
:10DF80004C0A80912A02882379F14091490A5091E4
:10DF90004A0A60914B0A70914C0A8091D706909181
:10DFA000D806A091D906B091DA066A017B01C80EA5
:10DFB000D91EEA1EFB1EC701B6010E946AF220E0CC
:10DFC00030E048EC52E40E94C9F269837A838B8383
:10DFD0009C83CE0101960E944B48BC018091DD06D6
:10DFE0009091DE060E94176680918D091091DF06E0
:10DFF000811106C01123D1F180912A028823B1F149
:10E000004091490A50914A0A60914B0A70914C0A1A
:10E010008091D7069091D806A091D906B091DA06E2
:10E020006A017B01C80ED91EEA1EFB1EC701B6019C
:10E030000E946AF220E030E048EC52E40E94C9F20B
:10E04000E091DB06F091DC06309721F0608371836C
:10E0500082839383112329F0E091E006F091E10699
:10E06000199580918D0981110E9402660F900F9081
:10E070000F900F90DF91CF911F910F91FF90EF9034
:10E08000DF90CF900895CF92DF92EF92FF920F939F
:10E090001F93CF93DF9300D01F92CDB7DEB780914F
:10E0A000490A90914A0AA0914B0AB0914C0AB7FFD5
:10E0B00008C01092490A10924A0A10924B0A109214
:10E0C0004C0A8091D3069091D406A091D506B091C8
:10E0D000D6064091490A50914A0A60914B0A7091C4
:10E0E0004C0A84179507A607B70744F48093490A9A
:10E0F00090934A0AA0934B0AB0934C0A80912A024B
:10E10000882379F14091490A50914A0A60914B0A5B
:10E1100070914C0A8091D7069091D806A091D906AB
:10E12000B091DA066A017B01C80ED91EEA1EFB1EF9
:10E13000C701B6010E9468F220E030E048EC52E4EA
:10E140000E94C9F269837A838B839C83CE010196F6
:10E150000E944B48BC018091DD069091DE060E9432
:10E16000176680918D091091DF06811106C0112379
:10E17000E1F180912A028823C1F14091490A50912E
:10E180004A0A60914B0A70914C0A8091D70690918F
:10E19000D806A091D906B091DA066A017B01C80EB3
:10E1A000D91EEA1EFB1EC701B6010E9468F220E0DC
:10E1B00030E048EC52E40E94C9F20E94E6F7E09198
:10E1C000DB06F091DC06309721F060837183828357
:10E1D0009383112329F0E091E006F091E10619956F
:10E1E00080918D0981110E94026680918D0988239A
:10E1F00029F0E091E006F091E10619950F900F905B
:10E200000F900F90DF91CF911F910F91FF90EF90A2
:10E21000DF90CF9008950F931F93CF938091490A79
:10E2200090914A0AA0914B0AB0914C0AB7FF08C0DE
:10E230001092490A10924A0A10924B0A10924C0A04
:10E240008091D3069091D406A091D506B091D606C0
:10E250004091490A50914A0A60914B0A70914C0AC8
:10E2600084179507A607B70744F48093490A90934B
:10E270004A0AA0934B0AB0934C0A80912A02882341
:10E2800031F14091490A50914A0A60914B0A7091CC
:10E290004C0A8091D7069091D806A091D906B091EA
:10E2A000DA068A019B01080F191F2A1F3B1FC901AB
:10E2B000B8010E946AF20E94E1F7CB010E949C49DA
:10E2C000BC018091DD069091DE060E941766809168
:10E2D0008D09C091DF06811106C0CC23A1F1809188
:10E2E0002A02882381F14091490A50914A0A60919B
:10E2F0004B0A70914C0A8091D7069091D806A09154
:10E30000D906B091DA068A019B01080F191F2A1F4E
:10E310003B1FC901B8010E946AF2E091DB06F0914F
:10E32000DC06309721F06083718382839383CC2352
:10E3300029F0E091E006F091E106199580918D09B0
:10E3400081110E94026680918D09CF911F910F91DA
:10E35000089561CF60DF882329F0E091E006F09115
:10E36000E106199408958091490A90914A0AA09172
:10E370004B0AB0914C0AB7FF08C01092490A10929C
:10E380004A0A10924B0A10924C0A8091D30690913F
:10E39000D406A091D506B091D6064091490A509175
:10E3A0004A0A60914B0A70914C0A84179507A60798
:10E3B000B70744F48093490A90934A0AA0934B0A02
:10E3C000B0934C0A80912A02882399F02091D706B5
:10E3D0003091D8068091490A90914A0A820F931F82
:10E3E0000E949C49BC018091DD069091DE060E944E
:10E3F000176680918D092091DF06811106C02223C6
:10E4000011F180912A028823F1F04091D7065091B2
:10E41000D8068091490A90914A0A840F951FE0918D
:10E42000DB06F091DC06309711F091838083222384
:10E4300029F0E091E006F091E106199580918D09AF
:10E4400081110E94026680918D0908958CCF8BDF27
:10E45000882329F0E091E006F091E10619940895EF
:10E46000CF93DF9360E085E00E947F65D0917209D1
:10E47000C0E0D11109C080912A028823E9F021E08F
:10E4800041E066EC75E115C0D13049F480912A0273
:10E49000882391F020E041E067EB75E10AC0D230BB
:10E4A00059F480912A02882339F020E041E06DEA96
:10E4B00075E18C2F0E94CC57CF5FDF5FC530C9F666
:10E4C00083E080937109DF91CF9108951F93CF93DB
:10E4D000DF9360E085E00E947F65D0917209C0E023
:10E4E00012E0D11109C080912A028823D9F121E0DC
:10E4F00041E060EA75E115C0D13049F480912A020B
:10E50000882381F120E041E067E975E10AC0D2305B
:10E5100061F480912A02882329F120E041E066E835
:10E5200075E18C2F0E94CC571DC0D33049F48091E7
:10E530002A028823B9F020E041E064E875E1F1CFD8
:10E54000D43081F480912A02882351F021E040E008
:10E5500069E775E18C2F0E94CC578C2F0E941EA377
:10E5600010932A02CF5FDF5FC53009F0BACFC093A6
:10E570007109DF91CF911F9108951F93CF93DF937E
:10E5800060E085E00E947F65D0917209C0E012E0F2
:10E59000D11109C080912A028823D9F121E041E0FC
:10E5A0006CE675E115C0D13049F480912A028823C8
:10E5B00081F120E041E063E675E10AC0D23061F408
:10E5C00080912A02882329F120E041E065E575E188
:10E5D0008C2F0E94CC571DC0D33049F480912A0261
:10E5E0008823B9F020E041E063E575E1F1CFD43054
:10E5F00081F480912A02882351F021E040E068E410
:10E6000075E18C2F0E94CC578C2F0E941EA3109373
:10E610002A02CF5FDF5FC53009F0BACFC09371091E
:10E62000DF91CF911F9108951F93CF93DF9360E007
:10E6300085E00E947F65D0917209C0E012E0D1119F
:10E6400009C080912A028823D9F121E041E06BE3DF
:10E6500075E115C0D13049F480912A02882381F1F7
:10E6600020E041E06BE275E10AC0D23061F48091B4
:10E670002A02882329F120E041E06AE175E18C2F2C
:10E680000E94CC571DC0D33049F480912A028823C0
:10E69000B9F020E041E06BE075E1F1CFD43081F4D6
:10E6A00080912A02882351F021E040E060E075E18A
:10E6B0008C2F0E94CC578C2F0E941EA310932A02ED
:10E6C000CF5FDF5FC53009F0BACFC0937109DF912A
:10E6D000CF911F9108951F93CF93DF9360E085E062
:10E6E0000E947F65D0917209C0E012E0D11109C08B
:10E6F00080912A028823D9F121E041E063EF74E19F
:10E7000015C0D13049F480912A02882381F120E09C
:10E7100041E063EE74E10AC0D23061F480912A02D4
:10E72000882329F120E041E066ED74E18C2F0E94FE
:10E73000CC571DC0D33049F480912A028823B9F008
:10E7400020E041E064ED74E1F1CFD43081F48091B8
:10E750002A02882351F021E040E069EC74E18C2F1B
:10E760000E94CC578C2F0E941EA310932A02CF5FC9
:10E77000DF5FC53009F0BACFC0937109DF91CF9147
:10E780001F910895EBE2F2E080E09191911104C0B5
:10E79000982F981B50E206C0863111F08F5FF5CF9D
:10E7A00096E1F7CF282F30E0492F480FF901E55DBA
:10E7B000FD4F463118F450838F5FF4CF10820895D7
:10E7C0004F925F926F927F928F929F92AF92BF9281
:10E7D000CF92DF92EF92FF920F931F93CF93DF932D
:10E7E00000D01F92CDB7DEB7109127021F3F01F175
:10E7F0000E94CE9FC0907809D0907909E0907A0964
:10E80000F0907B09DC01CB018C199D09AE09BF0991
:10E81000B7FD0EC02091730A8091720A30E08F5FBD
:10E820008F70082E000C990B2817390709F029C2A0
:10E830000E94C5C58091E51382FF39C080918E0981
:10E84000811137C081E080938E09909196048927C9
:10E8500080938D091092960483E080932A0210928F
:10E86000E5130E94CE9FDC01CB018C509E4FAF4F31
:10E87000BF4F8093E6139093E713A093E813B093F0
:10E88000E91348E853E162E070E080E090E00E9424
:10E8900074EB16E0115069F084E79AE00E9410A230
:10E8A00062E070E080E090E00E94969FF3CF1092CB
:10E8B0008E0919B11295117081E0182780918C0989
:10E8C000412F50E0282F30E042175307A9F01123C1
:10E8D00009F4FDC10E94125680918C09823029F002
:10E8E00060E080EE95E10E941CC610938C0983E0E5
:10E8F00080932A020E945CA20E94CE9F6B017C0141
:10E900008091880990918909A0918A09B0918B0919
:10E91000A7019601281B390B4A0B5B0B57FF05C05B
:10E920008091450A882309F425C2D701C6018C5974
:10E930009F4FAF4FBF4F8093880990938909A09351
:10E940008A09B0938B098091E31318162CF48091F7
:10E95000E313823074F408C08091E3139927819502
:10E960000CF4909502972CF480918D0981119BC035
:10E97000ABC080918709882309F46EC08091E313AE
:10E98000181654F48091E313082E000C990B97FD90
:10E990000196959587950CC08091E313082E000C85
:10E9A000990B97FD0196959587959195819591097C
:10E9B0008090830990908409A0908509B090860981
:10E9C00081149104A104B104D1F1BC01990F880B09
:10E9D000990B0E946AF22B013C01C701B60168192C
:10E9E00079098A099B090E9468F29B01AC01C30165
:10E9F000B2010E9479F720E030E04AE754E40E9437
:10EA0000C9F24B015C0120E030E040E253E40E9497
:10EA1000C3F887FF0FC020E030E046E952E4C501AB
:10EA2000B4010E94C3F887FD0AC02AE030E040E04C
:10EA300050E009C024E630E040E050E004C021E0AE
:10EA400030E040E050E0C0928309D0928409E09227
:10EA50008509F092860904C021E030E040E050E0F2
:10EA6000A091E3130A2E000CBB0B0E9487F622E054
:10EA700030E040E050E00E9461F68091490A9091B8
:10EA80004A0AA0914B0AB0914C0A820F931FA41F0F
:10EA9000B51F8093490A90934A0AA0934B0AB093FA
:10EAA0004C0A1092E313D701C6018856954CAF4F1C
:10EAB000BF4F80937F0990938009A0938109B09301
:10EAC000820981E080932A02209128023091290254
:10EAD00040E6203A340741F480919702882309F4F4
:10EAE00001C1815080939702255C374A71F480916F
:10EAF000181590911915891740F490919702992350
:10EB000009F400C19150909397022FB7F894809127
:10EB1000CB0E9091CC0EA091CD0EB091CE0E2FBF0A
:10EB20003AE0B695A795979587953A95D1F70097CE
:10EB300021E0A207B10520F08FEF9FEFA0E0B0E049
:10EB40009695879520912A02211105C03091450A9A
:10EB500031110CC159C0009741F040917D0950918D
:10EB60007E094817590708F04FC08091450A811166
:10EB700013C0223050F0243028F0243031F41092A9
:10EB80002A0203C081E080932A020E94E29481E07D
:10EB900080937C098093450A84E00E94C1A281E0B1
:10EBA0008093780DE0912802F09129021995109236
:10EBB0008D0910927C098091450A882351F00E94AA
:10EBC000E09291E0811101C090E09093450A91118B
:10EBD000B1C080907D0990907E09A12CB12C0E943B
:10EBE000CE9FDC01CB018C199D09AE09BF098816A7
:10EBF0009906AA06BB0640F40E94CE9F6C197D09B7
:10EC000070937E0960937D0980912802909129027A
:10EC1000805A904621F08091480A882379F048E98B
:10EC2000C40E4AE3D41EE11CF11CC0927F09D092AD
:10EC30008009E0928109F09282090FC080917F09DA
:10EC400090918009A0918109B0918209C81AD90ACE
:10EC5000EA0AFB0AF7FE0E94FE658091450A8111CF
:10EC600089C080912A02813049F008F483C0843041
:10EC700008F080C081E080932A027CC010922A02B2
:10EC800079C054E01502F0011124E159FC4F20E055
:10EC900030E040E752E460817181828193810E947B
:10ECA00079F769837A838B839C83E12C8E010F5FD4
:10ECB0001F4F21E035E14DEF54E169EF74E185EF3D
:10ECC00094E10E9436C08FEF80932702B1CD10925D
:10ECD000A10A1092A20A823009F407CE60E083ED07
:10ECE00095E101CE8CE08093970280917D0990910F
:10ECF0007E09019790937E0980937D0981E080933E
:10ED00002A02F2CE96E09093970291E090932A0225
:10ED10008F5F80931815D701C6018856954CAF4F69
:10ED2000BF4F80937F0990938009A0938109B0938E
:10ED30008209EBCE80907D0990907E09A12CB12CA8
:10ED40000E94CE9FDC01CB018C199D09AE09BF0941
:10ED500088169906AA06BB0668F40E94CE9F6C1915
:10ED60007D0970937E0960937D0904C0009709F4C2
:10ED700013CFF3CE0F900F900F900F90DF91CF91A4
:10ED80001F910F91FF90EF90DF90CF90BF90AF90C9
:10ED90009F908F907F906F905F904F900895CF924B
:10EDA000DF92EF92FF920F931F930E94CE9F0091EC
:10EDB00074091091750920917609309177096B01DA
:10EDC0007C01C01AD10AE20AF30AF7FC13C02091B1
:10EDD0007309209520937309DC01CB018A549C4F61
:10EDE000AF4FBF4F8093740990937509A093760934
:10EDF000B093770981E090917309911101C080E08F
:10EE00001F910F91FF90EF90DF90CF9008950E9497
:10EE10005CA2A4E0B1E08C918F7D8C939FB7F894B5
:10EE2000E5E0F1E08081806280839FBF8C918F7BE1
:10EE30008C939FB7F8948081806480839FBF6A9889
:10EE4000729A54985C9A82E080938C090E94C5C59E
:10EE50001092E3130895CF93DF931F921F92CDB7C3
:10EE6000DEB789839A830E94DE6589819A810F903B
:10EE70000F90DF91CF910C9414956F927F928F92A7
:10EE80009F92AF92BF92CF92DF92EF92FF920F9339
:10EE90001F93CF93DF9300D01F92CDB7DEB76C01E5
:10EEA0003B014701580129833A834B835C830E94CD
:10EEB000DE6583E080932A02D092DE06C092DD06F2
:10EEC0007092DC066092DB0629813A814B815C817D
:10EED000CA01B9010E94E1F76093D7067093D80682
:10EEE0008093D9069093DA060E946AF26B017C0146
:10EEF0009B01AC01C501B4010E949CF60E94E1F7A0
:10EF00006093D3067093D4068093D5069093D6066B
:10EF1000A7019601F30160817181828193810E9432
:10EF20009CF60E94E6F76093490A70934A0A809320
:10EF30004B0A90934C0A89EA91E7909329028093B7
:10EF400028020F900F900F900F90DF91CF911F919B
:10EF50000F91FF90EF90DF90CF90BF90AF909F9078
:10EF60008F907F906F900895CF92DF92EF92FF92F3
:10EF70000F931F93CF93DF938C01EB016A0179010B
:10EF80000E94DE6523E020932A021093DE060093A0
:10EF9000DD06D093DC06C093DB06A601DD0C660B14
:10EFA000770B4093D7065093D8066093D906709399
:10EFB000DA06C701FF0CAA0BBB0B841B950BA60B33
:10EFC000B70B8093D3069093D406A093D506B09345
:10EFD000D60688819981092E000CAA0BBB0B841BD5
:10EFE000950BA60BB70B8093490A90934A0AA093FE
:10EFF0004B0AB0934C0A86E292E7909329028093E1
:10F000002802DF91CF911F910F91FF90EF90DF9039
:10F01000CF9008953F924F925F926F927F928F921E
:10F020009F92AF92BF92CF92DF92EF92FF920F9397
:10F030001F93CF93DF93CDB7DEB72C970FB6F8941D
:10F04000DEBF0FBECDBF5C01DC0159968D909C9058
:10F050005A97F40181859285A385B4859C01AD0101
:10F060002F5F3F4F4F4F5F4F29873A874B875C8712
:10F07000D5011496CD90DD90ED90FC901797C114BA
:10F08000D104E104F10439F0BFEFCB1ADB0AEB0A3B
:10F09000FB0A312C07C0F401C080D180E280F380EC
:10F0A00033243394260137011D821E821F82188665
:10F0B000F40181859285A385B4852D813E814F81A0
:10F0C0005885281739074A075B0708F064C0898507
:10F0D0009A85AB85BC858C159D05AE05BF0550F4A2
:10F0E00082E0C82ED12CE12CF12C92E0492E512C3B
:10F0F000612C712C9E012F5F3F4FB701A601C40107
:10F100000E94E6C9882309F446C089819A81AB81AF
:10F11000BC81892B8A2B8B2B41F0260137019FEF75
:10F12000491A590A690A790A05C0C414D504E604C3
:10F13000F70491F02D813E814F8158852F5F3F4F1D
:10F140004F4F5F4F2D833E834F8358873FEFC31A46
:10F15000D30AE30AF30AACCF0FEF1FEF2FEF3FE024
:10F16000B301A201C4010E9455C9F82E882399F069
:10F17000D50114964D915D916D917C911797411534
:10F1800051056105710549F093018201C4010E9496
:10F1900055C9811102C0F12C29C0D50114964D9298
:10F1A0005D926D927C921797332051F0D301C2018A
:10F1B0000196A11DB11DF40180839183A283B383C5
:10F1C000F50185899689A789B08D892B8A2B8B2B90
:10F1D00069F4D50155964D925D926D927C92589747
:10F1E00011968C911197806811968C938F2D2C9687
:10F1F0000FB6F894DEBF0FBECDBFDF91CF911F9148
:10F200000F91FF90EF90DF90CF90BF90AF909F90C5
:10F210008F907F906F905F904F903F9008951F92D6
:10F220000F920FB60F9211240BB60F922F933F93AC
:10F230004F935F936F937F938F939F93AF93BF93FE
:10F24000EF93FF93E091100A81E08E0F8F779091FA
:10F25000C6002091110A821731F0F0E0E057F64F16
:10F2600090838093100A20918F09422F50E04C30F8
:10F27000510508F046C0FA018827EE58FF4F8F4F1E
:10F280000C9488F99D3441F09E34B9F481E005C0B6
:10F290009A3330F09D3471F582E080938F0946C037
:10F2A000903308F043C0903209F440C09D3211F50C
:10F2B0003DC0913329F0943329F09032D9F436C00F
:10F2C00083E0EBCF88E0E9CF903321F0913391F4E4
:10F2D00086E0E3CF84E0E1CF983361F485E0DDCFD1
:10F2E000923341F487E0D9CF913321F489E0D5CF2F
:10F2F000903311F08BE0D1CF8AE0CFCF9A30B1F4C8
:10F3000013C09A3099F4273049F02A3059F025304B
:10F3100059F4109215021092960406C08EE796E1F9
:10F320000E945CAF0E94856C10928F09FF91EF9153
:10F33000BF91AF919F918F917F916F915F914F910D
:10F340003F912F910F900BBE0F900FBE0F901F900B
:10F3500018951F920F920FB60F9211240BB60F92B1
:10F360008F939F93EF93FF938091330AE82FF0E000
:10F37000EE5EF54F90818F5F8F718093330A90938B
:10F38000C6008091C00080648093C0009091320AD2
:10F390008091330A981305C08091C1008F7D8093BE
:10F3A000C100FF91EF919F918F910F900BBE0F9035
:10F3B0000FBE0F901F9018958F929F92AF92BF92A1
:10F3C000CF92DF92EF92FF920F931F93CF93DF9331
:10F3D000EC018B81811102C080E077C009891A8914
:10F3E0002B893C890417150726073707A8F36A01FC
:10F3F0007B01823029F4C886D986EA86FB860DC057
:10F40000C114D104E104F10451F4188619861A8656
:10F410001B861C821D821E821F8281E056C088844A
:10F420009984AA84BB84E98DFA8D258530E0275F15
:10F430003F4FB501A4014150510961097109022EE4
:10F4400004C076956795579547950A94D2F7D701EA
:10F45000C6010197A109B10904C0B695A795979572
:10F4600087952A95D2F784179507A607B70720F046
:10F4700089288A288B2849F44D895E896F89788D7F
:10F480004C835D836E837F8304C0841B950BA60B26
:10F49000B70B4C015D018E010C5F1F4F811491046D
:10F4A000A104B10409F4A7CF4C815D816E817F81F5
:10F4B0009801898D9A8D0E94E6C991E0891A910878
:10F4C000A108B1088111EACF87CFDF91CF911F91B9
:10F4D0000F91FF90EF90DF90CF90BF90AF909F90F3
:10F4E0008F9008952F923F924F925F926F927F92EA
:10F4F0008F929F92AF92BF92CF92DF92EF92FF9244
:10F500000F931F93CF93DF9300D01F92CDB7DEB739
:10F510009C838B834B015A01DC0113968C918111E2
:10F5200003C08FEF9FEFEBC0EB81FC81818180FFF7
:10F53000F8CFAB81BC8151960D911D912D913C91DD
:10F54000549718964D915D916D917C911B97C501D3
:10F55000A0E0B0E068017901C41AD50AE60AF70A0A
:10F56000C816D906EA06FB0618F45801A41AB50A0B
:10F5700075018B819C8104969A838983612C92E02A
:10F58000792EE114F10409F48BC0AB81BC8118968B
:10F590004D915D916D917C911B976A01B1E0DB22E9
:10F5A000EB81FC8123811A012B0189E05694479459
:10F5B000379427948A95D1F7818D928D223061F40A
:10F5C000FC01828D938DA48DB58DBC01CD01620DA2
:10F5D000731D841D951D4AC0DC0114961C911150A9
:10F5E0001221C114D10401F511111EC0452B462B67
:10F5F000472B59F4EB81FC8185899689A789B08DC9
:10F6000084839583A683B7830FC0AB81BC81149696
:10F610004D915D916D917C91179729813A810E945E
:10F62000E6C9882309F47DCFEB81FC81218D328DE1
:10F6300084819581A681B7810297A109B109F90159
:10F64000058404C0880F991FAA1FBB1F0A94D2F714
:10F650004685578560897189840F951FA61FB71F3E
:10F66000BC01CD01610F711D811D911D93012C19EC
:10F670003D0987012E153F0508F489010115F2E0C7
:10F680001F0779F52091EA083091EB084091EC08CA
:10F690005091ED08621773078407950719F421C08C
:10F6A000C5012DC09401AB01BC018091F30890917C
:10F6B000F4080E94BA46882309F433CF800E911EC5
:10F6C000EB81FC8180859185A285B385800F911F98
:10F6D000A11DB11D80879187A287B387E01AF10A27
:10F6E00050CF40E00E941DC9882309F41ACFB6010B
:10F6F0006651794FA801C4010E94A5F9DFCF0F9090
:10F700000F900F900F90DF91CF911F910F91FF906D
:10F71000EF90DF90CF90BF90AF909F908F907F90B1
:10F720006F905F904F903F902F900895DF92EF92EF
:10F73000FF920F931F93CF93DF937C01EB018A011C
:10F740008DE0D82E40E250E0BE01C701CBDE803212
:10F75000910539F021E0892B09F420E0822F819571
:10F760003EC02881222399F1253E61F32E3251F3C8
:10F770000115110541F13B853F733F3021F54A8D5D
:10F780005B8D452B01F52F713FEF320F3530D8F4EB
:10F7900030E021503109D29EC001D39E900D11243A
:10F7A000D801A80FB91FFE0120E0AD01253088F473
:10F7B00031813D932F5F32962D30C1F7288126FF8E
:10F7C00002C0FA0115862B8523FDBCCF08C080E05E
:10F7D00006C02B3010F43481ECCF3681EACFDF91B4
:10F7E000CF911F910F91FF90EF90DF9008950F93AD
:10F7F0001F93CF93DF93FC012381222311F080E03C
:10F8000044C08B01EC01FB018789803139F18032E2
:10F81000B1F783E08B83F801428D538D648D758D34
:10F820004D8B5E8B6F8B788F9E012F5E3F4FC80193
:10F830000E9466CA882319F31A8F098F81E0898391
:10F84000188619861A861B861C821D821E821F82BC
:10F85000188A1C861D861E861F8617C082E08B8331
:10F860001D8A1E8A1F8A188EFB01808D918DA0E053
:10F87000B0E025E0880F991FAA1FBB1F2A95D1F77A
:10F88000898B9A8BAB8BBC8BD7CFDF91CF911F919C
:10F890000F910895CF93DF93EC0141E0611101C016
:10F8A00040E06C857D858E859F850E941DC98823DB
:10F8B00041F0888920E2829FC00111248651994F2E
:10F8C00002C080E090E0DF91CF910895CF93DF9365
:10F8D000EC018B81882331F1898187FF1FC061E0B2
:10F8E000CE01D8DFFC01892BE9F08081853ED1F083
:10F8F0008B81823040F489899A89AB89BC89848F55
:10F90000958FA68FB78F8D899E89AF89B88D938F7C
:10F91000828FB58BA48B89818F778983DF91CF917B
:10F920000C94DDC881E0888380E0DF91CF91089559
:10F930002F923F924F925F926F927F928F929F92FF
:10F94000AF92BF92CF92DF92EF92FF920F931F93ED
:10F95000CF93DF9300D01F92CDB7DEB78C014B0160
:10F960001A01DC0113968C9113978130C1F4119622
:10F970008C9181FF14C082FF18C0F801418952891F
:10F980006389748980859185A285B38584179507DD
:10F99000A607B70751F0C8010FDD811106C081E04D
:10F9A000F80180838FEF9FEF2EC1610185C0D801E0
:10F9B00059968D919C915A97FC01248121502A01DE
:10F9C0003B0139E076946794579447943A95D1F780
:10F9D000722E74207A01F1E0FF22772009F478C0BA
:10F9E00080E092E08E199F0956018C159D0508F460
:10F9F0005C01D80159962D913C915A9714968D919E
:10FA00009D910D90BC91A02D0297A109B109F9011A
:10FA1000058404C0880F991FAA1FBB1F0A94D2F740
:10FA20004685578560897189840F951FA61FB71F6A
:10FA30009C01AD01270D311D411D511D29013A01C8
:10FA4000A11432E0B30609F089C08091EA089091D0
:10FA5000EB08A091EC08B091ED0884159505A6057A
:10FA6000B70569F41092F2088FEF9FEFDC018093E5
:10FA7000EA089093EB08A093EC08B093ED0894018A
:10FA8000B301A2018091F3089091F4080E945846B6
:10FA9000882309F484CFF80180859185A285B385F8
:10FAA0008A0D9B1DA11DB11D80879187A287B387F9
:10FAB0008A0C9B1CCA18DB08D80118964D915D91E1
:10FAC0006D917C911B97C114D10409F070CF7CC05B
:10FAD000E114F10409F084CF14964D915D916D917C
:10FAE0007C911797411551056105710559F455969B
:10FAF0008D919D910D90BC91A02D0097A105B10510
:10FB000039F521C09E012F5F3F4F0E94E6C988232F
:10FB100009F445CF89819A81AB81BC81F801218D9F
:10FB2000328DF9012789203139F4883FFFEF9F0793
:10FB3000A105B10540F40CC0883F2FEF9207A20742
:10FB40002FE0B20728F0C80165DA811149CF27CF2D
:10FB5000F80184839583A683B78342CFE114F1042F
:10FB600019F5D80118964D915D916D917C911B9777
:10FB700051968D919D910D90BC91A02D48175907DC
:10FB80006A077B0788F00E94DDC8882309F407CF45
:10FB900081E08093F2084092EA085092EB0860926C
:10FBA000EC087092ED0808C041E0C301B2010E9468
:10FBB0001DC9882309F4F3CEA501B401C7018651FC
:10FBC000994F0E94A5F967CF51968D919D910D9007
:10FBD000BC91A02D84179507A607B70740F4F8013C
:10FBE000418B528B638B748B818180688183D801B8
:10FBF00011968C9183FD02C0C10105C0C80166DE6B
:10FC00008111FACFCCCE0F900F900F900F90DF9113
:10FC1000CF911F910F91FF90EF90DF90CF90BF9009
:10FC2000AF909F908F907F906F905F904F903F909C
:10FC30002F900895CF93DF93EC0148DE1B82DF9174
:10FC4000CF9108954F925F926F927F92AF92BF9241
:10FC5000CF92DF92EF92FF920F931F93CF93DF9398
:10FC60001F92CDB7DEB78C017B015A01D22EDB018A
:10FC700059968D919C915A97F801928F818F40E00F
:10FC800050E0BA01C70198DBC12CF701808591854E
:10FC9000A285B38541895289638974898417950740
:10FCA000A607B70708F062C025E0B695A795979517
:10FCB00087952A95D1F7F82FFF707F2ED7011396DD
:10FCC0008C91823008F462C041E050E0BE016F5F69
:10FCD0007F4FC70107DC019719F4898190E002C0CA
:10FCE0008FEF9FEF019609F451C0F7018085918550
:10FCF000A285B3854F96A11DB11D80879187A287EC
:10FD0000B387F0E27F9EC0011124BC016651794F98
:10FD100061157105D9F1DB012C91222319F0253EE3
:10FD2000D1F466C1C1100EC04091EA085091EB08B1
:10FD30006091EC087091ED08F8014487558766875B
:10FD40007787708AFC01E651F94F8081882361F042
:10FD5000CC24C3949ACF4BE050E0C5010E9498F99F
:10FD6000892B09F092CF14C0CC24C3948D2D8274BA
:10FD7000823461F4CC2009F489C0D80150967C907B
:10FD800061E0C80187DD009709F006C180E033C15A
:10FD9000D7FCFCCFF0E27F9EA00111249A012651EE
:10FDA000394FD9011B968C91817121F08D2D827173
:10FDB00009F068C08091EA089091EB08A091EC08E6
:10FDC000B091ED08F80184879587A687B787708A78
:10FDD000FA01E651F94F4489558960E070E0BA01B3
:10FDE00055274427D80155964D935D936D937C9389
:10FDF0005897828D938DA0E0B0E0482B592B6A2B49
:10FE00007B2BD80155964D935D936D937C935897BA
:10FE1000D9011B968C91887159F4848D958DA68D8E
:10FE2000B78DF801818B928BA38BB48B81E010C0CE
:10FE3000803141F598012F5E3F4FD80159968D9141
:10FE40009C915A970E9466CA8823E1F084E0F801E9
:10FE500083838D2D8F70D80111968C931197F801A3
:10FE6000148215821682178218961D921D921D9279
:10FE70001C921B97D4FEB0C0C8010E944596811108
:10FE8000ABC084CFD80113961C9280CFF701838139
:10FE9000823009F47BCF81899289A389B489803E1D
:10FEA0009F4FAF41B10508F071CFC701B3D8882388
:10FEB00009F46CCF0E94DDC8882309F467CFD7010D
:10FEC00059962D913C915A9714968D919D910D9034
:10FED000BC91A02D0297A109B109F901058404C0C4
:10FEE000880F991FAA1FBB1F0A94D2F74684578414
:10FEF00060887188480E591E6A1E7B1E81E08093BF
:10FF0000F2084092EA085092EB086092EC08709276
:10FF1000ED0880E092E0EAEEF6E0DF019C011D9240
:10FF200021503040E1F7CC24C394D7015996ED918C
:10FF3000FC915A978481C81698F42AEE36E0B301F2
:10FF4000A2014C0D511D611D711D8091F30890910E
:10FF5000F4080E945846882309F418CFC394E5CFCB
:10FF600080E092E0A0E0B0E0058404C0880F991F13
:10FF7000AA1FBB1F0A94D2F7F701418952896389EE
:10FF80007489840F951FA61FB71F818B928BA38B3B
:10FF9000B48B8AEE96E0712C20E2DC011D922A954A
:10FFA000E9F72BE0F501DC0101900D922A95E1F7CC
:10FFB00021E238E2FC01318B208B40E058E057878A
:10FFC0004687338B228B318F208F578B468B0E9435
:10FFD000DDC88111DFCEDACED5FE08C0F801418937
:10FFE000528963897489C801E7D905C081E003C0DB
:10FFF000C110AECE99CE0F90DF91CF911F910F918E
:020000021000EC
:10000000FF90EF90DF90CF90BF90AF907F906F9078
:100010005F904F9008952F923F924F925F926F9210
:100020007F928F929F92AF92BF92CF92DF92EF9288
:10003000FF920F931F93CF93DF93CDB7DEB7C254D8
:10004000D1090FB6F894DEBF0FBECDBF4C015B01E6
:100050008A01322E1C8E1F8E19821C826115710539
:1000600011F410E0A3C0FC0183818111FACFFA01E1
:1000700080818F3209F098C0F501838182508230EF
:1000800058F0618D728DCE010196B1DB882349F362
:10009000CE0101967C0101C07501C8018C01019659
:1000A000F80120812F32D1F36E01FCE1CF0ED11C7B
:1000B0003601CE0101962C012396CFAE23972D2C2D
:1000C0009BE09150E7E3F0E0EC0FFD1FE90FF11D1D
:1000D00080E280839111F5CFD80127E04A2F3B2F92
:1000E0008D91811107C08FA9803209F4BACF842F76
:1000F000932F2CC08F32B9F38E3231F42A3009F4A9
:10010000B0CF98E02AE0EACFEEE6F6E1349133236F
:1001100021F031963813FACFA4CF291708F4A1CFD4
:10012000813208F49ECF8F3709F49BCF31E0390F2D
:10013000E7E3F0E0EC0FFD1FE90FF11D9FE9980FD9
:100140009A3108F480528083932FC8CF8C01FC0130
:10015000208101962F32D1F32223E9F021E0AE0174
:10016000495C5F4FB701C6016DDD882309F479CF83
:10017000EA14FB0411F0C7015DDDC614D70441F099
:1001800023969FAD2397822D7601C92ED82E98CF26
:10019000942D852DF9CF232DAE01495C5F4FB7011A
:1001A000C40150DD182F02C07B017ECFCE01019625
:1001B0000E944BC5CE014C960E944BC5812FCE5B51
:1001C000DF4F0FB6F894DEBF0FBECDBFDF91CF91EA
:1001D0001F910F91FF90EF90DF90CF90BF90AF9065
:1001E0009F908F907F906F905F904F903F902F9057
:1001F0000895CF93DF93EB01FC012381211102C00D
:1002000080E027C02250223020F48FE288831982B8
:100210001FC060E03FDB009799F3FC0190E080E0B5
:100220002EE23081303269F0883029F4DE01A90FE6
:10023000B11D2C939F5F3081DE01A90FB11D3C934E
:100240009F5F8F5F31968B3061F7C90FD11D188288
:1002500081E0DF91CF9108952F923F924F925F926C
:100260006F927F928F929F92AF92BF92CF92DF92C6
:10027000EF92FF920F931F93CF93DF93EC0142EF26
:1002800055E181E090E0FA0125913491C217D3073E
:100290000CF05DC09C0121503109220F331F220F49
:1002A000331FD901A051BA4EFD01659174912251BD
:1002B0003A4EF901A590B490FC01EE0FFF1FEE0F2E
:1002C000FF1FE051FA4EE590F490FD01C590D490E7
:1002D000FA0105911491F90125903490072E000C34
:1002E000880B990B0E946AF22B013C01CA19DB09A9
:1002F000BE01DD0F880B990B0E946AF24B015C0175
:10030000B7016C197D09072E000C880B990B0E9410
:100310006AF29B01AC01C501B4010E94C9F26B01F4
:100320007C01B80162197309072E000C880B990B28
:100330000E946AF29B01AC01C701B6010E9479F7E5
:100340009B01AC01C301B2010E949DF611C0019650
:100350004C5F5F4F8032910509F095CFECE6F6E1F6
:1003600065917491072E000C880B990B0E946AF21C
:10037000DF91CF911F910F91FF90EF90DF90CF9081
:10038000BF90AF909F908F907F906F905F904F90B5
:100390003F902F90089560918C0470918D0480910E
:1003A0008E0490918F0408954F925F926F927F9286
:1003B000AF92BF92CF92DF92EF92FF920F931F9373
:1003C000CF93DF93009709F456C0FC01208121FDF3
:1003D00052C0EB018C0147A050A461A472A4AFA04D
:1003E000B8A4C9A4DAA49501A601C301B2010E9470
:1003F00064F287FF40C0A3019201C301B2010E94D1
:10040000C9F22B013C01F80183A994A9A5A9B6A9B9
:10041000BC01CD0190589B01AC010E949DF6F801F2
:1004200027A530A941A952A90E94C9F29B01AC019C
:10043000C301B2010E949CF60E9408F97B018C0165
:100440009B01AC01B501C6010E9464F287FF02C0A6
:10045000750186019701A801B501C6010E9464F2E9
:10046000882349F0A701B8014FA358A769A77AA725
:10047000888181608883DF91CF911F910F91FF90D8
:10048000EF90DF90CF90BF90AF907F906F905F9094
:100490004F9008952F923F924F925F926F927F926A
:1004A0008F929F92AF92BF92CF92DF92EF92FF9284
:1004B0000F931F93CF93DF93CDB7DEB768970FB637
:1004C000F894DEBF0FBECDBF1C015B018A01DC01C9
:1004D000D7966D917D918D919C91DA970E9468F2EB
:1004E0006B017C01F50120813181428153810E94A1
:1004F000C9F20E9463F70E94E6F769877A878B87C3
:100500009C87D8012D913D914D915C91C701B60119
:100510000E94C9F20E9463F70E94E6F76D877E870A
:100520008F87988B29853A854B855C8528373105DF
:100530004105510540F488E790E0A0E0B0E08987EC
:100540009A87AB87BC872D853E854F85588928378C
:1005500031054105510540F488E790E0A0E0B0E0A6
:100560008D879E87AF87B88B91012D5B3F4FD90157
:100570008D919D910D90BC91A02D8D839E83AF8315
:10058000B887BC01CD010E946AF269837A838B83AC
:100590009C8369857A858B859C850E9468F2698B2E
:1005A0007A8B8B8B9C8B20E030E0A90169817A816A
:1005B0008B819C810E9464F2882339F1A701960106
:1005C000C701B6010E94C9F24B015C0129893A8931
:1005D0004B895C89CA01B9010E94C9F29B01AC0137
:1005E000C501B4010E949CF64B015C0129813A814E
:1005F0004B815C81CA01B9010E949DF69B01AC014F
:10060000C501B4010E9479F703C060E070E0CB013E
:100610000E9463F70E94E1F72B013C016D817E810E
:100620008F81988590958095709561957F4F8F4FBC
:100630009F4F0E946AF24B015C016D857E858F851C
:1006400098890E9468F26D837E838F83988720E06B
:1006500030E0A901C501B4010E9464F2882349F188
:100660002D813E814F815885CA01B9010E94C9F28E
:100670006D8B7E8B8F8B988FA7019601C701B6017A
:100680000E94C9F29B01AC016D897E898F89988D8A
:100690000E949CF66B017C01A5019401C501B40187
:1006A0000E949DF69B01AC01C701B6010E9479F73B
:1006B00003C060E070E0CB010E9412F8F101828873
:1006C0009388A488B58875016401C418D508E60824
:1006D000F7080E94E1F7C61AD70AE80AF90AF7FEF6
:1006E0006BC020E030E0A90169817A818B819C8117
:1006F0000E9464F2882309F447C029813A814B8122
:100700005C81CA01B9010E949DF66B017C01C501A3
:10071000B4010E9468F29B01AC01C701B6010E94BE
:10072000C9F26B017C0129893A894B895C89CA012C
:10073000B9010E94C9F29B01AC01C701B6010E9438
:100740009CF66B017C012D813E814F815885CA0149
:10075000B9010E94C9F29B01AC01C701B6010E9418
:100760009DF66B017C0120E030E040E850E46981B7
:100770007A818B819C810E94C9F29B01AC01C701E7
:10078000B6010E9479F703C060E070E0CB010E94DF
:1007900063F70E94E1F72B013C0197FF03C0412C56
:1007A000512C3201481459046A047B0410F02401CE
:1007B0003501C12CD12C76018FB7F894D1019C91D1
:1007C00093FD22C0F101468A578A608E718EC40C57
:1007D000D51CE61CF71C5A96CD92DD92ED92FC9248
:1007E0005D9729853A854B855C85DB962D933D93F6
:1007F0004D935C93DE97FF962D853E854F855889F6
:1008000020833183428353838FBF68960FB6F89459
:10081000DEBF0FBECDBFDF91CF911F910F91FF9033
:10082000EF90DF90CF90BF90AF909F908F907F9090
:100830006F905F904F903F902F900895CF92DF92EE
:10084000EF92FF9280918114882371F1C0907D1402
:10085000D0907E14E0907F14F090801420E030E07F
:10086000A901C701B6010E9464F28823E9F020E0E3
:1008700030E040E05FE3C701B6010E94C9F29B018E
:10088000AC010E94C9F22BED3FE049E450E40E9424
:10089000C9F29B01AC0160E070E080E89FE30E9438
:1008A00079F76B017C0106C0C12CD12C80E8E82EC1
:1008B0008FE3F82EC0922204D0922304E092240405
:1008C000F09225046091020270910302072E000C41
:1008D000880B990B0E946AF22AE037ED43E25CE351
:1008E0000E94C9F2A70196010E94C9F260931C02FE
:1008F00070931D0280931E0290931F02FF90EF9051
:10090000DF90CF90089591E09093C7043FB7F8949B
:100910002091320A9091330A3FBF291304C090916D
:10092000C00095FD3EC09091320A9F5F9F7120915B
:10093000330A921325C00FB607FCF9CF2091C000EF
:1009400025FFF5CF2091330AE22FF0E0EE5EF54F60
:1009500030812F5F2F712093330A3093C60020918E
:10096000C00020642093C0003091320A2091330AE5
:100970003213DDCF2091C1002F7D2093C100D7CF4E
:10098000E091320AF0E0EE5EF54F80832FB7F894E5
:100990009093320A8091C10080628093C1002FBF82
:1009A00008959FB7F8948093C6008091C00080643A
:1009B0008093C0009FBF08952F923F924F925F9205
:1009C0006F927F928F929F92AF92BF92CF92DF925F
:1009D000EF92FF920F931F93CF93DF93CDB7DEB7C4
:1009E000C456D1090FB6F894DEBF0FBECDBF6096D6
:1009F0009FAF8EAF609749AB59AF6EAF21967FAF77
:100A00002197322EDC01CD90DD90ED90FC9080910D
:100A1000620A9091630AA091640AB091650AC81AAB
:100A2000D90AEA0AFB0A6096EEADFFAD60974481F1
:100A30005581668177818091660A9091670AA091BD
:100A4000680AB091690A8A019B01081B190B2A0BDD
:100A50003B0B0DA71EA72FA738AB4085518562859C
:100A6000738580916A0A90916B0AA0916C0AB0918B
:100A70006D0A8A019B01081B190B2A0B3B0B0DAB5E
:100A80001EAB2FAB38AF4484558466847784809145
:100A90006E0A90916F0AA091700AB091710A530189
:100AA0004201881A990AAA0ABB0A09F496C08091E1
:100AB0000904811139C06091000270910102072E72
:100AC000000C880B990B0E946AF29B01AC016091AB
:100AD0008C0470918D0480918E0490918F040E94FB
:100AE00064F287FF21C040926E0A50926F0A6092B2
:100AF000700A7092710AE5EDF6E184918F010F5F43
:100B00001F4F882319F0FFDEF801F7CFE6EAF6E180
:100B100084918F010F5F1F4F882319F0F4DEF801D5
:100B2000F7CF812C912C5401C501B4010E946AF2C7
:100B300014E0319EF0011124E45EFD4F20813181EB
:100B4000428153810E94C9F20E94E1F72B013C01CE
:100B500097FF08C07094609450944094411C511CBD
:100B6000611C711C60911115709112158091131503
:100B7000909114150E94E1F79B01AC01A8ECB0E044
:100B80000E947DF664157505860597054CF56096FF
:100B9000EEADFFAD609784859585A685B78580937A
:100BA0006E0A90936F0AA093700AB093710AE5EDF4
:100BB000F6E184918F010F5F1F4F882319F0A3DEA8
:100BC000F801F7CFE7E8F6E184918F010F5F1F4F3F
:100BD000882319F098DEF801F7CF812C912C54016D
:100BE000D701C6018827B7FD83959927AA27BB2778
:100BF000182F2DA53EA54FA558A957FD12608DA908
:100C00009EA9AFA9B8ADB7FD1460B7FC1860C501C7
:100C1000B4010E946AF2A4E03A9EF0011124E45E5D
:100C2000FD4F20813181428153810E94C9F24B01E5
:100C30005C0120E030E0A9010E94C3F818164CF4D2
:100C400020E030E040E05FE3C501B4010E949DF682
:100C500008C0A501940160E070E080E09FE30E947D
:100C60009CF60E94E1F76AAF7BAF8CAF9DAF80919D
:100C7000720A8F5F8F706B968FAF6B978091730A3C
:100C80006B960FAD6B97801304C080E00E9467677E
:100C9000F5CFE091720A2E2F30E03CA72BA73FE45E
:100CA000E39FF0011124E251F14F108212A3D7010A
:100CB000C601F7FE07C088279927DC018C199D091A
:100CC000AE09BF0982839383A483B5838FE40BA508
:100CD0001CA5809FF001819FF00D1124E251F14F7E
:100CE0008DA59EA5AFA5B8A9B7FF07C0B095A095E3
:100CF000909581959F4FAF4FBF4F86839783A08775
:100D0000B1878FE40BA51CA5809FF001819FF00D9A
:100D10001124E251F14F8DA99EA9AFA9B8ADB7FF3B
:100D200007C0B095A095909581959F4FAF4FBF4F4D
:100D300082879387A487B5878FE40BA51CA5809F26
:100D4000F001819FF00D1124E251F14F2AAD3BAD2E
:100D50004CAD5DAD26873787408B518B42815381E7
:100D600064817581068117812085318504171507F7
:100D70002607370714F48A019B018FE4ABA5BCA5B5
:100D80008A9FF0018B9FF00D1124E251F14F828573
:100D90009385A485B58580179107A207B30764F4EE
:100DA0008AAD9BADACADBDAD80179107A207B3076F
:100DB00064F4D901C8010DC00AAD1BAD2CAD3DAD29
:100DC000081719072A073B0724F08AAD9BADACAD85
:100DD000BDAD2FE40BA51CA5209FF001219FF00DB8
:100DE0001124E251F14F828B938BA48BB58B069724
:100DF000A105B10510F40C94A390DF01A95BBF4FCE
:100E0000809191049091920411969C938E931296E6
:100E100080919304909194048D939C933182452BFF
:100E2000462B472B09F017988FE40BA51CA5809F34
:100E3000F001819FF00D1124E251F14F86819781DD
:100E4000A085B185892B8A2B8B2B09F016988FE40E
:100E50000BA51CA5809FF001819FF00D1124E2518C
:100E6000F14F82859385A485B585892B8A2B8B2BA1
:100E700009F015982AAD3BAD4CAD5DAD232B242B6D
:100E8000252BB1F08091380A882319F08150809386
:100E9000380A311004C0149880E28093380A3090E8
:100EA000460420904704009148041091490408C06A
:100EB0003090420420904304009144041091450472
:100EC000232D322DA80169A979AD8EAD21969FAD54
:100ED00021970E9464F287FD02C00C949B90C70189
:100EE000B6010E946AF22091D4043091D504409159
:100EF000D6045091D7040E94C9F22B013C01698BA2
:100F00007A8B8B8B9C8B6DA57EA58FA598A90E9453
:100F10006AF22091D8043091D9044091DA045091BA
:100F2000DB040E94C9F26DA77EA78FA798AB6D8BDB
:100F30007E8B8F8B988F6DA97EA98FA998AD0E940B
:100F40006AF22091DC043091DD044091DE0450917E
:100F5000DF040E94C9F26B017C01698F7A8F8B8F4D
:100F60009C8F2091E0043091E1044091E204509183
:100F7000E304C501B4010E94C9F26D8F7E8F8F8F8B
:100F800098A32FE44BA55CA5249FF001259FF00DAD
:100F90001124E251F14F82809380A480B58056E005
:100FA00085169104A104B104E4F486809780A0849E
:100FB000B184A6E08A169104A104B10494F4828459
:100FC0009384A484B584B6E08B169104A104B10483
:100FD00044F4DC01CB01BF7787A790ABA1ABB2ABE8
:100FE00034C0A3019201C301B2010E94C9F22B01D6
:100FF0003C012DA53EA54FA558A9CA01B9010E94E3
:10100000C9F29B01AC01C301B2010E949DF64B01E4
:101010005C01A7019601C701B6010E94C9F29B01BC
:10102000AC01C501B4010E949DF60E9408F92FE4AD
:101030004BA55CA5249FF001259FF00D1124E251E2
:10104000F14F67A770AB81AB92AB8FE4ABA5BCA5AA
:101050008A9FF0018B9FF00D1124E251F14F27A5DB
:1010600030A941A952A960E070E080E89FE30E94A6
:1010700079F726966CAF7DAF8EAF9FAF26979B0119
:10108000AC01632D722DC8010E94C9F26B017C0175
:101090008091720A9091730A891B8F7027968FAF87
:1010A0002797A701960160E074E284E799E40E9423
:1010B00079F70E94CEF84B015C0127968FAD2797F8
:1010C00082508630D0F580913E0490913F04A091EB
:1010D0004004B091410488169906AA06BB0668F53B
:1010E00088199909AA09BB09BC01CD01660F771FB0
:1010F000881F991F2796BFAD27970B2F10E020E080
:1011000030E0A90198010E943FF6CA01B9010E948E
:1011100068F20E94CEF8860E971EA81EB91EC50161
:10112000B4010E9468F29B01AC0160E074E284E7C4
:1011300099E40E9479F76B017C012FB7F8948091B4
:10114000CB0E9091CC0EA091CD0EB091CE0E880E0C
:10115000991EAA1EBB1E8092CB0E9092CC0EA0921E
:10116000CD0EB092CE0E2FBF8FE4EBA5FCA58E9FC7
:1011700080018F9F100D11240251114FD8019F96AD
:101180002D913D914D915C91D2976F962CAF3DAFD3
:101190004EAF5FAF6F97A70196016F966CAD7DADB7
:1011A0008EAD9FAD6F970E94C9F22E966CAF7DAF4A
:1011B0008EAF9FAF2E97F80163A374A385A396A368
:1011C00022893389448955892DA73EA74FA758AB5B
:1011D000CA01B9010E9468F26DAB7EAB8FAB98AFCC
:1011E000A70196010E94C9F20E9463F70E94E6F7E8
:1011F00064966CAF7DAF8EAF9FAF6497F80167AB1D
:1012000070AF81AF92AF8E010F5E1F4F1FAF0EAF59
:101210000051110966961FAF0EAF66970AE514E0FC
:1012200068961FAF0EAF68978E010F5D1F4F1AA70C
:1012300009A766960EAD1FAD669722961FAF0EAF3B
:101240002297212C312C10E819AB0FE309AFAEAD7A
:10125000BFAD6D917D918D919D91BFAFAEAFA70157
:1012600096010E94C9F22296EEADFFAD22976193DE
:101270007193819391932296FFAFEEAF22974B012A
:101280005C01E894B7F86896AEADBFAD68974D9035
:101290005D906D907D906896BFAFAEAF6897A301EB
:1012A0009201C501B4010E94C3F81816A4F4A50167
:1012B0009401C301B2010E9479F75B018C019B018B
:1012C000AC01B10189A999AD0E94C3F818161CF4AC
:1012D000150109AB19AF0EAD1FAD29A53AA502172F
:1012E000130709F0B4CF20E030E040E85FE3B1013C
:1012F00089A999AD0E9464F287FF4BC07E0131E15C
:10130000E30EF11C66960EAD1FAD6697910149A9DB
:1013100059ADD8016D917D918D919C910E94C9F23A
:10132000F80161937193819391938F01EE15FF05FD
:1013300069F78FE42BA53CA5829F8001839F100D48
:1013400011240251114F910149A959AD2E966CAD4E
:101350007DAD8EAD9FAD2E970E94C9F2D8019396B8
:101360006D937D938D939C93969764966CAD7DADB4
:101370008EAD9FAD64970E9468F2910149A959AD65
:101380000E94C9F20E94E6F7F80167AB70AF81AF27
:1013900092AF26962CAD3DAD4EAD5FAD26976DA9B3
:1013A0007EA98FA998AD0E94C9F269AB7AAB8BABCD
:1013B0009CAB8FE40BA51CA5809FF001819FF00DD5
:1013C0001124E251F14F82809380A480B580811472
:1013D0009104A104B10409F586819781A085B185A6
:1013E000892B8A2B8B2BC9F482859385A485B5859F
:1013F000892B8A2B8B2B89F42091651430916614EC
:10140000409167145091681469A97AA98BA99CA985
:101410000E94C9F20E9463F727C22AAD3BAD4CADD2
:101420005DAD232B242B252B49F06091691470911D
:101430006A1480916B1490916C1408C060916114CF
:1014400070916214809163149091641429A93AA94F
:101450004BA95CA90E94C9F20E9463F70E94E6F7BB
:101460006B017C018091C70E9091C80EA091C90EAE
:10147000B091CA0E0DA51EA52FA538A980179107FA
:10148000A207B30708F4E2C081149104A104B104D7
:1014900041F120914A0430914B0440914C04509109
:1014A0004D042C153D054E055F05D8F46DA57EA5B0
:1014B0008FA598A90E9430F62B013C01A701960147
:1014C000C501B4010E9430F6461657066806790633
:1014D00040F4C301B201A50194010E943FF66901E5
:1014E0007A018FE40BA51CA5809FF001819FF00D70
:1014F0001124E251F14F86809780A084B184811439
:101500009104A104B10441F120914E0430914F04A3
:1015100040915004509151042C153D054E055F0536
:10152000D8F46DA57EA58FA598A90E9430F62B0151
:101530003C01A7019601C501B4010E9430F6461690
:1015400057066806790640F4C301B201A50194016B
:101550000E943FF669017A018FE40BA51CA5809FCC
:10156000F001819FF00D1124E251F14F82849384A8
:10157000A484B58481149104A104B10441F12091A3
:1015800052043091530440915404509155042C1549
:101590003D054E055F05D8F46DA57EA58FA598A9DC
:1015A0000E9430F62B013C01A7019601C501B40150
:1015B0000E9430F6461657066806790640F4C301C5
:1015C000B201A50194010E943FF669017A018FE4FE
:1015D0000BA51CA5809FF001819FF00D1124E25105
:1015E000F14F86849784A088B18881149104A10466
:1015F000B10409F43DC12091560430915704409143
:101600005804509159042C153D054E055F0508F00E
:101610002FC16DA57EA58FA598A90E9430F62B013C
:101620003C01A7019601C501B4010E9430F646169F
:1016300057066806790608F01BC1C301B201A5016F
:1016400094010E943FF669017A0112C1811491044C
:10165000A104B104A9F160914A0470914B048091F6
:101660004C0490914D046C157D058E059F0540F549
:101670000E9468F22DA93EA94FA958AD0E94C9F257
:101680002B013C01C501B4010E946AF24B015C01CF
:10169000C701B6010E9468F2A50194010E94C9F237
:1016A000A30192010E94C3F8181654F4A5019401F5
:1016B000C301B2010E9479F70E94E6F76B017C0139
:1016C0008FE40BA51CA5809FF001819FF00D1124D4
:1016D000E251F14F46805780608471844114510477
:1016E00061047104A9F160914E0470914F048091DE
:1016F0005004909151046C157D058E059F0540F5B1
:101700000E9468F22DA93EA94FA958AD0E94C9F2C6
:101710004B015C01C301B2010E946AF22B013C0142
:10172000C701B6010E9468F2A30192010E94C9F2AA
:10173000A50194010E94C3F8181654F4A301920164
:10174000C501B4010E9479F70E94E6F76B017C01A4
:101750008FE40BA51CA5809FF001819FF00D112443
:10176000E251F14F428453846484758441145104DE
:1017700061047104A9F16091520470915304809145
:101780005404909155046C157D058E059F0540F518
:101790000E9468F22DA93EA94FA958AD0E94C9F236
:1017A0004B015C01C301B2010E946AF22B013C01B2
:1017B000C701B6010E9468F2A30192010E94C9F21A
:1017C000A50194010E94C3F8181654F4A3019201D4
:1017D000C501B4010E9479F70E94E6F76B017C0114
:1017E0008FE40BA51CA5809FF001819FF00D1124B3
:1017F000E251F14F86849784A088B18881149104C6
:10180000A104B104A9F1609156047091570480912C
:101810005804909159046C157D058E059F0540F57F
:101820000E9468F22DA93EA94FA958AD0E94C9F2A5
:101830002B013C01C501B4010E946AF24B015C011D
:10184000C701B6010E9468F2A50194010E94C9F285
:10185000A30192010E94C3F8181654F4A501940143
:10186000C301B2010E9479F70E94E6F76B017C0187
:101870008FE42BA53CA5829F8001839F100D11242E
:101880000251114FF801ED5BFF4FC082D182E2821D
:10189000F382C701B6010E9468F26B017C0129A99D
:1018A0003AA94BA95CA90E9479F76A966CAF7DAF03
:1018B0008EAF9FAF6A97D801D3966D937D938D932A
:1018C0009C93D69720E030E040E85BE4C701B60186
:1018D0000E94C9F220E034E244EF59E40E9479F713
:1018E0000E94E1F7F801668F778F80A391A3F3A19F
:1018F000F9AFD8019496BC91BEAFF801F5A121963D
:10190000FFAF2197D8019696BC912396BFAF23973E
:101910000AE614E0A1961FAF0EAFA1972E0111E1C8
:10192000410E511C4AE6242E44E0342E66966EACDD
:101930007FAC669709AD0AAF1EAD1DA7FDABB9AB75
:1019400010E0D3018D909D90AD90BD903D01E89445
:10195000B7F8F101C190D190E190F1901F01A7017A
:101960009601C501B4010E94C3F8181674F511233D
:1019700039F129AD3EAD21964FAD219723965FAD4C
:101980002397C701B6010E94C9F26B017C012AAD01
:101990003DA54DA959A9C501B4010E94C9F2A701ED
:1019A00096010E94C3F818167CF4A5019401C701A2
:1019B000B6010E9479F76AAF7DA78DAB99AB04C0E1
:1019C000CAAEDDA6EDAAF9AA11E06414750409F007
:1019D000B8CF27960FAD2797002309F455C1C090C3
:1019E0004E0AD0904F0AE090500AF090510A2DEB29
:1019F00037E346E855E3B601C7010E9464F287FD6C
:101A000043C19601A70169AD7EAD21968FAD2197A7
:101A100023969FAD23970E9464F287FD05C00C2D8D
:101A20002D2C3E2C1F2D08C009AD2EAC21963FACAD
:101A3000219723961FAD23979601A701602F722D42
:101A4000832D912F0E9479F7A5966CAF7DAF8EAF55
:101A50009FAFA59722E53AE062963FAF2EAF62971F
:101A600080E090E0A0E8BFE32A968CAF9DAFAEAFD8
:101A7000BFAF2A972B961FAE2B976296AEADBFAD28
:101A800062976D917D918D919D916296BFAFAEAF42
:101A90006297A5962CAD3DAD4EAD5FADA5970E946A
:101AA000C9F26B017C016696EEADFFAD6697819041
:101AB0009190A190B1906696FFAFEEAF66972B968E
:101AC000FFAD2B97FF23B1F02A962CAD3DAD4EAD67
:101AD0005FAD2A970E94C9F26B017C012A962CAD5A
:101AE0003DAD4EAD5FAD2A97C501B4010E94C9F26C
:101AF0004B015C01A5019401C701B6010E94C3F826
:101B000020E030E0A90118162CF5C501B4010E94AF
:101B1000C3F818164CF020E030E0A901C701B60167
:101B20000E9464F287FF05C0A5019401C701B601B8
:101B300024C02401350177FA709477F87094A301DA
:101B40009201C701B6010E94C3F818165CF5260180
:101B5000370128C0C501B4010E9464F287FD09C0A5
:101B600020E030E0A901C701B6010E94C3F81816B1
:101B70004CF4A7019601C501B4010E949CF62B010B
:101B80003C0110C02601370177FA709477F8709401
:101B9000A5019401C301B2010E94C3F8181614F004
:101BA00024013501A196AEADBFADA197CD90DD90DA
:101BB000ED90FD90A196BFAFAEAFA197A7019601A2
:101BC000C301B2010E94C3F81816ECF4A3019201FC
:101BD000C701B6010E9479F79B01AC012A966CAD52
:101BE0007DAD8EAD9FAD2A970E94C9F22A966CAF4B
:101BF0007DAF8EAF9FAF2A972B96BFAD2B97BF5F60
:101C00002B96BFAF2B976296EEADFFAD6297E25673
